:020000040800F2
:1000000000000220793F0608050406089907040845
:10001000294006082940060829400608000000007B
:100020000000000000000000000000004504060879
:1000300041040608000000003D0406086D6B050839
:1000400029400608294006082940060829400608D4
:1000500029400608294006085D7B05086D7B0508D8
:1000600029400608697B0508657B05080D1F060801
:10007000FD1E0608ED1E0608DD1E0608C91E060840
:10008000B51E0608A11E060829400608000000004B
:10009000000000000000000000000000617B050877
:1000A000BD1F0608951F06086D1F0608E51F0608F8
:1000B000591F0608451F0608311F06082940060873
:1000C0002940060829400608294006082940060854
:1000D00029400608592606084D260608000000009B
:1000E000597B0508294006084D2C06080000000031
:1000F0000000000000000000000000008D1E060847
:1001000000000000294006081D1F060829400608B7
:1001100000000000000000000000000000000000DF
:10012000791E0608651E0608511E06083D1E0608B3
:10013000291E06080000000000000000000000006A
:10014000000000000000000000000000C1120608CE
:10015000151E0608011E0608ED1D060829400608A2
:1001600029400608294006080000000000000000A1
:10017000000000000000000000000000000000007F
:1001800000000000294006080000000000000000F8
:08019000294006082940060879
:08019800183B06000100000005
:1001A000B01B01200208000003001423D01B012013
:1001B000020E000003001423F01B012001110000B7
:1001C00000007600101C01200112010000007700E1
:1001D000301C01200118000000001E00501C0120EE
:1001E000011E000000000D00701C0120011F000016
:1001F00000000E00901C01200120000000001E00E5
:10020000B01C0120011B000000000C00D01C0120CC
:10021000011C000000000E00F01C0120011D000068
:1002200000000C00101D0120022B010000012C0019
:10023000301D01200233000000012200501D01206A
:100240000134000000003C00701D0120013200005C
:1002500000004000901D0120013700000000200038
:0C026000B01D0120013800000000290042
:1080000009284FF0010307D903EB83035B00B0FBA2
:10801000F3F2092AF8D883B3F0B4DFF864C000257E
:108020000EE00A2A1E460F462346B4BF30245724CA
:108030002244092E01F1010105F101053A700FD921
:10804000ACFB0324E408B0FBF3F203FB1200002DA9
:10805000E7D1002AE5DC092B06D8303201F8012BE4
:108060000023F0BC0B707047ACFB0436B0FBF4F29D
:10807000234604FB1200F408EBE700230B70704763
:10808000CDCCCCCCF0B40D6800240CE0BCF1050FD5
:1080900018D8A0F137030A2B14D104EB840415F887
:1080A000010B03EB4404A0F13003DEB2092EA0F172
:1080B0006107A0F1410CF0D9052FE7D8A0F15703D3
:1080C0000A2BEAD00D601460F0BC704700B583B095
:1080D0000268074B8188CDF8012032221B68ADF879
:1080E00005108DF800206846984703B05DF804FB42
:1080F000C8150020204B2DE9F0415D68064600F1CF
:108100000708002406E01B68394698473C4446456A
:10811000A4B215D016F8017BA7F17D03012B2846E8
:108120002B684FF07D01EED81B6898472B6887F0CD
:1081300020011B6828469847E8E7E3B203EB1424C4
:10814000FF2CFAD8C4F1FF04E4B2A4F17D03012BA3
:108150002B6805D9214628461B68BDE8F041184721
:1081600028461B687D2198472B6884F0200128460B
:108170001B68BDE8F0411847C81500200A4AD369BA
:1081800030B41C6855695D6019810025611C196057
:108190009D812070D36951691A685A604FF6F67252
:1081A00030BC19609A817047C8150020084B242202
:1081B00003F12101016010B483F8202002683233FA
:1081C000541C5421C0E9004311705DF8044B704702
:1081D000C8150020F8B5CE1E0F4606440239421ECF
:1081E00004464FF6FF7312F8015F5B1BB2429BB26D
:1081F000F9D1C5194354064E1B0A05F8013C14F881
:10820000011B706B4EF048FDA542F8D1F8B2F8BDE5
:10821000C815002010B582B00B4660F05F001A0E42
:1082200008211C14ADF802308DF8010000236846C7
:108230008DF804408DF805208DF80010ADF806305B
:10824000FFF7C8FF02B010BD30B5062283B060F062
:108250005F030D460024114668468DF80130ADF8E5
:1082600002508DF80020ADF80440FFF7B3FF03B0D3
:1082700030BD00BF284A116821F0604323F07F031E
:10828000002B0CBF012002204B07536848BF04306D
:10829000D90744BF0A3080B29A0744BF143080B275
:1082A000D90544BF283080B25A0744BF643080B239
:1082B000190744BFC83080B29A0644BF00F5C870A1
:1082C00080B2D90644BF00F57A7080B2DA040FD5C7
:1082D00000F5FA5080B2990403D500F51C50103017
:1082E00080B29A050AD5A0F5C740403880B27047E1
:1082F00019050AD500F5FA6080B2ECE75B0503D5F5
:1083000000F59C40203080B270475A0644BF00F50B
:108310007A6080B2DFE700BF583D0120022805D017
:10832000A0F10100B0FA80F040097047054B93F8C6
:10833000403023B9044B1868C0F380007047102008
:1083400038F048B8C8150020583D012030B4054623
:108350000C482C6800F123039C424FF0000205D921
:1083600013F8011BA34282EA0102F9D1631C2B60BE
:1083700022702A6804496A60806F2960521A30BCF2
:108380004EF068BCC8150020E8150020014B93F89A
:108390007C007047C8150020F0B4434D434BC5F82E
:1083A0008030C823013885F8843005F1850205F155
:1083B000BF014D2428E0DCB25BB2002B34DB63004C
:1083C000DCB25BB2002B36DB6400E3B264B2002C9B
:1083D00038DB5C00E3B264B2002C3ADB5C00E3B251
:1083E00064B2002C3CDB5C00E3B264B2002C3EDBE8
:1083F0005C00E3B264B2002C4FEA4303B8BF83F0E1
:10840000D5038A42DCB238D010F8013F02F8013BB4
:10841000634013F0800F4FEA4303CCD083F0D504C0
:1084200063B2002BE4B2CADA640084F0D50463B20C
:10843000002BE4B2C8DA630083F0D5035CB2002CF1
:10844000DBB2C6DA5B0083F0D5035CB2002CDBB292
:10845000C4DA5B0083F0D5035CB2002CDBB2C2DA75
:108460005B0083F0D5035CB2002CDBB2C0DA5B00AA
:1084700083F0D5035CB2DBB2BDE70D4E85F8BF409B
:10848000A6F144070FCF0FC60FCF0FC60FCF0FC6F1
:1084900097E80F00402785F8C04086E80F0085F870
:1084A0000471F0BC704700BFC8150020C83E7BEACD
:1084B0008C16002070B5214D95F80531EA181C4640
:1084C00092F808218AB11E4E09225C1CA6FB0413F7
:1084D0005B0803EBC303E31AE918DCB291F8081157
:1084E00009B1013AF1D185F8054102681549561CD8
:1084F00006600C2616700268561C06600026167070
:108500000268561C066003EB430603EB86031470F7
:1085100019440D2255F0DAFE95F80511084B4A1C56
:10852000A3FB02035B08294403EBC3030120D31A16
:1085300081F8080185F8053170BD00BFC81500201D
:10854000398EE338DC16002038B504460D460A465D
:108550000068FF2161F037F921682944216038BDA6
:10856000026810B57F21541C046011700268002459
:10857000511C01600E211470FFF7E6FF012010BDB1
:1085800030B5324C94F88931012B85B001D005B05B
:1085900030BD94F88A01022826D0A0F10100B0FA7B
:1085A00080F0400948B36368002BF0D1D4F88C21E7
:1085B000002AECD094F8485094F8411092F9040045
:1085C000002D14BF08220022002908BF42F001023A
:1085D00003254FF46141CDE9015200911A46202153
:1085E0002EF084FA6060D2E794F84030DBB9184B83
:1085F0001868C0F380000028D5D16268002AC6D070
:10860000D4F89431934213D0D4F8A0319A420ED0CA
:10861000D4F8AC319A4214D0D4F8B8319A4212D07E
:1086200000236360B3E7102037F0D4FEBAE70120DF
:1086300000EB4000002104EB8003D162C3E9651127
:10864000EEE70220F4E70320F2E700BFC8150020A0
:10865000583D012070B51D4E1D4D96F8C80163228E
:10866000002157F095F8B6F8EC3104461948333B31
:1086700080FB0320DB17C3EB20100922002157F0F9
:1086800087F8AA68C0F10903642000FB0344A4B280
:10869000910744BF04F57A74A4B22B68D20744BF93
:1086A00004F5FA64A4B25B0701D4204670BD15201E
:1086B00037F090FE0028F8D06B6813F4016F04BF08
:1086C00004F57A64A4B2204670BD00BFC81500202E
:1086D000583D01201F85EB512DE9F047724C82B0C7
:1086E000E269D2E900239B1A002B00AF40F39B8084
:1086F000002384F808326D4B236103F18002A3F15B
:108700001406C4E97E33C4E90526C4E9E32203F56F
:10871000C075E5610025421800F10109C4E9029223
:1087200003785909012940F0858003F00F0813F000
:10873000100310D1002D00F0968094F89D130131A4
:1087400001F00F0141457ED01846083784F8083201
:10875000BD46BDE8F087831CA360C31C4278D4F8F3
:1087600010A0A3608078C6F800A00AEB0203736033
:10877000424084F89C23D4E90292002584F8081230
:108780003081B581A2EB0902D5B2A3EB0A0A5FFAE8
:108790008AFAEB1D03F4FC73AA45ADEB030D67D217
:1087A00052464946684660F0DBFD09EB0A03524633
:1087B00030466946A36055F089FD2369306894F816
:1087C0009C238342C6E9003009D00133336013F89B
:1087D000011C984282EA0102F7D184F89C23A36825
:1087E0001B78934232D12369E169C6E9003063699D
:1087F0004B600023A0690B818B813A1D84F80832FD
:108800007B603AF005F9013046D07B680BB100205F
:108810009847E3696269196801200837C3E90021B4
:10882000BD46BDE8F08794F80852002D3FF463AFD1
:10883000A66970E700210846FFF7A0FC0120083771
:10884000BD46BDE8F087D6E900A39BE70023B6F953
:10885000081084F808320120FFF790FC0120083747
:10886000BD46BDE8F08728460837BD46BDE8F0871D
:108870002A464946684660F073FD09EB0503304619
:108880002A466946A36055F021FD0020083784F888
:108890009D83BD46BDE8F087E26913680221581C3C
:1088A00010601970B1E700BFC8150020D417002070
:1088B0002DE9F04D2D4D2E4EB5F99E13B5F8A4C3FC
:1088C000B5F8A08386FB0146CC17C4EBA604A4B27E
:1088D000A44582B016461F4603D1B5F8A6334345DA
:1088E00033D003680190591C342201601A70036868
:1088F0000022591C01601A70214655F017FD01989D
:10890000414655F013FD019847F6FF7155F00EFDF5
:10891000019847F6FF7155F009FD019847F6FF7180
:1089200055F004FD019847F6FF7155F0FFFC0198E2
:108930000221FFF709FE0120C5E9EA67A5F8A44373
:10894000A5F8A68302B0BDE8F08DD5E9EA32B6EB12
:10895000030A67EB020B0023064A5B4508BF52453A
:10896000BFD3002002B0BDE8F08D00BFC8150020C5
:108970006766666680841E00604AD3682DE9F04110
:10898000064613F0800000F09A80906810F0020014
:1089900000F095805A4F97F8C811052940F293804E
:1089A000632900F28E800024DFF860C189B2254679
:1089B000ACFB0132D20802EB8203A1EB4303E0B22D
:1089C0008E469BB280008340BEF1090F91B245EA0A
:1089D000030504F10104EBD8EDB2D7F8D431494ACC
:1089E00082FB0312D917C1EB623189B2002900F072
:1089F00082804FF0000CDFF814E16446AEFB0132D8
:108A0000D20802EB8203A1EB43035FFA8CF08846A5
:108A10009BB280008340B8F1090F91B244EA03048D
:108A20000CF1010CEAD8E4B2B7F8E43136494FF45E
:108A3000F36213FB02F381FB0312D917C1EBA211FE
:108A400089B242F20F73994240D8C9B10027DFF8CA
:108A5000BCE0BC46AEFB0132D20802EB8203A1EBC4
:108A60004303F8B288469BB280008340B8F1090FF7
:108A700091B24CEA030C07F10107EBD81FFA8CF115
:108A800033681722581C30601A7033680022581C53
:108A900030601A70304655F049FC4FF0FF313046D7
:108AA00055F02CFC33685A1C32601D7033685A1C18
:108AB000326030461C700621FFF746FD0120BDE8FC
:108AC000F081992589E70020BDE8F0810020DFF8DA
:108AD0003CC00146ACFB0372D20802EB8207A3EB59
:108AE00047039BB283400430102841EA030193B24C
:108AF000F0D189B2C4E70C4696E700BF583D01208B
:108B0000C815002089B5F814D34D6210CDCCCCCC5B
:108B10002DE9F04FC14AD368804613F0800083B03E
:108B200000F06F81906810F0020000F06A81DFF8B9
:108B30000CB39BF8C831052B40F26881DBF8CC31CF
:108B4000B74D0093002BB8BF5B42A5FB0342B5486D
:108B5000B549920D00FB0233C3EB03139B0085FB69
:108B6000034502EB8202DC1702EB8202C4EBA55440
:108B700000FB043304EB8204A4B281FB0321DB1766
:108B8000C3EBA111BCB10025A84F2E46A7FB0432B0
:108B9000D20802EB8203A4EB4303E8B2A4469BB2E3
:108BA00080008340BCF1090F94B246EA030605F148
:108BB0000105EBD8340489B2B9B100259B4F2E468C
:108BC000A7FB0132D20802EB8203A1EB4303E8B218
:108BD0008C469BB280008340BCF1090F91B246EAFB
:108BE000030605F10105EBD83443DBF8D0E18C4DE9
:108BF0008C4E8D498EEAEE70A0EBEE70A5FB003234
:108C0000920D06FB0200C0EB0010830085FB0350B1
:108C100002EB8202DD1702EB8202C5EBA05506FBD8
:108C2000053305EB8205ADB281FB0321DB17C3EBF6
:108C3000A111C5B10020DFF8F4C10646ACFB053236
:108C4000D20802EB8203A5EB4303C7B2A9469BB24D
:108C5000BF00BB40B9F1090F95B246EA030600F127
:108C60000100EBD8350489B2C1B10020DFF8BCC1E6
:108C70000646ACFB0132D20802EB8203A1EB4303B0
:108C8000C7B289469BB2BF00BB40B9F1090F91B290
:108C900046EA030600F10100EBD83543DBF8D43196
:108CA000624A0193002B1846B8BF5842A2FB00301D
:108CB0005F4E6049030AA6FB0363DB0901FB03F176
:108CC000C1EBD00189B2B9B1002691463746A9FB64
:108CD0000132D20802EB8203A1EB4303F0B28C46CF
:108CE0009BB280008340BCF1090F91B247EA0307B1
:108CF00006F10106EBD8B9B2BBF8E671DFB1002688
:108D0000DFF828A1B446AAFB0732D20802EB82039F
:108D1000A7EB43035FFA86F938469BB24FEA89090D
:108D200003FA09F3092897B24CEA030C06F101068D
:108D3000E9D81FFA8CF7BBF8EC313C4AA2FB0306DA
:108D4000F608632E28BF6326092B63D900209346BB
:108D50008146ABFB0632D20802EB8203A6EB43034B
:108D60005FFA80FAB4469BB24FEA8A0A03FA0AF322
:108D7000BCF1090F96B249EA030900F10100E8D8F5
:108D80005FFA89F9009B019A002BCCBF3923382365
:108D90001616BEF1000F26F07F0635DD264A334356
:108DA000964543F00206C8BF43F00606D8F80030E7
:108DB0001622581CC8F800001A70D8F8003000229B
:108DC000581CC8F800001A70404655F0AFFA21460A
:108DD000404655F093FA2946404655F08FFA4046F2
:108DE000394655F0A3FAD8F800305A1CC8F80020CC
:108DF00083F80090D8F800305A1CC8F800200120F1
:108E00001E7003B0BDE8F08F1E43CFE7002003B013
:108E1000BDE8F08F4FF00009B4E700BF583D0120D6
:108E20006BCA5F6B806967FFD34D6210CDCCCCCC31
:108E3000C55A7C0AA0860100FFC99A3BC8150020CC
:108E400003687E22591C10B501601A700368002265
:108E5000591C01601A704FF6FF71044655F040FA34
:108E60000D4B93F8463083B127F0C4FA01462046F3
:108E700055F036FA204647F6FF7155F031FA204694
:108E80000821FFF761FB012010BD27F0C9FA014658
:108E9000204655F025FAEDE7C815002043090122C8
:108EA00000F01F00023B02FA00F0032B07D8DFE8B6
:108EB00003F0020C11070A4B5A6C104358647047B8
:108EC000074B5A6B104358637047054B1A6C10439D
:108ED00018647047024B1A6B10431863704700BF49
:108EE00000380240054BD3F8CC25B3F8D035516992
:108EF0000B4214BF53831383704700BFC815002073
:108F000080F0010101484EF0C5BD00BF941B002058
:108F10000B68144A30B40568CC682A402343D1E971
:108F2000054513432343D1E907242B4313434A6ADE
:108F30004D6B234313438C6BCA6A2B43234343F487
:108F40000033036044690B6B0D6924F0070413437D
:108F50002343D1E9014243614560846030BCC26073
:108F6000704700BF3F801CF030B403681A68537923
:108F70007BB159B2002920DB174C0120651803F0A2
:108F80001F03490900FA03F3302085F8000344F871
:108F9000213093797BB15AB2002A15DB0E480121AA
:108FA000841803F01F03520901FA03F3302184F8F7
:108FB000001340F8223030BC7047084903F00F031B
:108FC000194430230B76E4E7044A03F00F031A44F4
:108FD0003023137630BC704700E100E0FCEC00E089
:108FE00010B40B4C0023224601330A2B02F1140269
:108FF00009D011798142F7D103EB830304EB83009D
:109000005DF8044B704700205DF8044B704700BFCB
:10901000FC98060870B50B46ADF5815D0146144617
:109020000DF581501A460023CDE9010304AD6846D1
:10903000FD260393ADF80860009555F047F9009BB5
:10904000019320466946022200952AF031FE0DF573
:10905000815D70BD2DE9F047041E0D4612DB092C21
:1090600026DC824A0B468248A0FB0410C00800EBB5
:109070008000A4EB40000021125C1A705970284651
:10908000BDE8F08764422D23092C01F8013B24D868
:10909000764A774BA3FB0403DB0803EB8303A4EBC3
:1090A00043030020D35C48700B702846BDE8F0876E
:1090B0006F4B632CA3FB04264FEAD60621DC6B4AD8
:1090C0000B466B49A1FB0601C90801EB8101A6EB28
:1090D0004101515C03F8011BC5E7654A632CA2FB03
:1090E00004364FEAD60637D8604A614BA3FB060325
:1090F000DB0803EB8303A6EB4303D35C01F8013BDE
:10910000C7E7A3FB0627B4F57A7F4FEAD7070DD24E
:10911000564A0B465649A1FB0701C90801EB8101DC
:10912000A7EB4101515C03F8011BCAE7A3FB072829
:1091300042F20F7294424FEAD80836D84B4A0B4697
:109140004B49A1FB0801C90801EB8101A8EB4101D2
:10915000515C03F8011BDDE7A2FB0637B4F57A7F0B
:109160004FEAD7070CD2414A414BA3FB0703DB0868
:1091700003EB8303A7EB4303D35C01F8013BB4E7A4
:10918000A2FB073842F20F739C424FEAD80821D85D
:10919000364A374BA3FB0803DB0803EB8303A8EB3A
:1091A0004303D35C01F8013BDEE7324AA3FB080925
:1091B00094424FEAD90921D82C4A0B462C49A1FBED
:1091C0000901C90801EB8101A9EB4101515C03F8D8
:1091D000011BB5E7274BA2FB08099C424FEAD909BE
:1091E00021D8224A224BA3FB0903DB0803EB8303AC
:1091F000A9EB4303D35C01F8013BCAE71E4AA3FB7A
:10920000090394424FEAD30A21D80B461849174A5A
:10921000A1FB0A01C90801EB8101AAEB4101515CE4
:1092200003F8011BCAE7144BA2FB09029C424FEA58
:10923000D20A13D80E4B0D4AA3FB0A03DB0803EB3B
:109240008303AAEB4303D35C01F8013BCAE70A227C
:10925000BAFBF2F054F094FD0346D7E70A22BAFBBA
:10926000F2F054F08DFD0146E4E700BF0C2A070838
:10927000CDCCCCCC9F8601003F420F002DE9F047BA
:1092800088B0541C03941478002C00F04081002511
:10929000074688461E46A9460BE0791C02D02146A7
:1092A0003846C047039A0135531C03931478002CA9
:1092B00058D0252CF1D1931CCDE9033950782D28B5
:1092C00000F0C8804FF0000A302800F0AB80A0F119
:1092D0003003DBB2092B4FF0000440F2AF806C2862
:1092E0004ED0782838D8572840D9A0F15803202BE1
:1092F00032D8DFE813F0F4003100310031003100E2
:10930000310031003100310031003100DA0000015C
:109310003100C10031003100310031003100310035
:109320003100E3003100310031003100BB00310079
:10933000210031003100F40056F8040B05A9FEF7B6
:109340005FFE05ABCDE90043049B42464FF0FF3181
:10935000384655F0D5FA0544039A531C0393147804
:10936000002CA6D1284608B0BDE8F0870028F9D027
:109370002528F1D17B1C95D025213846C04791E79F
:10938000039B5A1C0392197878298DD8572967D9DD
:10939000A1F15803202B87D801A050F823F000BF7B
:1093A000C7940008A9920008A9920008A992000891
:1093B000A9920008A9920008A9920008A9920008A1
:1093C000A9920008A9920008A9920008AB9400088D
:1093D00003950008A992000879940008A992000852
:1093E000A9920008A9920008A9920008A992000871
:1093F000A9920008A9920008BF940008A992000849
:10940000A9920008A9920008A99200086D9400088A
:10941000A992000839930008A9920008A9920008AF
:10942000C7940008039B5A1C03921878A0F13003DC
:10943000DBB2092B4FF001043FF651AF04AA03A998
:10944000FEF720FEBAF1000F3FF449AF049B5B42E8
:10945000049344E7D31C039390784FF0010A33E759
:1094600000293FF47FAF252984D01DE756F8042B4F
:10947000049BCDE9009268E7073626F00706F6E878
:1094800002015AF03BFA00EE100A05A854F00EFC57
:1094900005ABCDE900434246049B4FF0FF3138460F
:1094A00055F02EFA039A0544FEE67A1C3FF4FAAE14
:1094B00056F8041B3846C9B2C047F3E6039A56F87B
:1094C000043B1D60F0E6A1F15802B2FA82F256F8B0
:1094D000040B520905AB102154F0AEFC31E7A0F1AA
:1094E0005802B2FA82F256F8040B520905AB102169
:1094F00054F0A2FC25E756F8040B05A954F058FCDB
:109500001FE756F8040B05A954F052FC19E725464D
:1095100028E700BF2DE9F04FD0F804C0DCF8103088
:10952000804665480E4691B017464FEA133E190A29
:1095300000256A01013583588EEA133481EA13232A
:1095400004F0030403F00F031C4307D0102DF0D1E7
:109550000020C8F80C0011B0BDE8F08F00EB020A43
:10956000DCF800309AF81C20C8F80CA01AB120468C
:1095700011B0BDE8F08FB3F84420504D6FEA42427D
:109580006FEA524292B2A3F844201A8892B242F093
:1095900080021A809CF805101A8C29444FF00109AA
:1095A00091F8C81009FA01F189B292B222EA0102D7
:1095B0001A841A8C92B2114319841A8892B242EA20
:1095C00009021A80504658F005FCD8F80CB00A235E
:1095D000AAF81C30584658F0FDFB9BF91430384A65
:1095E000CBF81880002BCBF80C205DDB354903F05D
:1095F0001F02C8185B094FF0300C09FA02F280F81C
:1096000000C341F82320D8F80C30986858F04CFB80
:10961000D8F80C309868036823F00103036058F011
:1096200043FB0023CDE90C33CDE90E33D8F80420F9
:1096300006930A935379032B05D8DFE803F0322F02
:109640002C0214684034127CD8F80C30029405EBDC
:1096500082059868D5F8CC3001934FF480614022A0
:109660004FF4003307914FF480454FF4805401A923
:1096700004920B93CDE9084505970396FFF748FC44
:10968000D8F80C309A681368012043F01003136077
:1096900011B0BDE8F08F14683C34D4E71468383456
:1096A000D1E714683434CEE7074A03F00F031A44B5
:1096B00030231376A7E700BF00000020FC980608BF
:1096C000D5C9050800E100E0FCEC00E0F8B5B44CB9
:1096D000B44DB54BC4F800560225B44AB44FB54E4C
:1096E000B54984F804564FF0A045C4F80856C4F8AC
:1096F000543605F51465A3F5DC63C4F80C26C4F8EC
:10970000147602F550726037C4F85066C4F8181623
:109710006036A1F5A461C4F81C56C4F8C836A5F596
:10972000886503F5B073C4F85826C4F82076A2F50E
:10973000C462A7F58467C4F85C66C4F81016A6F581
:10974000C06601F5C071C4F88C56C4F8A036C035A7
:109750009A4B9B48C4F89026C4F89476C03207F51B
:109760002C67C4F89866C4F89C1606F5D55601F522
:109770002A51C4F8A4564FF05025C4F8FC05C4F88B
:10978000A82600208F4AC4F8CC76C4F8D066C4F866
:10979000D41606F5C0460121C4F8D836C4F8DC5604
:1097A000A3F5485307F5C04704F2FC55C4F8E0267A
:1097B000C4F8E8660246C4F8E4760E4684F8071654
:1097C000C4F8083784F80E1784F8100701462B46B2
:1097D000402083F81C21A3F822210132042AC3E986
:1097E000490183F81D6183F81F11C3F8301103F19B
:1097F0002803EED1002211462B46402083F8742323
:10980000A3F87A230132042AC3E9DF0183F8751330
:1098100083F87713C3F8881303F12803EED14FF0D0
:10982000A04369489A6822F001029A60DA6842F01F
:109830004002DA6057F0A4F894F80536002221219E
:1098400061F317420BB142F4801294F8FF15D4F87B
:10985000083601299A6307D19A6822F03E0141F047
:109860002A0161F307029A60DA68D4F80867D4F82D
:109870000C06C2F3076121F0600141F0400161F381
:109880001F620021DA603160026861F3CC2202605D
:1098900094F80726012A10D101684C4A4C4E41F039
:1098A00003010160802159629E62C3F804214FF4D4
:1098B000A072C3F80821C3F80C211021454857F0C5
:1098C000B1FB444857F094FBD4F80C6694F8FD358E
:1098D00000204FF0FF3230617061B261F06143B33C
:1098E00005F114073C4A07EB83074FEA830E4FF05C
:1098F000FF0C52F8043F19680029ACBF00214FF05B
:109900009041BA4219601861C3F808C0F1D15035CE
:10991000324A75440027FF2052F8043F1968002995
:10992000ACBF00214FF09041954219601F619860D3
:10993000F2D1336994F8FF1543F480730129336140
:109940001ED0D4F80826264800294FF000036FF0F7
:1099500080414FF0FF349361516108BF1023546080
:109960005161906143F47013916943F4605343F083
:1099700008030B439361936843F001039360F8BDC0
:10998000D4F80826174B33636FF080411448002346
:109990004FF0FF3493615161546051619061E1E790
:1099A000C815002040004001200B00500008005066
:1099B00000090050000B00502009005000400050EA
:1099C0000804010000600050D01B0020C00080008F
:1099D00080004000C41B0020D81B0020141C002065
:1099E000000800800301810030B51C4B5021082283
:1099F00083B083F84313C3F88820BFF34F8FBFF3BE
:109A00006F8F174D174C2B6B43F001032B634FF4F3
:109A1000C05240F2023369462046CDE9002358F097
:109A2000F3F8636A104A23F470436362636A43F491
:109A300020436362636A23F470236362636A43F4BE
:109A4000202363626B6C43F480436B646B6B012176
:109A500043F080036B63516103B030BD00E100E06F
:109A60000038024000000240003C014010B5802157
:109A7000044656F0E9FC2046002156F0E5FC20465D
:109A8000BDE8104056F0A2BF2DE9F041B24C94F869
:109A9000033CC4F8F00B82B088465A2B00F2B98020
:109AA000DFE813F0CC00B700B700DC00B700B70068
:109AB000B700B700B700B700B700B700B700B700EE
:109AC000B700B700B700B7001D01B700B700B70077
:109AD000B700B700B700B70041017400B700B70086
:109AE0007400B700B700B700B700BA01B70064014F
:109AF000B700B7007C00B700FE01B700B700B700A1
:109B0000B7005B00B700B700B700B700B700B700F9
:109B1000B700B700B700B700B700B700B700B7008D
:109B2000B700B700B700B700B700B700B700B7007D
:109B3000B700B700B700B700B700B700B700B7006D
:109B4000B700B700B700B700B700B700B700B7005D
:109B5000B700B700B700B700E60194F8043C9B07D4
:109B600000F15082B4F80A3CD4F8052CD4F8441C17
:109B70005BBA9BB212BAD0188842C4F8503CC4F801
:109B80004C2C03D956F040FC002854DB0020A4F8EC
:109B90003C0C0546284602B0BDE8F08194F8483CEC
:109BA000002B40F0018194F9003C002B31DAD4F80D
:109BB000383C08469B689847002840F00782B4F874
:109BC0000A0CD4F8052CD4F8443C40BA80B212BA3E
:109BD00015189D42C4F8500CC4F84C2C07D956F007
:109BE00013FC002827DBD4F84C2CD4F8500CD4F804
:109BF000403CD4F8FC6B00FB03F002FB03F20225AF
:109C0000B042C4F84C2CC4F8500C84F8485C00F006
:109C1000D18094F8143C5A1CD2B204EBC303052043
:109C20004FF40051042A84F8142C83F8180CC3F85C
:109C30001C1C00F095814FF0FF35ABE7D4F8FC3BDE
:109C4000002BE6D1D4F8383C08469B689847054677
:109C5000002840F0BB81A4F83C0C9BE73F4B00225E
:109C600003F1120103F8012F8B42FBD13C4994F818
:109C70003E3C94F8140C70250D7098424FF00C0582
:109C8000CD7110D004EBC300013390F8185C8D70D7
:109C9000B0F81C0CDBB2042B40BA888114BF84F8E6
:109CA0003E3C84F83E2C94F8073C12229342A4F8E0
:109CB0003C2C0FD8A4F83C3C00256BE7B5F5805F41
:109CC00028BF4FF48055D4F8F00B254AABB20121E0
:109CD00056F0B4FC0025284602B0BDE8F08194F8A7
:109CE000043CDA0700F12581D4F8383C94F8070CDD
:109CF000DA6901EBC10102EB81010A79531D83424C
:109D000028BF0346A4F83C3C002BE3D0013B144899
:109D10009BB201331944034411F8012D03F8012DBE
:109D20008342F9D1D6E70F480F4E01460823073882
:109D3000C1F10705A4F83C3C002202E092F8F420AF
:109D400019460B46814203F8012905EB030216FA76
:109D500082F2F3D1BEE700BFC81500204F470020B4
:109D60005047002057470020FC980608D4F8383C9C
:109D7000BB4A5B680846111D98470546002840F01D
:109D80002581D4F8443CB74AD4F8401C013B180E56
:109D90001070180C09BAD37050701B0A0820937009
:109DA0005160A4F83C0CF5E6D4F8506CD4F84C2C77
:109DB000D4F8403CD4F8385CB2FBF3F24FF480574F
:109DC000BE4228BF3E462D69A649A4F83C7C4046C9
:109DD000B6FBF3F39BB2A8470028C0F2AF8033462E
:109DE000A04AD4F8F00B812156F062FBD4F84C2C39
:109DF000D4F8500CD4F85C3C3244851B9E1BC4F84C
:109E00004C2CC4F8505CC4F85C6C002D7FF462AF3D
:109E1000032384F8483CBDE6924F00263B4607F1F9
:109E20000C0203F8016B9A42FBD1D4F8383C40464F
:109E30005B686A4601A998470546002840F0D08033
:109E4000019BBDF80020013B190E52BAFB7139711C
:109E5000190C1B0A79710820BB7102217A810C232D
:109E6000BDF80220F87039727A72A4F83C3C91E691
:109E70007D487E4E014608230738C1F10705A4F846
:109E80003C3C002202E092F8FC2019460B46884236
:109E900003F8012905EB030216FA82F2F3D119E760
:109EA00094F8483C002B61D194F9003C002BFFF65C
:109EB000B0AED4F8383C08469B689847002840F07C
:109EC0008580D4F8383C4046DB6898470546002832
:109ED00040F0AC80B4F80A3CD4F8052CD4F8440C1B
:109EE0005BBA99B212BA53188342C4F8501CC4F832
:109EF0004C2C00F29180D4F8403CD4F8FC0B03FBCE
:109F000002F203FB01F38342C4F84C2CC4F8503C2A
:109F10007FF47FAEB3F5805F28BF4FF480530121FB
:109F2000D4F8F00B4F4A84F8481C9BB256F086FBDD
:109F300030E607234E49A4F83C3CE7E694F8143C8D
:109F40005A1CD2B204EBC30304204FF4885182425E
:109F500084F8142C83F8180CC3F81C1C7FF46BAE27
:109F6000002384F8143C4FF0FF3513E6D4F8506C0E
:109F7000D4F8380CD4F8403CD4F84C2C4569B2FBEA
:109F8000F3F2B6F5805F28BF4FF480560846B6FB63
:109F9000F3F334499BB2A847002856DBD4F84C2C85
:109FA000D4F8505CD4F85C3C3244AD1B9B1BC4F825
:109FB0004C2CC4F8505CC4F85C3C002D7FF47EAEA1
:109FC000D4F8F00B294656F08DFBE3E594F8143CE9
:109FD0005A1CD2B204EBC30302204FF4685121E6AD
:109FE00094F8143C04EBC3020133DBB202204FF4BB
:109FF0006851042B82F8180CC2F81C1C20D084F87D
:10A00000143C18E694F8143C5A1CD2B204EBC30377
:10A0100005204FF4105105E656F0F6F90028FFF63A
:10A020000AAED4F84C2CD4F8501C64E794F8143CD5
:10A030005A1CD2B204EBC30302204FF41C51F1E5C9
:10A0400084F8146C4FF0FF35A4E594F8143C5A1CC6
:10A05000D2B204EBC30304204FF4407177E700BF92
:10A06000082200205047002057470020FC9806088F
:10A07000E899060870B50020FEF742FF0D4B0E4D23
:10A0800001244FF40676184601211BB1DE801C72B4
:10A090004CF08CFE032C08D055F8243001210134FB
:10A0A0001846002BF2D1032CF6D1BDE870400020F9
:10A0B000FEF726BF941B0020009A060899B10A6B90
:10A0C000824216D9154BD3F8942C914221D34C39A6
:10A0D00091421ED30B6B9842F9D38B6B9842F6D802
:10A0E0000B46184670470D4BD3F8941C0A6B9042F0
:10A0F00012D30B680BB9F4E70A6B90420B4602D3FC
:10A100008A6B9042EDD951F84C3F002BF4D11846A0
:10A1100070470023184670470A46D8E7C815002044
:10A120002DE9F047CC0143D10346224A43F8082BDE
:10A130004FF0FF324260022418467E26DFF8788016
:10A14000D8F8989C2644013E051D49466FF070479B
:10A150004FF0010A08E0A3421CD0631C45F8043C00
:10A16000321B1C460435CAB10B6BA34202D88B6B61
:10A17000A34204D22046FFF7A1FF014690B10A791D
:10A180004B6B002AE7D1A34204D0E6D245F8042C59
:10A19000631CE5E745F8047C631CE1E7C8F8981CFC
:10A1A000BDE8F08745F804AC321B631C4946D8E78C
:10A1B0008026C3E7F8FFFF0FC815002070B50546DD
:10A1C000144895F91030AA6803EB830300EB83036E
:10A1D0009207D3F800620C4610D5D4E90123216818
:10A1E000304658F0ADFDD4E90423E168304658F01C
:10A1F000A7FDAB689B0708D5012070BD68694CF0CE
:10A20000A7FE08204CF09CFCE7E728464DF0E8FD4F
:10A21000012070BD000000202DE9F04F2DED108BC6
:10A22000034693B004331193DFEDC1AA10900223CB
:10A230000F928B460E938946109C4FEADB0504EB88
:10A24000451202EB0511A5EB85034FEAC5084FEA5D
:10A25000051E05EB850A009101EBC30308F104001C
:10A260000EF104012E46204405EB450521444FEA3A
:10A27000CA040D9602942C01C6EBC60C0394EC00A4
:10A280000D9D04944FEACC0405946C010194119D3A
:10A29000009C03EB46174FEACB0A02EBC6064FF0D1
:10A2A000000C55ED011A11ED012AD6ED005AD7ED3B
:10A2B000004A92ED003AD4ED003A10ED015A93EDC8
:10A2C000004A72EE238A34EE248A71EE836A35EEF8
:10A2D000257A36EEA86A77EE087A35EE655A76EE7C
:10A2E000275A36EE676A45ED015A82ED006A90ED15
:10A2F00000AAD6ED012A93ED016AD7ED019A94EDFB
:10A30000010AD1ED005AD5ED007A92ED019A34EEB2
:10A31000644A76EE690A7AEE624A35EEC01A31EE88
:10A32000C33A72EE633A34EEA02A77EEC91A74EE9D
:10A33000E04A75EE805A75EE440AB0EE410A35EEF9
:10A34000045AA2EE2A0ADC44E145A2EE6A1AB0EEF3
:10A35000434AB0EE432AA0EEAA2AA0EEEA4AB0EEA3
:10A36000613AF0EE610AE4EEAA0AA4EEEA3AF0EEEF
:10A37000634AE5EE6A3AE5EE2A4A7AEE222A36EE9A
:10A38000296A77EE897A72EE861A37EE487A32EECB
:10A39000C66A76EEE86AB0EE635A77EEA53A77EED3
:10A3A000E57A73EEA18A36EE868A73EEE13A76EEAE
:10A3B000C66A77EEC71A72EE002A77EE277A74EE35
:10A3C000015A30EEE46A33EE457A32EE402A34EE3A
:10A3D000414A74EEA04A35EE035AC5ED008AC2ED3B
:10A3E000013A554401ED018A5244C4ED006AC1EDC1
:10A3F000001AC4ED017A514440ED012A544487ED1E
:10A40000002AC6ED005A83ED004A80ED006AC7EDD0
:10A41000014A504486ED017A574483ED015A56446F
:10A4200053443FF63EAF0D9B072B40F2A3810198AA
:10A43000109D059B049A0399029C08302818083344
:10A440000A902846C318083282180593034608F17B
:10A4500008080EF10C0E0C3308340831069202463F
:10A46000454472440419411804934B460995D1465A
:10A470000894079103924FF001084FF0000E9A469E
:10A480000E9B9E440F9B03EBCE0303EBCE0202EB2D
:10A49000CE0000EBCE0404EBCE0505EBCE060C930C
:10A4A00006EBCE07AEEB8E030B9207EB031202EB2B
:10A4B000CE0C0CEBCE03029203EBCE0201931346BB
:10A4C000D3ED01DA019BD0ED007A93ED01DA029B26
:10A4D000CDED027A93ED01CA0B9BDCED01CAD3ED01
:10A4E000007A0C9BCDED017A02EBCE0202EBCE019D
:10A4F000009201EBCE02D3ED007A92ED01FA009AC0
:10A50000D1ED01EA92ED01EAD7ED00BA96ED00BA7D
:10A5100095ED00AAD4ED009ACDED007ADDE9037641
:10A52000DDE90554DDE90701DDE90923C44601E061
:10A53000F304353F91ED006A56ED01FAD0ED002AA3
:10A54000D4ED005AD5ED006A93ED007A57ED017A0B
:10A5500092ED002A96ED008A7FEE870A32EE061A07
:10A5600037EEA24A75EEA64A70EE841A31EE245AEE
:10A5700032EE462A31EE856A75EEE65A06ED016A3C
:10A58000D4ED018A92ED019A91ED013A95ED016ABF
:10A5900097ED000AD0ED016AD3ED013A3FEEC77A9C
:10A5A00077EEE27A78EEC6FA79EE432A39EE033A8C
:10A5B00030EE669A38EE866A70EE266A78EE638A26
:10A5C00032EEEF0A72EEAF2A78EE233A30EEC44A4A
:10A5D00032EE258AF0EE490A72EE655AE2EEAA0AD8
:10A5E000DC44E245A2EEEA9AB0EE682AF0EE472A91
:10A5F000E5EEAA2AA5EEEA7AA0EE2A2A73EE065A1A
:10A60000E0EE6A8AF0EE67FA33EEA60AE8EE6A7ABE
:10A6100071EE644A31EEC55A33EE463A70EE651A71
:10A6200073EEE63A34EE036A72EEA06A34EE434A01
:10A6300072EEE00A33EEE43AE8EE2AFA74EEA33A58
:10A6400065EE6D2A77EE094A37EE499A38EEE77AD9
:10A6500077EEA88A6DEEA17A9DED018AE9EE857A02
:10A66000E9EEA12A26EE6C5A6CEE831A32EE6F1ACE
:10A67000A8EE035AE8EE061A2EEEA33A24EE6E6A0E
:10A680009DED008A3FEE822AABEE043AABEE236AE0
:10A690002CEE014A66EECC3AA8EE264AE8EE013AE4
:10A6A0006FEE026A20EECF1AEBEEA06AABEE821AD2
:10A6B00064EECE0A2EEE072A9DED028AEAEE070A24
:10A6C000AAEE242A2DEE287A69EE4D4AA8EE097AE0
:10A6D000E8EE284A70EE255AC6ED005AC3ED007A1E
:10A6E000C3ED012A4E4447ED011A87ED005A4B4451
:10A6F00080ED003A80ED016A4F4482ED004AC2EDE0
:10A70000013A4844C5ED006A85ED011A4A4481EDDD
:10A71000002A4D44C1ED010A84ED007AC4ED014ADE
:10A7200049444C443FF606AF0A9B08330A93099B01
:10A7300008330993089B08330893079B0833079352
:10A74000069B08330693059B08330593049B083347
:10A750000493039B083303930D9B08F101084345C1
:10A760007FF48EAE0E9BDDF834B0DB009BB2D14699
:10A770000E9361E513B0BDEC108BBDE8F08F00BF08
:10A78000804BB3FBF2F399420DD300234FF07E527E
:10A7900043608360C360036102600023836143619F
:10A7A0000362C361704707EE902A9FED777AF8EE57
:10A7B000676A07EE901A66EE876AF8EE677A66EEC9
:10A7C000A76AFDEEE67A17EE903A2033402B00F2AE
:10A7D000CA80DFED6E7AF4EEE76AF1EE10FAF0EE81
:10A7E000667A0CDDDFED6A5A9FED6A6AB0EE677A31
:10A7F000B4EEC67AF1EE10FA77EEE57AF6DC9FED6C
:10A80000667AF4EEC77AF1EE10FA0CD5DFED605AF5
:10A810009FED626AB0EE677AB4EEC67AF1EE10FA96
:10A8200077EEA57AF6D49FED5E7AF4EEC77AF1EE74
:10A8300010FA00F390809FED5B7AF4EEC77AF1EEA8
:10A8400010FA44BF9FED547A77EE677A27EEA76A35
:10A85000DFED554A9FED557A9FED555ADFED555A7C
:10A86000A6EE247A67EE864AA6EE075AB6EE007A7E
:10A87000E6EE055AE4EEA57A27EE877A9FED486A60
:10A8800076EE867AFDEEE75A15EE903A2033402BAD
:10A8900066D8F4EEC66AF1EE10FA0CDDDFED3C5A34
:10A8A0009FED3C6AF0EE676AF4EEC66AF1EE10FACC
:10A8B00077EEE57AF6DCDFED386AF4EEE67AF1EE73
:10A8C00010FA0CD5DFED325A9FED346AF0EE676A6C
:10A8D000F4EEC66AF1EE10FA77EEA57AF6D4DFED63
:10A8E000306AF4EEE67AF1EE10FA3FDDDFED276A2A
:10A8F00076EEE77A67EEA76ADFED2B4A9FED2B5ADB
:10A90000DFED2B5A9FED2B6AA6EEA45A67EEA64AFE
:10A91000E6EE855AB8EE005AA6EEA56AE4EE867A0F
:10A9200067EE857AC7EE006AB7EE006A76EE865A61
:10A9300076EE666A86EE257A67EE277A66EE876A95
:10A94000C0ED017AC0ED037A80ED007A80ED027AE5
:10A95000C0ED046A21E79FED0D7A77EE677A75E71F
:10A96000DFED157ADEE79FED147A87E7DFED0D6AFC
:10A97000F4EEE67AF1EE10FA44BFDFED076A76EE08
:10A98000E77AB7E720A1070027D4D236DB0F49408A
:10A99000DB0FC940E4CB1641DB0F49C0E4CB16C145
:10A9A000DB0FC93FDB0FC9BF9A7C2E36FAAF4FB918
:10A9B0003587083CA4AA2ABE000000000023034AF1
:10A9C000426003608360C360704700BF83F9223E2A
:10A9D00010B40549054A064B4160002404608260BA
:10A9E0005DF8044BC36070475B128B3A6F12033BF8
:10A9F0008943273F034B6428B8BF6420C3F804068B
:10AA0000704700BF00000020034B64281B69B8BFDB
:10AA10006420D860704700BF583D01202DE9F04701
:10AA200090B0DDE918480E460746914601A83C2241
:10AA300000219A461A9D5EF0C6FE2E4B8DF80460EA
:10AA4000CDF834800293002E50D0B31E012B4FD985
:10AA5000042E14BF00230323DFF89C808DF80530FB
:10AA6000D8F8E03C03941C440123CDE90557049435
:10AA70008DF83130B9F1000F06D05246494607A88B
:10AA80005EF06EFC8DF830A098F8E6EC0023BEF185
:10AA9000010F0E931CD801AC0FCC98F8E5CCCCEB91
:10AAA0000C1508EB850505F6E8450FC50FCC0FC55D
:10AAB0000FCC0FC594E80700BCFA8CFC0EF1010E18
:10AAC0004FEA5C1C85E8070088F8E6EC88F8E5CCDE
:10AAD0003B6843B153464A463146384610B0BDE85C
:10AAE000F0472BF059BB10B0BDE8F0870523B3E762
:10AAF0000223B1E768220020C8150020002303606C
:10AB0000704700BF0023094980ED010A01228162DC
:10AB100002708360C3604361036183634363C36303
:10AB2000C362036303648361436470470000204190
:10AB300030B4174B1749C3F8841D03F55A6500213B
:10AB40001224154A154883F8684D83F8641D42F6AF
:10AB5000F82403F66851C3F8945D0025C1E9024565
:10AB6000C3F8880D30BC0120C3F8A02DC3F8A42D74
:10AB7000C3F8A82DC3F8AC2DC3F8B02DC3F8B42D7D
:10AB8000C3F8B82DC3F8BC2DC3F8C02D704700BF63
:10AB9000C8150020F1BB0208E003E003FDBB02087A
:10ABA000074B0849D3F8942DC3F8841D931E4FF426
:10ABB0007871223223F8021F9342FBD1704700BF05
:10ABC000C8150020D9B7020870B5244E244BC6F82A
:10ABD000843D11244FF4787506F6C8534FF478700D
:10ABE00086F8684D4FF47874C3E90045C3E902451F
:10ABF000C3E90445C3E90645C3E90845C3E90A4575
:10AC0000C3E90C45C3E90E451649C6F8080E84B0E1
:10AC100006F6685241F60B2400254020C2E90245A1
:10AC2000C6F8881D2CF02CF9B0B196F8133E0E4AE8
:10AC300090F904000092012B0CBF0822002203238C
:10AC4000CDE901324021094A00232BF04FFFC6F81D
:10AC50002C0E003818BF012004B070BDC8150020AC
:10AC60000DC3020805C40208A068060019D0020836
:10AC700070B40D4B0D4CA34203D311E00C33A3422F
:10AC80000ED25A798242F9D1DA798A42F6D11A681B
:10AC90001E791579AE42F1D115689D42EED100E0E2
:10ACA0000022104670BC7047A00100086C0200082A
:10ACB000642828BF64201C4B00EB800070B5450061
:10ACC000A3FB05235E095B0918BF002422D00134D1
:10ACD0009F204DF0D7FAE3B29E42F8D80A2E00D159
:10ACE00070BD1248A0FB05300009C6EB8613C6EB09
:10ACF000830366381844C0B24DF0C4FA092E06F139
:10AD00000104EDD001349A20E4B24DF0BBFA0A2CD4
:10AD1000F8D170BD0548A0FB053000096638C0B207
:10AD20004DF0B0FA0124EDE71F85EB51CDCCCCCC32
:10AD3000F0B41A4E96F8303E032B2CD80C2202FBAE
:10AD4000036202F6386252F8041C0133CC07DBB20E
:10AD50000ED501420CD092F90070114C002194F9EB
:10AD60000050BD4204F10C040BD001310429F6D18E
:10AD7000042B02F10C02E6D186F8303E0020F0BC34
:10AD8000704701EB410106EB810186F8303ED1F8B6
:10AD90009401F0BC70470020F1E700BFC815002007
:10ADA000581700200144884218D030B4441E4D1E6C
:10ADB000002041F2210114F8012F082380EA02202B
:10ADC00010F4004F81EA40020ABF400090B280B206
:10ADD000013BF5D1AC42EED130BC7047002070474A
:10ADE000D0ED017AF5EE407AF1EE10FA05D19FED43
:10ADF0000C7AF0EE477A80ED017A30EEA77AD0ED4A
:10AE0000007AC0ED020AC0EE876A30EE670AC0ED34
:10AE1000036AE6EE807AB0EE670AC0ED007A70470A
:10AE200083F9223EBCEEC00A7F4AB2FBF1F210EE7B
:10AE3000103A9BB2934208D300234FF07E524360F6
:10AE40008360C36003610260704707EE901A9FED54
:10AE5000777AF8EE676A07EE903A66EE876AF8EE60
:10AE6000677A66EEA76AFDEEE67A17EE903A20332F
:10AE7000402B00F2CA80DFED6E7AF4EEE76AF1EE65
:10AE800010FAF0EE667A0CDDDFED6A5A9FED6A6A21
:10AE9000B0EE677AB4EEC67AF1EE10FA77EEE57AA4
:10AEA000F6DC9FED667AF4EEC77AF1EE10FA0CD577
:10AEB000DFED605A9FED626AB0EE677AB4EEC67A53
:10AEC000F1EE10FA77EEA57AF6D49FED5E7AF4EE05
:10AED000C77AF1EE10FA00F390809FED5B7AF4EE02
:10AEE000C77AF1EE10FA44BF9FED547A77EE677A95
:10AEF00027EEA76ADFED554A9FED557A9FED555A2B
:10AF0000DFED555AA6EE247A67EE864AA6EE075A7A
:10AF1000B6EE007AE6EE055AE4EEA57A27EE877AD9
:10AF20009FED486A76EE867AFDEEE75A15EE903A86
:10AF30002033402B66D8F4EEC66AF1EE10FA0CDD31
:10AF4000DFED3C5A9FED3C6AF0EE676AF4EEC66AAC
:10AF5000F1EE10FA77EEE57AF6DCDFED386AF4EE22
:10AF6000E67AF1EE10FA0CD5DFED325A9FED346A35
:10AF7000F0EE676AF4EEC66AF1EE10FA77EEA57AA3
:10AF8000F6D4DFED306AF4EEE67AF1EE10FA3FDD4A
:10AF9000DFED276A76EEE77A67EEA76ADFED2B4AE8
:10AFA0009FED2B5ADFED2B5A9FED2B6AA6EEA45A8C
:10AFB00067EEA64AE6EE855AB8EE005AA6EEA56AF6
:10AFC000E4EE867A67EE857AC7EE206AB7EE006A0D
:10AFD00076EE865A76EE666A86EE257A67EE277AF0
:10AFE00066EE876AC0ED017AC0ED037A80ED007AE3
:10AFF00080ED027AC0ED046A70479FED0D7A77EE1E
:10B00000677A75E7DFED157ADEE79FED147A87E75B
:10B01000DFED0D6AF4EEE67AF1EE10FA44BFDFEDF3
:10B02000076A76EEE77AB7E720A1070027D4D23681
:10B03000DB0F4940DB0FC940E4CB1641DB0F49C0B1
:10B04000E4CB16C1DB0FC93FDB0FC9BF9A7C2E369C
:10B05000FAAF4FB93587083CA4AA2ABE0000000009
:10B06000D0ED015A037830EE605AF0EE407A65EE8A
:10B07000255A002B47D190ED0C7A37EE607AD0ED4F
:10B080000A4AC0ED0C0AF5EEC04AF1EE10FAC7EE1E
:10B09000016A3DDC90ED037A26EE877A90ED056A31
:10B0A000D0ED0B6A27EE866A67EE222A76EE267AC4
:10B0B00077EEA57A77EEA27AF4EEE17AF1EE10FA65
:10B0C00048D4F4EEC27AF1EE10FA8CBFB0EE420A28
:10B0D000B0EE670A70EE677AD0ED044A90ED027A1E
:10B0E000C0ED0D6A67EEA47AC0ED0E5AE5EE077A60
:10B0F000C0ED0F2AE1EE276A80ED106A80ED110A9B
:10B10000C0ED0B6A704700239FED147A0370B6E719
:10B1100090ED076A90ED034AB5EE406AF1EE10FA41
:10B1200005D19FED0F7A87EE246A80ED076A31EE34
:10B13000066A90ED067A80ED081AC1EE064A76EEB0
:10B14000C76AC0ED094AA4EEA67A80ED067A24EE1D
:10B15000077AA3E7B0EE610ABCE700BF0000000079
:10B1600083F9223E70B4344890F8683EA3F1300170
:10B17000092957D800F66864224600F6776012F86D
:10B18000015FA5F13001092904D88242F7D10020DE
:10B1900070BC7047141B022C4ADD2848002101E0D6
:10B1A00010F8013B01EB810103EB4103161A303B20
:10B1B000022E044603F0FF01F2DC214B03FB01F1F8
:10B1C000A2424FF000030DD903EB830314F8016B87
:10B1D0005B00303B3344A24203F0FF03F4D1194833
:10B1E00000FB03F32E2D06D01748A0FB032301EB31
:10B1F000930070BC7047013204200024157804EBE2
:10B200008404303D6400092D00F1FF30A4B202D85F
:10B210002C44A4B2013210F0FF00EFD1642202FBF3
:10B220000433E1E700211D4600F668620B46D9E7CA
:10B23000064C0021C4E700BFC815002031240020BF
:10B240008096980040420F00ABAAAAAA30240020A2
:10B250009B1A00FB03F090FBF1F01044704700BF15
:10B26000094BD3F8780ED3F87C2ED3F8803E824277
:10B2700002DB114602460846984204DD9A42B8BFF6
:10B280001A46104670477047C815002030B4144A5B
:10B29000D2F8840ED2F8883ED2F88C4ED2F8901EA6
:10B2A000D2F8942E834202DB1D46034628468A428A
:10B2B00002DB15460A4629468842A8BF0846934243
:10B2C000B8BF1346A04202DC224604461046834221
:10B2D00003DAA342B8BF2346184630BC704700BF0C
:10B2E000C81500200B6810B414681B1B0360546859
:10B2F0004B681B1B43608B6892685DF8044B9B1A7C
:10B30000836070472DE9F041804684B008461646B8
:10B3100052F016FF4FF47A72002304460D4658F09F
:10B320004BFCB6F900C00746294620464FF47A7216
:10B330003C2400230CFB047758F03EFC002594B21B
:10B340004FF47A73C3FB07452B46224601A852F0FF
:10B3500043FE404B93F89A3E012B2FD0022B10D185
:10B360009DF80670FB1E082B0BD83B1F062B1BD924
:10B37000BDF80400394652F0C5FD032F36D00B2F1F
:10B3800041D022462B46404652F026FE04B0BDE88E
:10B39000F081032F55D00A2FF3D19DF80870B7FA2A
:10B3A00087F77F09002FECD033882B4A3C33A41851
:10B3B0004FF00002338042EB0505E2E79DF806708E
:10B3C000FB1E072BDDD83B1F052BEDD9BDF8040074
:10B3D000394652F097FD9DF807309842D9D0033F87
:10B3E00018BF0127002FDFD1CBE707380E28FCDC80
:10B3F0009DF80730834212D0CCBF01270027002FD1
:10B40000D2D1BEE707380728FCDC9DF8073083421D
:10B410000ED0B4BF01270027002FC5D1B1E79DF89A
:10B420000870012F94BF00270127002FBCD1A8E787
:10B430009DF80870012F8CBF00270127002FB3D182
:10B440009FE79DF80870003F18BF0127002FABD180
:10B4500097E700BFC815002080EE36002DE9F041C7
:10B46000274B86B09C1D1E4603F160081F464FF017
:10B47000000C94F800E0A0EB0E05A0EB0C02002DF0
:10B48000B8BF6D42002AB8BF52429542B8BF2746A6
:10B4900004F10604B8BF4FFA8EFCA045E9D17C88C0
:10B4A00003F15A0E002204E02546B64516D016F8E0
:10B4B000062F6245F8D1B6F80280A1EB08020B1BFB
:10B4C000002AB8BF5242002BB8BF5B4293422546C8
:10B4D000EBDDB645444645463746E8D17E793C79B2
:10B4E00002953A78019200910346CDE90346054A58
:10B4F0000321012054F02CFB384606B0BDE8F08152
:10B500000C9A0608342A0708074BD3F8A42ED3F860
:10B510009C1ED3F8A00EC3F89C0E5242C3F8A01E86
:10B52000C3F8A42E704700BFC815002030B50468CA
:10B53000E46985B02CB10DF10F050095A04705B069
:10B5400030BD204605B030BD38B50A4C0A4D232128
:10B55000D5F8A80E50F04AF914F8011F0029F7D1C8
:10B56000064850F07DF995F8AC3E13B1012385F8FB
:10B57000AD3E38BD702A0708C81500207C2A070890
:10B580002DE9F04F89B0CDE90621DFF8B0800746FC
:10B5900099460026069B002B07DBB34205D00136F7
:10B5A000042EF7D109B0BDE8F08FF22303FB06FBB0
:10B5B000079B03EB0B0A204B00249B44B9F1000FBF
:10B5C00033464246384601DBA14530D13BF81450A2
:10B5D0003AF81410009415F4006FA1EB050114BFA4
:10B5E0004FF0560E4FF0480E05F01F0CB1FA81F1E6
:10B5F000C5F344154909CDE901C5CDF80CE0059125
:10B6000047F0B6FC3AF814300599009413F4006F33
:10B6100003F01F0214BF56204820C3F34413CDE9A2
:10B620000123039033464246384647F0BDFC0134BF
:10B63000792CC3D1B3E700BF782400208C2A0708F7
:10B640002DE9F04F3B4C3C4B94F8E85A3B4ADFF86D
:10B65000F4808946002D08BF1A4694F9E91A8BB088
:10B660000746374846F00EFA04F5A9644D46002611
:10B67000B9F1000F3ED022782B789A426A683BD00D
:10B68000D5E902CE0021A87D0790B5F914000690F7
:10B69000B5F912000590B5F910000093CDE903E06B
:10B6A000CDE9012C334642463846099147F060FC0B
:10B6B0000999A37D6268B4F914B0B4F912A0B4F981
:10B6C00010E0D4E9020C079314F8183B0093CDE97D
:10B6D00001203346CDE905ABCDE903CE4246013624
:10B6E000384647F061FC3C2E05F11805C0D10BB07F
:10B6F000BDE8F08F4946DCE76168D5F808C09142A3
:10B7000002D0D5F80CE0BDE7A168D5F80CE06145A2
:10B71000B8D1E1687145B5D1206929698842B1D1B4
:10B720006069696920F07F4021F07F418842A9D19A
:10B730000121A8E7C0260020A82A0708AC2F070887
:10B74000AC2A0708BC2A07081D4A2DE97003546972
:10B750001C4E002CD6F8F83503600EDD183200239D
:10B7600006F5BF6501E09C4207D052F8041BA942D0
:10B7700003F10103F7D1012200E00022D6F80436DC
:10B7800083600271104A96F8083643711346F3E855
:10B790000289D3E90045D6F8283652F8042CD6F8A9
:10B7A000201681625B0943EAC2635209C0E9048939
:10B7B000C0E90645C0E90832BDE87003704700BF24
:10B7C000583D01200000002030060020014BD3F836
:10B7D0007802704700000020014BD3F8080370473F
:10B7E00000000020014BD3F8C00270470000002089
:10B7F0000C4608B505462BF04FF920462BF04CF9C6
:10B800000020FDF77DFB28464BF020FAB0B920461A
:10B810004BF01CFA0028F6D00120FDF771FB204602
:10B820004BF00CFA014628464BF036FA0020FDF7A3
:10B8300067FB28464BF00AFA0028E8D00120FDF704
:10B840005FFB28464BF0FAF9014620464BF024FAFC
:10B850000020FDF755FBDAE7F0B50023C1E900331E
:10B86000C1E902330B610268DFF88CC089B004AD16
:10B87000C2F385572E4647FA03F0C007344604D575
:10B8800013F80C0004F8010B26460133062BF2D105
:10B890001748C2F303240444002394F8784133701A
:10B8A0008DF8184000F5C07CC2F305370DF119067C
:10B8B00047FA03F0C007344604D513F80C0004F827
:10B8C000010B26460133062BF2D100233370C2F35D
:10B8D000834406ABCDE90134084602F00F03054965
:10B8E0000095C2F3031252F02BFD09B0F0BD00BF6A
:10B8F000FC980608DC2A07086C9A060870B51F4EEB
:10B9000096F8D4342DED028B04460D467BB3D6F861
:10B91000E014D6F8E424D6F8DC340360C0E9011260
:10B9200006F59B6393ED008ADFED158A95ED000A1D
:10B9300080EE280A5AF01AFF23681844206028EE87
:10B94000288A95ED010A80EE080A5AF00FFF636815
:10B950001844606095ED020A5AF008FFBDEC028BB6
:10B96000A3680246134496F8D404A36070BDC0E9EE
:10B9700000338360B7EE008AD6E700BFC026002000
:10B980002C7D8E3FF0B4244B93F8D45482B03DB953
:10B990000023036043608360284602B0F0BC704718
:10B9A0004C68D3F8DC7401940C68D3F8E0649FED24
:10B9B0001B6AE71B019CA41B07EE904A03F59B64DE
:10B9C000D4ED006A07EE107A66EE866AB8EEC77AA2
:10B9D000F8EEE77A27EE067A67EEA67A012A80ED7E
:10B9E000007AC0ED017A0DD08A68D3F8E434D21A17
:10B9F00007EE902AF8EEE77AC0ED027A284602B008
:10BA0000F0BC7047D1ED027AF8EEE77AC0ED027A29
:10BA1000284602B0F0BC7047C02600202C7D8E3F27
:10BA200010B4414A92F8A530D2F88C00023BD2E91A
:10BA30002114062B74D8DFE803F05A5C60500655D9
:10BA4000040064424942404280EAE073A3EBE073A1
:10BA500006EE903A84EAE473A3EBE47307EE103A3F
:10BA6000F8EEE66A9FED316AB8EEC77A26EE866A8E
:10BA700081EAE173A3EBE17307EE903AB4EEC76A93
:10BA8000F1EE10FAF8EEE77A04DDB4EEE76AF1EED3
:10BA900010FA34DC9FED256A27EE066AB4EEE76AF9
:10BAA000F1EE10FA04DDF4EEC66AF1EE10FA2DD4D0
:10BAB0009FED1E6A67EE867AB4EEE77AF1EE10FA31
:10BAC0002BD5F4EEE76AF1EE10FA26D50029CCBFAB
:10BAD000042005205DF8044B70474B42404221464C
:10BAE0001C46B1E7634240420C461946ACE7494266
:10BAF000AAE74B4261421C46A6E76442A4E700283D
:10BB0000CCBF002001205DF8044B7047002CCCBF57
:10BB1000022003205DF8044B70474FF0FF30D9E757
:10BB200023460C4619468FE7583D0120ABAA2A3F11
:10BB300070B5294B294C93F8151E93F8163EDFED8E
:10BB4000286A94F81C2BD4F8405B07EE101A07EE15
:10BB5000903AB8EEC77AF8EEE77A27EE267A67EEE3
:10BB6000A67A04EB4206BDEEC77A0132FDEEE77A13
:10BB700002F00F01B6F8203B84F81C1B17EE102AC8
:10BB800017EE901AC31A2B448A42C4F8403B82B085
:10BB9000A6F8200B4FEA131312DC17EE101A17EE5B
:10BBA000902A98B240F2FF350023009553F0CEFD65
:10BBB0002A46002153F0ECFDA4F8440B02B070BDFE
:10BBC0009BB29942D4BF581A00208242A6BF101AD5
:10BBD00080B20020E6E700BFC8150020C026002084
:10BBE00014AE2341064B93F8911103F2844203F201
:10BBF0006C43002918BF134693ED020A704700BF3B
:10BC0000C02600202DE9F04F2DED028B87B00446B1
:10BC1000324D039310460E46B0EE408A174657F059
:10BC2000D9F9D5F848BB9DF848A0DBF800308BF86F
:10BC30000B604FF0000820448BF80A00CDF800801C
:10BC400058463246D3F814B09DF84C903B462146F6
:10BC5000D8479FED230A039B019328EE000A534621
:10BC6000FDEEC07ACDF8008017EE901A424604A887
:10BC700012F0C4FDD5F84C3B13B11B784B452AD0CC
:10BC8000D5F8583B13B11B784B4524D0D5F8643B0D
:10BC900013B11B784B451ED0D5F8703BCBB11B7848
:10BCA000A3EB0909B9FA89F94FEA5919384657F04F
:10BCB00091F901340444E1B2D5F8480BCDF8009075
:10BCC00004AB32464BF0B4FF07B0BDEC028BBDE8CD
:10BCD000F08F9946EAE74FF00109E7E7C026002018
:10BCE0000000C84230B41C7884B1012C0CD1B3F9E7
:10BCF00002408AB1157B94FBF5F40470B3F904306B
:10BD0000527B93FBF2F30B7030BC70479A78027051
:10BD1000DB780B7030BC7047054A82FB0452E41795
:10BD2000C4EB62040470B3F904301222E9E700BFE7
:10BD3000ABAAAA2A30B41C784CB1012C05D1B3F9B6
:10BD40000220B3F9043002600B6030BC70479C786D
:10BD500052B1157BDB7815FB04F40460527B03FBC6
:10BD600002F330BC0B60704704EB4404A400DB78A2
:10BD700004601222F3E700BF30B583B00C460546DD
:10BD800001920FF08DF8019B224629464CF006F8EF
:10BD9000094A92F97C3B02EB430101335BB2352B3C
:10BDA000C8BF0023012081F8805B81F8814B82F8B5
:10BDB0007C3B03B030BD00BFC02600200F4B93F882
:10BDC000342D012A12D910B582B004220C888B7848
:10BDD0008DF804000DEB02017420ADF805408DF8DC
:10BDE00007302BF063F9012002B010BD01D0002014
:10BDF000704793F8353D622BE5D8F8E7C026002060
:10BE0000F8B5214D1D260C46074685F85C6D2AF0D5
:10BE100065FD00202AF0EEFC08202AF0EBFC0E2045
:10BE20002AF0E8FC30462AF0E5FC04202AF0E2FC87
:10BE300004202AF0DFFC00202AF0DCFC30202AF06D
:10BE4000D9FC00202AF0D6FC20462AF0D3FC0020A2
:10BE50002AF0D0FC2AF024FD05F556602AF02EFCCD
:10BE600000B9F8BD95F8603D63B995F8613D302B98
:10BE700000D03BB995F8623D23B995F8633D3B701E
:10BE80000120F8BD0120F8BDC02600202DE9F04FAB
:10BE9000DFF8F4822DED028B00220023C8E93A235B
:10BEA000002387B008F1F0011A4601F8332001336E
:10BEB000122BFAD1B14CB24DDFF8D092DFF8D0A2FC
:10BEC0009FEDB08A04F5407605F188070DE007EB99
:10BED000C303227853F8883C02B16BB900232B606E
:10BEE0001834A64205F1080541D094F90130002B21
:10BEF000EDDA2378002BF1D02B79DB07F0D4A168A1
:10BF0000207927F043FC21698346207B27F03EFC03
:10BF1000A2780346282AE1D8DFE812F039006F0042
:10BF20005400680083008C005200340013021B028E
:10BF30002102470229022E0236023E0296009F008D
:10BF4000AA00B300C300D300ED00B101B901BF01E5
:10BF5000D601DC01E201E801F1010602FF0008015F
:10BF600021013C01610170017F01A201760097F877
:10BF7000883013B197F88A309BB907B0BDEC028BBB
:10BF8000BDE8F08FBBF1000FA8D00028A6D0237D1C
:10BF900001222A60DA07A3D52B7943F001032B7124
:10BFA0009EE797F88920D7F88C0040214CF086F85E
:10BFB000002387F88A3007B0BDEC028BBDE8F08F14
:10BFC00040F282639B45D4BF4FF0000B4FF0010B52
:10BFD000237DC5F800B0DB0782D5BBF1000F3FF42D
:10BFE0007FAF2B7943F001032B7179E78345ACBF19
:10BFF0004FF0000B4FF0010BEAE7ABEB000BBBFA85
:10C000008BFB4FEA5B1BE3E70028E1D09BFBF0F0E2
:10C0100047F6FF7203FB10B0494653F0B9FB834665
:10C02000D6E740F234539B45CCBF4FF0000B4FF0A6
:10C03000010BCDE7ABF2355BBBF5A77F2CBF4FF013
:10C04000000B4FF0010BC3E700FB0BF047F6FF724C
:10C05000494653F09DFB8346BAE70028B8D09BFBC6
:10C06000F0F047F6FF72494653F092FB8346AFE784
:10C070005FFA8BF01946009327F062FB009B9B460A
:10C08000A6E75FFA8BF201901046009227F072FB50
:10C09000019B009A03EB000B5946104627F050FB1A
:10C0A00096E75FFA8BF201901046009227F062FB50
:10C0B000019B009AA0EB030B5946104627F040FB6A
:10C0C00086E75FFA8BFBBBF1070F00F27381C2B208
:10C0D000003A97F8891018BF01220120524200FA55
:10C0E0000BFB4A4002EA0B024A409B4687F8892034
:10C0F00087F88A006CE7D8F8E830227D43F0010326
:10C10000C8F8E830D0074FF001032B607FF5E8AEA8
:10C110002B7943F001032B71E2E6D8F8E830C8F838
:10C1200000B243F08003C8F8E83051E707EE90BA58
:10C13000B8EEE70A002808BF4FF4FA7320EE080AA9
:10C14000009353F08FFC009B07EE903AF8EEE77AED
:10C1500027EE800AFDEEC07A17EE90BA38E707EEB8
:10C1600090BAB8EEE70A002808BF4FF4FA7320EE41
:10C17000080A009353F0FCFBE5E700BF30340020D1
:10C180003037002035FA8E3C583D01200080FFFFFB
:10C190001F85EB5107EE90BAF8EEE78A002868EEAB
:10C1A000888A08BF4FF4FA73B0EE680A009353F020
:10C1B00059FCF0EE407AB0EE680AF0EE678A53F070
:10C1C000D7FBC8EE807A009B07EE103AB8EEC77A2C
:10C1D00067EE877AFDEEE77A17EE90BAF8E61A4630
:10C1E00058460021009353F0D3FA009B00221946D1
:10C1F0004FF47A73FFF72CF88346E9E600904FF48A
:10C200007A725846002153F0C3FA009B00224FF483
:10C210007A71FFF71DF88346DAE6009011220BF1E0
:10C22000FF30002153F0B4FA009B08EBC00B184616
:10C2300001234FF4FA624FF47A718BF8F03053F027
:10C24000A7FAD8F8E820217DCBF8F400012342F4C6
:10C250008072C9072B60C8F8E8203FF59DAE3FE625
:10C26000642000FB0BF053F0ABFA8AFB003BC017D5
:10C27000C0EB6B1B0FFA8BF02CF09CFEA8E6D8F8F5
:10C28000E830227DC8F8DCB143F0020338E7D8F883
:10C29000E830227D43F0040332E7D8F8E4319B45CF
:10C2A0003FF41CAEB86F02A94AF07EFB002846D0CE
:10C2B00058469DF80A20012153F06AFA8346C8F8CF
:10C2C000E40187F87E0083E6D8F8E830227D43F069
:10C2D000080315E7D8F8E830227D43F010030FE794
:10C2E000D8F8E830227D43F0200309E7D8F8E83099
:10C2F000C8F8F4B143F04003C8F8E83068E6D8F86D
:10C30000F8319B453FF4EAADB86F02A94AF04CFB07
:10C31000A8B158460522012153F03AFA8346C8F8DD
:10C32000F80187F87C0053E6D8F8FC319B453FF4D0
:10C33000D5ADB86F02A94AF037FB00283CD1286080
:10C34000CEE5BBF1000F7FF422AE00287FF41FAED4
:10C35000C5E5BBEB000B18BF4FF0010B38E6BBF196
:10C36000000F3FF414AE00283FF411AEB6E5BBFA5F
:10C370008BFB4FEA5B1B2BE6BBF1000F7FF407AE94
:10C3800028BBD5F800B023E6584447F6FF7249466B
:10C3900053F0FEF983461BE6ABEB000047F6FF7255
:10C3A000494653F0F5F9834612E65BEA03033FF48E
:10C3B000EEAD93E583460BE658460822012153F083
:10C3C000E7F98346C8F8FC0187F87D0000E6C5F868
:10C3D00000B085E5164991F8682E32B3F0B40646F0
:10C3E00000200346074602E092F8682EDAB100EB1F
:10C3F00080002E2A4FEA400004D10133CA1832448B
:10C4000082F8687ECA18A0F1300592F8682EA2F171
:10C410003004092C98BF50190E2B03F1010301EBD6
:10C420000302E1D90020F0BC70470020704700BF34
:10C43000C815002070B5174DD5F8902013791E3B14
:10C44000012B064603D9104600214AF025FC002E98
:10C4500009DD114C264414F8011BD5F890004AF070
:10C460001BFCA642F7D195F8E7306BB90B4AB5F83B
:10C47000F030D2F8E02CC5F8E82001330022A5F80E
:10C48000F030C5F8EC2070BDD5F8900000214AF0DE
:10C4900003FCEBE7B83700204C380020C81500201B
:10C4A00010B50A4C04F6EC2009F0D6FBD4F8F83AA3
:10C4B000C01A53F091F90028B8BF404242F21073FD
:10C4C0009842D4BF0020012010BD00BFC02600202C
:10C4D00038B5084CB4F8625131F07CFF854205DD77
:10C4E000054BB4F86221A3F82A2238BDBDE83840D4
:10C4F00008F0F4BEB8370020583D0120036813F05F
:10C50000400004D013F4057F14BF012000207047C1
:10C510002DE9F043244D254C85B005F128098046CE
:10C520000F461646C4F8989DC4F8945DFEF738FB94
:10C530001F4BC4F8883D122284F8682D04F6685118
:10C5400042F6F82200234020C1E902232AF098FC99
:10C55000044610B3FFF7D2FF98F800203F78034657
:10C5600094F9040000961C1E14BF03210121002A27
:10C570000CBF07220622012F0CBF082300231A43F9
:10C58000CDE901124B460B4A40212AF0AFFAA5F53E
:10C59000BC752CB9003818BF012005B0BDE8F08388
:10C5A000C5F8E001F6E700BF30390020C8150020CB
:10C5B0004DB90208C9C802080348044A00F61361CD
:10C5C00000F61260A4E700BFC8150020400D03006C
:10C5D0000348044A00F6136100F6126098E700BFB2
:10C5E000C8150020A086010070B5C44CD4F8E461E1
:10C5F00084B02EB13046FFF781FF002840F06D81F6
:10C6000094F8F001FBF78AFE94F8E831834205467E
:10C610001CD0002800F07E81C6B1B94B96F9040009
:10C6200093F84120B2FA82F252094FF416510023D6
:10C630000225CDE9015200911A4604212AF056FA4A
:10C64000C4F8EC0110B1012384F8E83194F8F10149
:10C65000FBF764FE94F8F231834205461ED00028B1
:10C6600000F01881D4F8F431C3B1A54A93F904005D
:10C6700092F84820002A18BF08224FF49641002360
:10C680000325CDE9015200911A4608212AF02EFA1D
:10C69000C4F8F80110B1012384F8F231FBF770FF00
:10C6A000D4F8FC512DB12846FFF728FF002840F0B0
:10C6B000FA8094F80802FBF731FE94F800328342C6
:10C6C000064631D0002800F02E818D4E96F84B3072
:10C6D000012B00F03681022B0CBF8A4A8A4AC4F82B
:10C6E00004220DB32A7A002A00F02881022A00F0E1
:10C6F0002C81012A40F03781824BC4F804324FF478
:10C70000966395F90400009300250221019102959A
:10C710002B462A4610212AF0E9F9B06720B10123FF
:10C7200084F8095284F8003294F80A02FBF7F6FD07
:10C7300094F80B328342054636D0002800F0A180E1
:10C74000D4F80C32D3B11A7A002A00F0F4806F4981
:10C7500001EB8202D2F8882193F9040000920023B1
:10C760000321019102931A464FF480712AF0BEF919
:10C77000C4F8100210B1012384F80B32604A644BF4
:10C78000B2F8701092F8725092F87300A3F8C619BC
:10C7900092F8741092F8752083F8CA5983F8CE097C
:10C7A00083F8CF1983F8D02994F81402FBF7B6FD6B
:10C7B00094F815328342054627D058B34FF4FA70E7
:10C7C000FEF718F9D4F81832FBB11A6802F41072A7
:10C7D000B2F5107F19D093F9040003214FF4E13230
:10C7E00000230825CDE9011500924FF400711A4687
:10C7F0002AF07CF9C4F8200238B141490122002313
:10C80000486384F8152284F81C3294F824526DB1E0
:10C8100004B070BDD4F820022AF04CF9C4F82052BC
:10C8200084F8155294F82452002DF1D1D4F828320E
:10C83000002BEDD0032293F90400CDE901251A7AEB
:10C84000324B03EB82034FF40021D3F8883100937D
:10C850002A462B462AF04AF9C4F82C020028D7D0E1
:10C86000274BC4F83452D3F8E03C84F8385203F52F
:10C870001C5310330122C4F8303284F8242204B04F
:10C8800070BDD4F810022AF015F9C4F8105284F8DB
:10C890000B5289E7D4F8F8012AF00CF9C4F8F851E2
:10C8A00084F8F251FAE694F80032002B7FF43CAFA2
:10C8B000D4F8E031002B3FF437AF114A92F84B1017
:10C8C0009367012948D002290CBF0E4B0E4BC4F8C8
:10C8D0000432012384F8003226E794F8E831002B73
:10C8E0007FF4B4AED4F8E031002B3FF4AFAE0122B8
:10C8F000C4F8EC3184F8E821A8E600BFB83700207E
:10C90000C8150020AC090020B8090020FC980608D2
:10C9100000000020D4F8EC012AF0CCF8C4F8EC5167
:10C9200084F8E85192E6134DA86F2AF0C3F8AE6779
:10C9300084F80062F8E64FF461420DE74FF4964345
:10C94000DFE60D4AC4F80422CBE64BB90A4BC4F823
:10C9500004324FF41663D4E6074BC4F80432B8E748
:10C960004FF41663CDE6054B03EB8202D2F8883113
:10C97000C7E600BFC8150020A0090020FC980608E3
:10C9800008490138002310F8012F222A04D001336E
:10C990000F2B01F8012FF6D1034A1344002283F82C
:10C9A0004E20704715160020C815002010B5084C01
:10C9B00082B00223C4F83C32019056F00BFB01997F
:10C9C000C2B2D4F82C0202B0BDE810404AF042B91D
:10C9D000B837002070B5254C064604F14E0056F0DD
:10C9E000F9FA94F84E502B2D38D0302D27D0382D11
:10C9F0002ED01F49002301E011F8015F0C464DB312
:10CA00000133102BF8D1324606F11005134612F807
:10CA1000011B222926D0AA42F8D1002820DDC0F12E
:10CA200001001918621C013301E08B4218D013F881
:10CA3000014D12F8010D8442F7D0002070BD94F82A
:10CA40004F20A2F13101012903460DD9362A0BD01E
:10CA50000138CEE7002BF0D04C1ED4E70538C8E7EC
:10CA6000012070BD013BD8E7981EC2E7C815002021
:10CA7000161600202DE9F04F2DED028B87B0884669
:10CA800000AF164620B10378303B012B40F2858180
:10CA9000DFF83493DFEDC58A9FEDC58A98F8003042
:10CAA000002B3CD036B1C34B3268D3F8E03C9A42FD
:10CAB00040F2BB83C04C94F84052002D40F0BA8243
:10CAC00094F84302BD4B03EB4003B3F8CC3163BB96
:10CAD000012384F84332BA4BDA6811061DD59A68EF
:10CAE000920740F17F83B34AB2F8E43112684FF401
:10CAF000F36113FB01F389FB0301DB17C3EB611344
:10CB000010203021C7F81330082338747974BB74AF
:10CB100038180024904788F80040002EBED11C37FA
:10CB2000BD46BDEC028BBDE8F08F0130C0B2B3F55D
:10CB30008A6F84F8430200F0868127D8B3F5806FAE
:10CB400000F027826BD9B3F5866F00F007824ED9CB
:10CB5000B3F5886FE1D1DFF85CA29AF84530002B7D
:10CB6000DBD0974ADAF80030B2F93022C7F8132048
:10CB700010204021042238747974BA7438180024C3
:10CB8000984788F80040002E88D1C8E7B3F5006FB9
:10CB900000F0348140F28880B3F5046F00F0168114
:10CBA0006CD9B3F5116F00F01882B3F5206FB4D1D2
:10CBB000834BD3F82C329A06AFD5D4ED9F7A7D4BB8
:10CBC00067EEA87A1B68FCEEE77A102117EE902A30
:10CBD0000024C7F813200A2239747C74BA747818B8
:10CBE000984788F80040002E7FF458AF97E7B3F5D8
:10CBF000826F00F0E181B3F5846F8ED1704BDA68FB
:10CC000012068AD59A68950740F1C782D4F8D822CF
:10CC1000684BC7F8132010202021042242E0B3F50E
:10CC2000007F00F0778169D9B3F5047F7FF475AF99
:10CC3000634BDB689D077FF570AFDFF878A19AF84A
:10CC40004630002B40F0B18294F85232012B0CBFD9
:10CC5000B4F86032B4F86232C7F8133010220221FF
:10CC6000DAF800303A747A74B974B8180024984726
:10CC700088F80040002E7FF411AF50E7B3F5026F43
:10CC80005ED14F4BDA6811067FF547AF9A6892077D
:10CC900040F19B82474BD3F8D421C7F813201020D2
:10CCA000202108221B6866E7B3F5E26F00F01581CA
:10CCB0004ED9B3F5E46F7FF430AFDFF8F8A09AF8FF
:10CCC0004530002B7FF429AF3D4B93ED2D0A20EE2C
:10CCD000080A59F04BFD102420210722C7F8130041
:10CCE0003C743819DAF800307974BA740024984723
:10CCF00088F80040002E7FF4D1AE10E7B3F5807FB6
:10CD000000F0C380B3F5887F7FF407AF2C4BD3F8D6
:10CD10002C325B077FF501AF2A4B93F8911103F298
:10CD2000844203F26C43002918BF134693ED050AB1
:10CD300059F01CFD1F4AC7F813001023012163E1BD
:10CD4000B3F5036F3FF4C7AE002E7FF4A7AEE6E65F
:10CD5000B3F5C06F00F08880B3F5E06F7FF4DDAE0F
:10CD6000144D95F84540002C7FF4D7AE144B93ED4D
:10CD70002B0A20EE080A59F0F9FC102107222B6833
:10CD8000C7F813007C743974BA747818984788F817
:10CD90000040002E7FF482AEC1E601300621FBF791
:10CDA0009BFC054B83F8400272E600BFB80C473E7F
:10CDB0000000C842C8150020B8370020FC980608BB
:10CDC000583D0120C02600201F85EB51954B964A07
:10CDD000B3F93432126803EB83035B001020C7F809
:10CDE00013304021082338747974BB743818904785
:10CDF00088F80050002E7FF451AE90E6894BDA6837
:10CE000015067FF58AAE9A68940740F10982C30738
:10CE100000F1F281DFF810A2DAF8CC2182EAE273A5
:10CE2000A3EBE27303EB5303A9FB0313DB08002A14
:10CE3000B8BF43F08043C7F813301021DAF8003050
:10CE400000240822C8E6774BDA6815067FF565AE40
:10CE50009A68940740F1CB81734BB3F9E621C7F888
:10CE6000132010205021D8E6DFF8BCA19AF84930F1
:10CE7000002B40F05E8123F05BFA0024DAF80030EA
:10CE8000C7F8130010210622A6E6664BD3F82C3211
:10CE900059077FF542AE654B634A93F891011168DB
:10CEA00003F2844203F26C43002818BF1346D3ED0B
:10CEB000027AFCEEE77A102217EE903A0024C7F8C7
:10CEC000133001233A747C74BB74B818884788F80F
:10CED0000040002E7FF4E2AD21E6534D95F8454029
:10CEE000002C7FF41AAE4F4B93ED2C0A20EE080A6B
:10CEF00059F03CFC10230721C7F813002A683B7443
:10CF00007B74B974F818904788F80040002E7FF4BD
:10CF1000C5AD04E6434BDB6818057FF5FEAD94F81C
:10CF20005032002B3FF4F9AD3F49414AB1F99E33ED
:10CF30007D7482FB0302DB17C3EBA2031BB2102438
:10CF40000220B8740A68C7F813303C743819904747
:10CF500088F80050002E7FF4A1ADE0E5324B93F845
:10CF60004520002A3FF4D9AD2E4A1B68B2F932227F
:10CF7000C7F81320102230213A7404227974BA744D
:10CF800007F11000984788F80050002E7FF486AD16
:10CF9000C5E5FBF76FF9244BC7F8130010210422F5
:10CFA0001B687D743974BA747818984788F80050F3
:10CFB000002E7FF473ADB2E51A4BDA6815067FF5E3
:10CFC000ACAD9A68940740F10881FBF743FB164A21
:10CFD000C7F813001023042116E0124BDB689907F1
:10CFE0007FF59BAD94F844324BB194F85222012A5C
:10CFF0000CBFB4F86022B4F86222B2FBF3F30A4A21
:10D00000C7F813300921102312683B747B74B9747C
:10D01000F8180024904788F80040002E7FF43EADB9
:10D020007DE500BF583D0120C8150020C026002026
:10D0300067666666DFF83CA207F108033B61DAF831
:10D040001C9007F10E037B61D9F80020DAF8143048
:10D050009A426E4694F8413200F0828007F109024C
:10D060003A615A1C84F8412203F00F030522D9F8D3
:10D0700004B03B7294461346D9F80010ABEB010B99
:10D08000D01D5FFA8BFB20F00700DC45ADEB000DF7
:10D0900040F2D4805A4668465CF062F9D9F8003014
:10D0A0005B44C9F800305A46694607F1100051F058
:10D0B0000DF9DAF81C20DAF81430D9F80000117AEA
:10D0C000C9F80400C21A4A40D2B28342C9F80030FB
:10D0D00084F842220AD00133C9F8003013F8011C49
:10D0E000984282EA0102F6D184F842223B69591C37
:10D0F00039611A70D7E90432D21A012A08DD0021F9
:10D100005A1C3A611970D7E90432D21A012AF7DCA5
:10D1100007F10800FAF7DAFF002500231C37B546AF
:10D1200084F8405288F80030BD46BDEC028BBDE863
:10D13000F08F4F4AD26812057FF5EFAC94F8502279
:10D14000002A3FF4EAAC012B00F08F80D4F864325F
:10D15000C7F813301021DAF80030002406223BE52E
:10D16000B9F90C20591C03F00F0343F01003002AF7
:10D17000B8BF43F0200307F109023A613B72D9E9D5
:10D18000003B0422ABEB030384F8411207F10A01D0
:10D190007B723961134694466EE71B6818077FF56A
:10D1A00035AD002E7FF47AACB9E494F84432002B0C
:10D1B0003FF452AD94F85222012A0CBFB4F8602219
:10D1C000B4F86222B2FBF3F346E51B681B077FF558
:10D1D00061AD002E7FF462ACA1E41B6818077FF5F7
:10D1E000F4AE9AE41B681B077FF57DAC95E41B68E1
:10D1F00018077FF531AE90E4DFF878A0DAF8D02197
:10D2000082EAE273A3EBE27303EB5303A9FB03137C
:10D21000DB08002AACBF43F0004343F040430AE67A
:10D220001B6819077FF5F3AD77E400231C3788F8F6
:10D230000030BD46BDEC028BBDE8F08F6846C7E903
:10D2400000325CF08DF8D9F800107A683B68114420
:10D25000C9F8001007F110001A46694651F036F877
:10D2600007F10800FAF732FF57E7DAF8A0336FE763
:10D27000583D0120C81500202DE9F041DFF820813C
:10D2800098F88931012B82B002D002B0BDE8F0815C
:10D29000D8F804000028F8D0D8F8E03C3E4C3F4EC7
:10D2A00001330025019304F537778DF803500AE028
:10D2B0001B2B84F8E45248D00D2B5CD0012386F858
:10D2C000D139D8F8040003685B689847002849D032
:10D2D000002D47D1D8F804000368DB68984783B273
:10D2E0007E2B4BD096F8D129002AEAD194F8E4227B
:10D2F000002ADDD17D2B4BD094F8E8222AB180F0B2
:10D300002003D8B284F8E852034694F8E322062AB0
:10D310000BD8B4F8E6C2A11863440132A4F8E6328F
:10D3200081F8DC0284F8E322CBE7B4F8E622134468
:10D33000C3F3072252FA83F30122A4F8E632FF2B4B
:10D3400008BF3D4686F8D129BBE7D8F8040003683A
:10D350005B6898470028B1D101238DF8033086F827
:10D36000D139AEE7284601AA0DF10301FFF782FB90
:10D3700002B0BDE8F081A4F8E652A2E701238DF8DF
:10D38000035084F8E35286F8D15984F8E43298E7E0
:10D39000012384F8E83294E7B83700200000002029
:10D3A000C8150020054B93F889210AB10020704769
:10D3B0000222186083F8892101207047C8150020D7
:10D3C000F0B5224C224DC4F8945D85B0FDF7E8FB22
:10D3D00012232049204A84F8683D42F6F82604F6D4
:10D3E000685300274020C3E90267C4F8881DC4F8C9
:10D3F0008C2D29F045FD30B394F8133E94F8121E9D
:10D4000090F90400154A022B14BF082300230029B9
:10D4100008BF43F0010303244FF4E131CDE9014398
:10D4200000910023402129F061FBA5F53B75C5F86B
:10D430001003014620B10A48FFF7B4FF85F8140332
:10D44000081E18BF012005B0F0BD00BFC8150020A0
:10D45000A43A0020ADCA02088DD7020825CE0208E2
:10D4600061C2020810B50C4C94F889310BB1002050
:10D4700010BD202029F004FDC4F88C0150B12021FA
:10D4800029F0F4FC054B84F88A010120236084F81C
:10D49000890110BD012010BDC8150020F5800008CD
:10D4A0002DE9F041494B4A4F93F87630012BC6B035
:10D4B00066D097F81A0397F81B63FE2865D0012EF3
:10D4C00035460DD9BB1903F5497303E0013D012D24
:10D4D000CEB253D013F8012DEEB2711E002AF5D052
:10D4E000D7F82033B7F81C1397F81C83B7F81EC37E
:10D4F0006C46C3F317231A1222721A14E371627274
:10D5000097F8203320702A4661800DF10A003149D6
:10D51000A3716670A4F804C00A355BF021FF18F00F
:10D520000103B7F8181304EB050214D16155090A79
:10D53000984651700923434403331E4414FA86F677
:10D5400014F8011BD7F8100249F0A6FBA642F7D148
:10D5500046B0BDE8F081204B6155090A1D68586846
:10D56000517099681B7B9373C2F80250C2F8060091
:10D57000C2F80A104FF00D080923DCE73546AFE783
:10D58000FE2397F81B6387F81A33D7F82033B7F8D0
:10D590001E0397F820530F496C46C3F3172363719A
:10D5A0003246FE2360800DF10600237066702571FF
:10D5B0005BF0D6FEB31DB7F81823E2542344120AD9
:10D5C0005A704FF000080523B5E700BFC8150020CA
:10D5D000B8370020DC3A0020E63B00202DE9F04F70
:10D5E0000468DFB0D3001B1905900192039103601A
:10D5F00002D3436801334360019BC4F3C504002B8D
:10D6000000F0CD80059B2833049303E0019B002BA1
:10D6100000F0C580019BC4F14002DDE903109A428D
:10D6200028BF1A469B1A01930B4620441344144406
:10D6300003935BF095FE402CE8D1059A1EAE0EAB2D
:10D6400092F82B5092F82A4092F8290092F828106C
:10D650001D705C709870D97004339E4202F1040210
:10D66000EED1059B9A680692DA6807921A690892C9
:10D670005A6909929A690A92DA690B920DF1740A51
:10D680001A6A5B6A0C920D9352460DAB53F8041F55
:10D6900042F8041F1DA99942F8D14EAF3246916B52
:10D6A000134652F8040F5C6A1D684FEAF14383EA9F
:10D6B000714383EA91234FEAB0412C4481EAF0118F
:10D6C000234481EAD0010B449742D363E7D1354B21
:10D6D000009306F1FC030293DDE90869DDE90657D2
:10D6E000DDE90BECDDF834800A9C2F4B0BE0B146F2
:10D6F0003E462F461546009AE046F446A6461C468E
:10D7000052F8043F00924FEAF4212CEA040081EA27
:10D71000B41104EA0E0281EA746142405AF8040F1F
:10D720000A4487EA060B4FEA7531024481EAB501E3
:10D730000BEA050B07EA060081EAB5518BEA000007
:10D740000844029942441A44514502EB0903024439
:10D75000CDD1069911440A46079929440D460899E6
:10D7600039440F46099931440E460A9919440B9BD6
:10D7700023441C460C9B734418460D9B6344884607
:10D780001946059BC3E90740C3E90357C3E9056888
:10D790009A605962019B0024002B7FF43BAF5FB07D
:10D7A000BDE8F08FF49A0608982F8A42F0B5066813
:10D7B00093B0F70804460D468023472200210DF15F
:10D7C0000100C7F1770707F03F078DF800305BF0E5
:10D7D000FAFF12AB3B44606803F8406C07F10902A2
:10D7E000370A03F8417C370C360E4FEA102C03F849
:10D7F000427C03F8436C070C03F8440C060E6946A0
:10D80000204603F845CC03F8467C03F8476CFFF745
:10D81000E5FEE37A2B70A37A6B70637AAB70237AA0
:10D82000EB70E37B2B71A37B6B7113B0F0BD00BF7A
:10D830002DE9F04FA94C94F84874A3B017F00207F3
:10D840009DF8B0C0009159D1D4F84C241AB1127887
:10D85000D20700F135813E46BA46DFF8A89200991A
:10D8600003F10C05FD224D4484F81A2315F8012D0F
:10D870005FFA83FE002A40F01C81013B012BF5D1A9
:10D88000934600911A46009984F81B2384F81F03DD
:10D8900084F82013BAF1000F00F0188194F842E4E4
:10D8A0008DF815200EF10108FD250A21012784F8C5
:10D8B00042848DF81450019184F81EE3A4F81C737F
:10D8C00088460825D4F8207300998DF818E0C7F32E
:10D8D00017274FEA272E8DF819008DF81A103814E3
:10D8E00094F81C138DF81B7000278DF81CE08DF840
:10D8F0001D008DF816108DF8177036E0531E009934
:10D9000084F81B234FF0FE0A4FF006081FFA83FB32
:10D9100084F81F0384F8201384F81AA3CDF8048038
:10D9200013460425002604F5467994F842E48DF860
:10D9300014A00EF101014FF0000A8DF8152084F8B3
:10D940001EE384F84214A4F81CA3002F00F0BC804E
:10D95000D4F8207300998DF816E0C7F317278DF8D7
:10D9600017008DF818108DF819700DF11500054489
:10D970004FF6FF7101E010F8012F4A4082EA0212CF
:10D98000D2B2170987EA112141EA0221854281EAD0
:10D99000C201F0D1524D0BF10D029144284610F80E
:10D9A000012B4A4082EA0212D2B2170987EA1121FA
:10D9B00081EA022181EAC202484517B291B2EED152
:10D9C0008CEA070C8CEA0C1C5FFA8CFC4FEA1C12E8
:10D9D00082EA1121234481EA0C2181EACC0C83F8EC
:10D9E00024C394F81B332344CCF3072283F8252364
:10D9F000A4F818C3BAF1000F09D194F81B7308EB0F
:10DA000006000230384480B223B0BDE8F08FD4F86D
:10DA10004C1494F81B730029F1D00B78DB07EED57A
:10DA20004B7884F82E34CB68DFF8DC900393886859
:10DA3000BDF80C30C4F82F04A9F80430D1E9023243
:10DA4000013342F10002C1E90232264A0A92002360
:10DA5000CDE90833244A254B0B930C92244B254ADD
:10DA60000D930E92244B254A02900F9308A8244B45
:10DA70001092103120221193FFF7B0FD019A08A8EF
:10DA800005A9FFF7ABFD3A46294608A8FFF7A6FD12
:10DA9000E91908A80222FFF7A1FD09F1FF3108A842
:10DAA0000722FFF79BFD09F1060108A8FFF77EFE9C
:10DAB000A3E70EF1FF35009172461FFA85FBE2E6FF
:10DAC0000D264FF0010AC8E6BA46FBE64FF00A08F9
:10DAD000CDF8048008254FF0FD0A26E7B83700206E
:10DAE000DC3A002067E6096A72F36E3C85AE67BBDC
:10DAF0003AF54FA57F520E518C68059BABD9831F19
:10DB000019CDE05BD03A0020E73B002070B5A04C77
:10DB100094F89F5494B0262D28BF26252622002154
:10DB20000AA85BF050FE2A460AA804F595615BF04E
:10DB300017FC9DF84850012D02D0002014B070BD94
:10DB4000944B1B685B0746D49DF84C302BB1BDF855
:10DB5000463023F00402102A21D094F8A42494F82B
:10DB6000A3348DF8112003228DF81030ADF8122067
:10DB700099230499009300202F250423C4F824132B
:10DB800084F82203FA2184F82303012084F8215326
:10DB9000FFF74EFEFFF784FC012014B070BD9DF826
:10DBA0004A20032A38D0022A02D1142B00F0A18087
:10DBB00094F8A43494F8A3248DF8113002238DF83E
:10DBC0001020ADF8123099230093049900202F25DE
:10DBD00004230322D2E794F8A42494F8A3348DF804
:10DBE0001030ADF812508DF81120049AC4F8242397
:10DBF000002199232F2000930322042384F8221369
:10DC000084F8231384F82103FA212846FFF710FE35
:10DC1000FFF746FC284691E7D4F8C025BDF844003C
:10DC200090425ED10130142BC4F8C00508BF042512
:10DC30009FED596ADDED0E6A9DED0F7ADDED107AEC
:10DC4000DFED565AD4F8C4358DF8105066EE866A6A
:10DC500027EE067A67EEA57AFDEEE66ABDEEC77A94
:10DC6000FDEEE77A8342D4BFA52300230025C0B28E
:10DC700004A98DF82630CDED056A8DED067ACDED3F
:10DC8000077A0895ADF8245008F04EF9D4F8C0355D
:10DC9000D4F8C425934237DB414B93F8E81A0029A6
:10DCA00056D094F8A42494F8A3348DF809208DF864
:10DCB0000830ADF80A500298C4F824039923009361
:10DCC0002F2604230322FA21012084F8225384F80A
:10DCD000235384F82163FFF7ABFDFFF7E1FB01203D
:10DCE0002CE794F8A4348DF8113094F8A3240D2374
:10DCF00065E7D4F8C005BDF844309842F1D1013051
:10DD0000C4F8C005042593E794F8A31494F8A42458
:10DD1000ADF808308DF80B208DF80C508DF80A10F6
:10DD2000DDE90201E623C4F8240384F828130093F4
:10DD3000282605230422FA21012084F8225384F89E
:10DD4000235384F82163FFF773FDFFF7A9FBC6E7B0
:10DD500094F8A43494F8A3248DF8093005238DF8A1
:10DD60000820ADF80A30029884F822139923009312
:10DD70002F250423032284F82313C4F82403FA2153
:10DD8000012084F82153FFF753FDFFF789FBA6E735
:10DD9000B8370020583D01208096184B0000C8423B
:10DDA000C02600202DE9F047DFF8A08298F8C8359A
:10DDB0008AB0002B15BF012600264FF001154FF445
:10DDC000803522F077FC012800F0FC80032800F069
:10DDD000A7800228994C18BF4FF0011421F0ACFD28
:10DDE000012800F0A580032800F01081022808BF58
:10DDF00044F0040421F084FD012800F0A4800328ED
:10DE000000F00E81022808BF44F0080421F040FD14
:10DE1000012800F0A380032800F0FD80022808BF3D
:10DE200044F0100421F01CFD012800F0A28003281A
:10DE300000F0E780022808BF44F0200421F0F8FC3D
:10DE4000012800F0A180032800F0D680022808BF36
:10DE500044F0400421F038FD012800F0A0800328A0
:10DE600000F0C580022808BF44F4807498F8CF35CC
:10DE7000002B40F09F801BF049F945F0807544F07D
:10DE8000807408B946F080766D4FB7F8380200EB21
:10DE9000800040004FF47A72002151F079FCFF6855
:10DEA00017F002071FFA80F940F0928022F092FAF0
:10DEB000002840F0BA8007464FF0FF3A64204FF048
:10DEC000000CCDE90254CDE907CC0496ADF818A0BA
:10DED0008DF82600ADF81AC0ADF824C0ADF8149046
:10DEE000ADF8167002AD0FCD564C0FC495E80F007B
:10DEF00007C424F8023B1E0C1F23267001201A467B
:10DF00007C25FA2188F822C388F823C388F82103E6
:10DF10000095FFF78DFC0AB0BDE8F047FFF7C0BAE7
:10DF200021F00AFD0128454C45F002057FF45BAF66
:10DF300021F0E6FC012845F0040544F0040446F015
:10DF400004067FF45CAF21F0A3FC012845F008052E
:10DF500044F0080446F008067FF45DAF21F080FC31
:10DF6000012845F0100544F0100446F010067FF437
:10DF70005EAF21F05DFC012845F0200544F020044F
:10DF800046F020067FF45FAF21F09EFC012845F0AB
:10DF9000400544F0400446F040067FF460AF98F836
:10DFA000CF3545F4807544F4807446F48076002BB8
:10DFB0003FF461AF98F8D035002B3FF45CAF46F4E6
:10DFC000803658E71D4C45F0020546F0020605E78D
:10DFD00022F026FA00EB80004700BFB222F0FAF9E7
:10DFE00040BB4FF0FF3A22F0A3F940B267E745F497
:10DFF000807544F4807439E745F0400544F04004EE
:10E0000028E745F0200544F0200417E745F0040513
:10E0100044F00404EEE645F0100544F0100401E776
:10E0200045F0080544F00804F0E6074B6420B3F916
:10E030009EA344E7044BB3F99EA3D4E70300010079
:10E04000583D0120DC3A0020C8150020B8370020D8
:10E050002DE9F047B34C2DED028BD4F8042294F84F
:10E06000D135D55CEA0784B01ED4AB074CD42E075B
:10E0700000F12F81A80600F1FD80690700F19A8068
:10E08000EB0667D494F8D125A74B0132A3FB02130A
:10E09000DB0803EB8303A2EB430384F8D13504B020
:10E0A000BDEC028BBDE8F08702A8FAF77FF8029B6F
:10E0B0009E4F9F4E591C412202911A70B7F932228D
:10E0C00086FB0231D217C2EBA10189B202A850F03F
:10E0D0002DF9B7F9302286FB0231D217C2EBA1012C
:10E0E00089B202A850F022F9B7F9343286FB032135
:10E0F000DB17C3EBA10189B202A850F017F902A8FF
:10E10000FAF724F9AB07B2D502AE3046FAF74EF86B
:10E11000864BDFF82482D3F82C0210F0800000F048
:10E12000138198F8C731002B00F05581012B00F0C6
:10E130005A81022B14BF00270327B8F9E4317D4A26
:10E1400082FB0312DB17C3EB6213D8E973095FFA92
:10E1500083FAFCE002A8FAF729F8029B4E22591C28
:10E1600002911A70029B94F81426591C02911A709D
:10E17000029B94F81526591C02911A70029B94F880
:10E180001926591C02911A70029B94F81826591CE2
:10E1900002911A70029B94F81626591C02911A706B
:10E1A000029B94F81726591C029102A81A70FAF7DC
:10E1B000CDF867E7DFF8749102AE3046F9F7F6FF65
:10E1C000D9F80430DA0540F1EB804FF00008D9F8B7
:10E1D000007094F8E435C7F380070BB147F00207ED
:10E1E000029B5322591C02911A7022F019F900EB7C
:10E1F0008000410089B2304650F098F84E4B4FF6FF
:10E20000FF72D3F8A003002151F0C2FA81B2304668
:10E2100050F08CF8494B4A4AB3F8443B0299C3EB9F
:10E22000C3135B0082FB03021A44DB17C3EB6223B8
:10E230004A1C02920B70D9F82C3213F020030BD039
:10E24000D4ED9F6A9FED3F7AC6EE877AFCEEE77ABF
:10E25000CDED017A9DF80430029A511C02911370A1
:10E26000029B48EA07075A1C029230461F70FAF7D1
:10E270006DF805E702A8F9F799FF22F07FF9029BF4
:10E280002D4A591C029158211970B2F8EC1106461A
:10E2900002A850F04BF8029A94F80972531C86F0C9
:10E2A000010602931670029A531C029317703FF0F6
:10E2B000FDFF029A531C02931070029A0021561C13
:10E2C0007B1C029602A8117084F80932FAF73EF816
:10E2D000D3E602A8F9F76AFF029B4F22591C02916C
:10E2E0001A70D4F8D41502A850F008F8D4F8D8154C
:10E2F00002A850F003F8D4F8DC1502A84FF0FEFF96
:10E30000029B0A495A1C029201221A70029A8B68D7
:10E31000511C03F00103029102A81370FAF716F8DA
:10E32000A8E600BFB8370020CDCCCCCC583D0120AA
:10E33000676666661F85EB51C8150020C026002061
:10E34000030820800000C842814607468246FDF748
:10E3500049FC029A531C029347231370014630462E
:10E36000B0EE408A4FF0CAFF494630464FF0C6FF34
:10E37000029AFDEEC87A531C029317EE901A82F8A7
:10E3800000A030464FF0BAFF029A98F8C831511CED
:10E3900047EA8303029130461370F9F7D7FF66E628
:10E3A0001F051AD4D8061BD499061ED4DA041FD42C
:10E3B0001F0620D4580521D4190722D413F0440F86
:10E3C00022D1DA0723D413F0020F14BF4FF00C0848
:10E3D0004FF00408FBE60127AFE64FF02808F6E609
:10E3E0004FF03408F3E60227A7E64FF02408EEE6E4
:10E3F0004FF04808EBE64FF05008E8E64FF05408BD
:10E40000E5E64FF02008E2E64FF02C08DFE64FF09B
:10E410000808DCE62DE9F041407800F0F003802B9D
:10E4200082B000F00F0407D0902B15D0A02B2FD076
:10E43000002002B0BDE8F0810421002364F07F04D5
:10E4400068468DF801408DF80010ADF80230F9F7FC
:10E45000C1FE02B0BDE8F081CB4B04EB4402134493
:10E4600064F06F0093F8D45993F8D5298DF8010022
:10E470000621002368468DF802508DF803208DF8A0
:10E480000010ADF80430F9F7A5FE02B0BDE8F08148
:10E49000BE4ED6F82C1211F080076DD1B846BA4B9B
:10E4A00004EB4402134493F8D659012D00F0868002
:10E4B000072D00F0A080032D6BD0052D00F090807B
:10E4C000062D00F0B380092D00F0EB800E2D00F03A
:10E4D000F4800D2D00F0F8800C2D00F0FF80122D3F
:10E4E00000F0D080152D00F0AF80162D00F02181B6
:10E4F000412D00F0F680852D00F01081832D00F075
:10E500002281872D00F04A81082D00F02681142DEC
:10E5100000F031817E2D00F07081132D00F07C81A0
:10E520000A2D00F083810B2D00F08D81802D00F0ED
:10E53000B081812D00F0A381882D00F0DE81892D2E
:10E5400000F0CD81902D00F0E681912D00F0B48196
:10E55000822D00F0A881842D7FF46AAF002F00F097
:10E56000CE808B4B2046D3F8D411642391FBF3F17A
:10E5700089B2F9F769FE5CE7854B93F8C7319BB127
:10E58000012B50D0022B14BF4FF000084FF00308AE
:10E5900085E77F4B93F846304BB121F02BFF0146C6
:10E5A0002046F9F751FE44E74FF0010877E721F0E4
:10E5B00037FF01462046F9F747FE3AE74A07684623
:10E5C0003FD51BF0C7F840B3BDF9003013F5C87F45
:10E5D00023DB03F5C87399B22046F9F735FE28E727
:10E5E00021F0F8FE034648B1694B2046B3F89E136C
:10E5F000F9F72AFE1DE7B6F82A12EDE7062164F0C6
:10E600005F0468468DF80140ADF80230ADF8043083
:10E610008DF80010F9F7DEFD0BE74FF67063ADF8EB
:10E6200000300021D8E74FF0020838E721F0D2FE91
:10E630000346C0B1564B2046B3F8A013F9F704FEC9
:10E64000F7E61BF093F8BEE7514B316893F84A3078
:10E6500013F0780F3CD181F00401C1F38001204612
:10E66000F9F7F2FDE5E664F05F04294668468DF8A7
:10E6700001408DF80050ADF80230ADF80430F9F7E4
:10E68000A9FDD6E611F02003B8D0424BD3ED9F7A16
:10E69000FCEEE77A204617EE903A99B2F9F7D4FDEE
:10E6A000C7E6022006F0FAFFBDEEC00A204610EED3
:10E6B000103A99B2F9F7C8FDBBE6B6F8343203EB6D
:10E6C0008303590089B287E7B6F932325B42F6E735
:10E6D0002046C1F38001F9F7B7FDAAE6B6F830325B
:10E6E000EDE711F0040389D02A4B2046D3F84016F9
:10E6F0000A2391FBF3F189B2F9F7A6FD99E6062109
:10E7000064F05F0468468DF80140ADF80270ADF822
:10E7100004708DF80010F9F75DFD8AE611F004032E
:10E720003FF46CAF1B4B2046B3F83816F9F78CFD5D
:10E730007FE631F087FD184B0344204693F8F8122A
:10E74000F9F782FD75E611F0040110D0114B204657
:10E75000D3F83816F9F75EFD6BE6002FCFD00D4BDE
:10E760002046B3F84416F9F76FFD62E639462046B5
:10E77000F9F750FD5DE6002FC1D0064B2046B3F8F7
:10E78000D812F9F761FD54E600000020583D012041
:10E79000C8150020B8370020FC98060831F052FD5B
:10E7A000634B184490F80413002F3FF415AF6148F1
:10E7B000B66890F8C821B0F8EC0108EB8808C2EB05
:10E7C000421508EB880802EB85024FEA880303EB49
:10E7D000C20319448DB2F30744BF05F5FA718DB237
:10E7E0004FF47A7300210922B0FBF3F050F0D0FF10
:10E7F0000A2101FB005081B2EEE687B34D4BB3F81E
:10E80000E431242101FB03F120466423B1FBF3F141
:10E8100089B2F9F719FD0CE6002F3FF470AF454BB4
:10E820002046B3F8E411F9F70FFD02E6002F3FF49C
:10E8300066AF404B2046B3F9E63193FBF5F399B24E
:10E84000F9F702FDF5E5002F3FF459AF394B93F886
:10E85000C811204601EB0821F9F7F6FCE9E5002391
:10E86000062164F05F0468468DF801408DF80010C1
:10E87000ADF80230ADF80430F9F7ACFCD9E5002F63
:10E880003FF474AF2B4B2046D3F8D011F9F7C2FCFC
:10E89000CFE5002F3FF46AAF264B2046D3F8CC11CA
:10E8A000F9F7B8FCC5E5002F3DD0224B2046D3F840
:10E8B000D411F9F7AFFCBCE5002F3FF420AF1D4A9F
:10E8C0001D4BD2F8D02192FBF3F1204603FB11211E
:10E8D0000A2391FBF3F189B2F9F7B6FCA9E5002F01
:10E8E0003FF40DAF134A144BD2F8D01191FBF3F162
:10E8F000204689B2F9F7A8FC9BE5002F3FF4FFAE54
:10E900000C4A0D4BD2F8CC1191FBF3F1204689B2A1
:10E91000F9F79AFC8DE5002F3FF4F1AE054A064B5E
:10E92000D2F8CC21CFE720460021F9F773FC80E52F
:10E93000FC980608C8150020A086010010B5064CFA
:10E9400003E0D4F8F80148F079F9D4F8F80148F078
:10E950007DF90028F5D110BDB837002070B50B4EF9
:10E96000054606F24A6151F035FC2C686C6006F5EC
:10E97000C961641A182CA8BF18242960224606F51C
:10E98000CC605AF0EDFC86F8784670BDB8370020B0
:10E990005E2810B515D05D28014606D00F4BBDE8A6
:10E9A0001040D3F8EC0148F077B90C4CD4F8EC01E6
:10E9B00048F072F9D4F8EC013D21BDE8104048F070
:10E9C0006BB9064C5D21D4F8EC0148F065F9D4F838
:10E9D000EC013E21BDE8104048F05EB9B837002098
:10E9E00038B5074D04465E21D5F8EC0148F054F9DE
:10E9F000D5F8EC012146BDE8384048F04DB900BFDC
:10EA0000B83700200168504A0029B8BF49422DE9B3
:10EA1000F04105464D4CDFF83C81A2FB01039B0D04
:10EA200004FB0314C4EB0414A40098F8420082FB16
:10EA30000421E217C2EBA152002878D103EB830333
:10EA400003EB830302EB83073FB2404E404B06FBD0
:10EA5000024283FB02341320D217C2EBA414FFF747
:10EA6000BFFFF8B2FFF794FFC7F30720FFF790FF4F
:10EA70001B20FFF7B5FFE0B2FFF78AFFC4F30720C2
:10EA8000FFF786FF2320FFF7ABFF2B682E4C002BF0
:10EA9000B4BF53204E20FFF77BFF0020FFF778FF25
:10EAA0006A6898F84200002AB8BF5242A4FB0231BB
:10EAB000890D06FB0126C6EB0616B20084FB023464
:10EAC000D317C3EBA453002837D101EB810101EB2D
:10EAD000810103EB810636B21C491D4C01FB032367
:10EAE00084FB03241220DB17C3EBA414FFF778FF89
:10EAF000F0B2FFF74DFFC6F30720FFF749FF1A20DA
:10EB0000FFF76EFFE0B2FFF743FFC4F30720FFF704
:10EB10003FFF2220FFF764FF6B68002BB4BF572034
:10EB20004520FFF735FFBDE8F041002030E7C3EB9B
:10EB3000031302EB83073FB287E7C1EB011103EB3D
:10EB4000810636B2C8E700BF6BCA5F6B806967FF9A
:10EB5000D34D6210C81500202DE9F047302084B055
:10EB6000FFF73EFF022006F099FD57F0FFFDA74C8E
:10EB70000546C0B2FFF70CFFC5F30720FFF708FFFB
:10EB8000D4F8EC015E2148F087F894F8793613F058
:10EB900003062AD1D4F87C2641F288339A4200F247
:10EBA000DB811420FFF71CFF994B9A4AB3F93432EA
:10EBB00082FB0312D817C0EBA20005B2C0B2FFF768
:10EBC000E7FEC5F30720FFF7E3FE1C20FFF708FF71
:10EBD0000020FFF7DDFE0020FFF7DAFED4F8EC019D
:10EBE0005E2148F059F894F8793613F0070705D0FC
:10EBF000282B00F0D78004B0BDE8F0870220FFF793
:10EC0000EFFEF9F737FB0646C0B2FFF7C1FE804DB5
:10EC1000C6F30720FFF7BCFE0320B5F92A82FFF7F1
:10EC2000DFFE2B68590700F10581D4F880267A4B66
:10EC3000D068A3FB00308608C0F38700FFF7A8FE6A
:10EC4000C6F30720FFF7A4FEEB689B0700F10C81D9
:10EC5000D5F82C321E0640F1A581AB68DFF8C881DB
:10EC6000980740F1B4811120FFF7BAFEB8F8E4210B
:10EC70006A4B6B4E4FF4F36A12FB0AF283FB0239C4
:10EC8000D217C2EB69395FFA89F0FFF781FEC9F349
:10EC90000720FFF77DFE1920FFF7A2FEB8F8E43148
:10ECA00013FB0AF386FB0312DB17C3EB621386FB2D
:10ECB00003124FEAE379C9EB6219642202FB1939A6
:10ECC0005FFA89F0FFF764FEC9F30720FFF760FEE3
:10ECD000AB68990740F17B810720FFF781FED4F8EC
:10ECE000D8925FFA89F0FFF753FEC9F30720FFF7C8
:10ECF0004FFED8F8D431AA6886FB030192074FEA89
:10ED0000E376C6EB611640F16281F7B2C6F30726DF
:10ED10000120FFF765FE3846FFF73AFE3046FFF761
:10ED200037FE0920FFF75CFE0020FFF731FE0020D0
:10ED3000FFF72EFE0520FFF753FEF9F78BFC064682
:10ED4000C0B2FFF725FEC6F30720FFF721FEAA6831
:10ED50000023CDE90033930700F12E8194F8843627
:10ED6000012B00F02981DFED2F6A98ED0E7AD8EDA6
:10ED70000F7A27EE267A67EEA67ABDEEC77AFDEE09
:10ED8000E77A02A88DED027ACDED037AFFF73AFE1D
:10ED9000D4F8EC015E2147F07FFF94F87936282BF8
:10EDA0007FF429AF204B2148D3F8E05C0027A0FB7B
:10EDB0000535172084F87976FFF712FE3846FFF7FD
:10EDC000E7FD1B48AD09A0FB05367609A0FB063020
:10EDD0004009C0EB0010A6EB8000C0B2C6EB0616DF
:10EDE000FFF7D6FDA5EB86061820FFF7F9FDF0B278
:10EDF000FFF7CEFD3846FFF7CBFDD4F8EC015E21DE
:10EE000047F04AFF04B0BDE8F08700BFB8370020E4
:10EE1000583D012067666666CDCCCCCC89B5F81428
:10EE20001F85EB518096184BC8150020D34D6210FA
:10EE300089888888804B4FEAE87683FB0838C6EBE0
:10EE40006806384636B231F00FFC002800F0C18069
:10EE5000F0B2C6F30726FFF79BFD3046FFF798FD9B
:10EE6000EB689B077FF5F4AE21F0DAFA94F84422C0
:10EE7000DFF8D88100EB800052004300B3FBF2F3CF
:10EE8000C3F3032646EA03239EB20620FFF7A8FD3C
:10EE900006F00F00FFF77CFD300AFFF779FD21F047
:10EEA000BFFA98F84430012B064600F0B58000EB1D
:10EEB0008009624898F8463006EB490680FB06292F
:10EEC000F617C6EBA909002B40F0A1803A20FFF706
:10EED00087FD5B4B1FFA89F9A3FB09234FEA531AFD
:10EEE000C3F34710FFF754FD4FEA1A20FFF750FD18
:10EEF0003B20FFF775FD642000FB1A90514B80B258
:10EF00000530A3FB0030C0F3C700FFF741FD002030
:10EF1000FFF73EFD2820FFF763FDB8F99E33464A10
:10EF2000D81782FB0312C0EBA20006B2C0B2FFF7F3
:10EF30002FFDC6F30720FFF72BFD98F84960002E40
:10EF40004DD10420FFF74CFD21F0F2F9FFF720FD31
:10EF50003046FFF71DFD7BE6FCF744FEFDEEC07A70
:10EF6000102017EE907AFFF73BFD3548FD1780FB28
:10EF70000730C5EB6015E8B2FFF70AFDC5F30720BF
:10EF8000FFF706FD2120FFF72BFD642000FB157025
:10EF90000028B8BF4042C0B2FFF7FAFC3046FFF786
:10EFA000F7FCFEE5284B93E8030002AB83E803007F
:10EFB0001846FFF727FDEBE6D8E9732301216846E1
:10EFC000CDE9002384F88416FFF71CFDE0E6002657
:10EFD0009EE6EB68DA067FF53BAF06463BE721F09D
:10EFE000F9F900283FF434AE0420FFF7F9FC98F853
:10EFF0004930012B0CBFB8F9A063B4F96462F0B2D8
:10F00000FFF7C6FCC6F30720FFF7C2FC20E694F822
:10F010004432B9FBF3F959E73920FFF7E1FC09481D
:10F02000A0FB0630C0F3CF06C0F3C700FFF7B0FC6B
:10F03000300AFFF7ADFC6DE767666666310CC330DA
:10F040001F85EB51CDCCCCCC0C9C0608C8150020FC
:10F050000B2814D810B401EB4103094C01EB8303D6
:10F060002344184490F81431934205D021440023DE
:10F0700080F8142181F808315DF8044B704770471F
:10F08000C8150020F0B54C4D95F88546012C83B08D
:10F0900002460B4654D995F88666484FA11907EBEE
:10F0A0008107013695F88716D7F8187306F003061E
:10F0B00085F8866600294BD197B195F8A016E1B97D
:10F0C0003F490191123948F2A50000911521A5F898
:10F0D000BC0685F8BE166846B84710BB95F885464D
:10F0E000384B0134A3FB042323F0010202EB53034A
:10F0F000E41A85F8854603B0F0BD334933480191E1
:10F10000123990F8044A009148F2A6001621A5F899
:10F11000A40685F8A74685F8A6166846B8470028CD
:10F12000DCD095F8A016D9B1009929480191091AA7
:10F130000231009023F000FC002385F8D136CDE7A2
:10F140001E4901EB8401D1F81873002FB5D1C7E730
:10F15000D5F8880605F28C618842ADD11D4FACE729
:10F16000009E1D4A964214D9013A013E41F2210403
:10F1700012F8013F81EA0321082311F4004F84EAC9
:10F1800041000ABF490081B289B2013BF5D19642E4
:10F19000EED168464FF0CAF81049009E761A152E37
:10F1A000A8BF1526324601F118005AF0D9F895F893
:10F1B000854685F8E96693E7B8370020FC9806088D
:10F1C000893E0020ABAAAAAA723E002000000020BF
:10F1D0005C3E0020B5840008773E0020743E00208D
:10F1E0002DE9F04F2DED028BDFF874B291B09BF852
:10F1F0007C3002AF2BB93C37BD46BDEC028BBDE87D
:10F20000F08F9BF8042180468946002A40F0C9808F
:10F21000DFF850A29AF8EA4684BB9AF85437002BDC
:10F2200040F02281DAF850379AF855478A4AB2FB03
:10F23000F4F21A440023994508BF9045DBD39AF8AD
:10F240005657CAF850870AEB050393F85867F30737
:10F2500001F17884B00701F13182700701F1C980B2
:10F26000310700F16784F30600F1AF830135B5FB88
:10F27000F4F304FB13548AF85647BCE7DAF84C372A
:10F28000002B00F0D4800026C7E900893E610EE023
:10F2900001342644EFF31183502282F31288DAF806
:10F2A0004C27964280F2CF80DBB283F311880AEBC1
:10F2B0000603701C93F8EC46684B21461844F9F796
:10F2C0000BFA81460028E3D06B4690B008EE103A66
:10F2D0000DF1420002ABC7E90630DBF81C507B6140
:10F2E0002A68DBF814309A429AF8413268D0591CE7
:10F2F00039200DF1090203F00F0384468AF8411208
:10F300008DF80830BA61F860D5E90012634607331A
:10F31000521A23F00703D2B2ADEB030D824202ABC7
:10F320006ED21846FA605AF01BF82968FA6803464C
:10F3300088182860194607F118004EF0C7FFDBF85F
:10F340001C20DBF814302868117A6860C21A4A4021
:10F35000D2B283422B608AF8422209D001332B605B
:10F3600013F8011C984282EA0102F7D18AF842227E
:10F37000BB69591CB9611A70D7E90632D21A012A41
:10F3800008DD00215A1CBA611970D7E90632D21A79
:10F39000012AF7DC7869F8F7FFFF18EE103A9D466E
:10F3A00076E7DBF82C4E2368DD69002D00F0FA8249
:10F3B00020460BF1C401A84700238BF8043127E74E
:10F3C000B5F90C20D7F814C0591C03F00F0343F013
:10F3D0001003002A8AF841126146B8BF43F02003A7
:10F3E000624601F8023B0132BA61D5E90023401AB6
:10F3F000C0B29B1A8CF80130B961F860844683E78B
:10F4000062461846E04659F0ABFF2A68414611446F
:10F41000034608462860FA6807F1180019464EF0BE
:10F4200055FF7869C7F81090F8F7B6FFB5E73B616C
:10F430003B698AF8EA363C37CAF85087BD46BDECCE
:10F44000028BBDE8F08F0022D7E90089DBB2CAF851
:10F450004C2783F31188EBE7A0860100A43E00202F
:10F46000C8150020B8370020C94B8BF8C040C8220F
:10F470008BF88020C749C84A009307F11800C74B92
:10F480004EF05EFF9BF8C0308BF88140292183EA63
:10F4900001025200DB0918BF82F0D502D2B212F08D
:10F4A000800F4FEA420218BF82F0D502D2B212F0AA
:10F4B000800F4FEA420218BF82F0D502D2B212F09A
:10F4C000800F4FEA420218BF82F0D502D2B212F08A
:10F4D000800F4FEA420218BF82F0D502D2B212F07A
:10F4E000800F4FEA420218BF82F0D502D2B212F06A
:10F4F000800F4FEA420218BF82F0D502D2B212F05A
:10F50000800F4FEA420218BF82F0D502D2B2EA233E
:10F510008BF8833053405B00D20908BF83F0D503DA
:10F52000DBB213F0800F4FEA430318BF83F0D5031B
:10F53000DBB213F0800F4FEA430318BF83F0D5030B
:10F54000DBB213F0800F4FEA430318BF83F0D503FB
:10F55000DBB213F0800F4FEA430318BF83F0D503EB
:10F56000DBB213F0800F4FEA430318BF83F0D503DB
:10F57000DBB213F0800F4FEA430318BF83F0D503CB
:10F58000DBB213F0800F4FEA430318BF83F0D503BB
:10F59000DBB2C8228BF884205A40DB094FEA4203D1
:10F5A00008BF83F0D503DBB213F0800F4FEA4303AB
:10F5B00018BF83F0D503DBB213F0800F4FEA43038B
:10F5C00018BF83F0D503DBB213F0800F4FEA43037B
:10F5D00018BF83F0D503DBB213F0800F4FEA43036B
:10F5E00018BF83F0D503DBB213F0800F4FEA43035B
:10F5F00018BF83F0D503DBB213F0800F4FEA43034B
:10F6000018BF83F0D503DBB213F0800F4FEA43033A
:10F6100018BF83F0D503DCB207F118008BF8821015
:10F620008BF8C04053F0D6FC002801F05E855C4E9C
:10F6300007F118021518314628E0DCB25BB2002B46
:10F6400034DB6300DCB25BB2002B36DB6400E3B278
:10F6500064B2002C38DB5C00E3B264B2002C3ADB0D
:10F660005C00E3B264B2002C3CDB5C00E3B264B249
:10F67000002C3EDB5C00E3B264B2002C4FEA430393
:10F68000B8BF83F0D5039542DCB238D012F8013B05
:10F6900001F8013B634013F0800F4FEA4303CCD0E5
:10F6A00083F0D50463B2002BE4B2CADA640084F0BC
:10F6B000D50463B2002BE4B2C8DA630083F0D5034B
:10F6C0005CB2002CDBB2C6DA5B0083F0D5035CB21F
:10F6D000002CDBB2C4DA5B0083F0D5035CB2002CF3
:10F6E000DBB2C2DA5B0083F0D5035CB2002CDBB284
:10F6F000C0DA5B0083F0D5035CB2DBB2BDE7304417
:10F7000002460023210602F8013B4FEA440348BFAA
:10F7100083F0D503DBB213F0800F4FEA430318BF29
:10F7200083F0D503DBB213F0800F4FEA430318BF19
:10F7300083F0D503DBB213F0800F4FEA430318BF09
:10F7400083F0D503DBB213F0800F4FEA430318BFF9
:10F7500083F0D503DBB213F0800F4FEA430318BFE9
:10F7600083F0D503DBB213F0800F4FEA430318BFD9
:10F7700083F0D503DBB213F0800F4FEA430318BFC9
:10F7800083F0D503DBB200F10D04002132E000BFAD
:10F79000582B07084C2B0708442B07083C2B07085D
:10F7A0004D160020DDB25BB2002B30DB6B00DDB20A
:10F7B0005BB2002B32DB6D00EBB26DB2002D34DB9F
:10F7C0005D00EBB26DB2002D36DB5D00EBB26DB2C9
:10F7D000002D38DB5D00EBB26DB2002D3ADB5D0031
:10F7E000EBB26DB25B00002DB8BF83F0D503A2422F
:10F7F000DBB235D013F0800F02F8011B4FEA430350
:10F80000D0D083F0D5056BB2002BEDB2CEDA6D000F
:10F8100085F0D5056BB2002BEDB2CCDA6B0083F02E
:10F82000D5035DB2002DDBB2CADA5B0083F0D503ED
:10F830005DB2002DDBB2C8DA5B0083F0D5035DB2A8
:10F84000002DDBB2C6DA5B0083F0D5035DB2002D7C
:10F85000DBB2C4DA5B0083F0D5035DB2DBB2C1E793
:10F8600013F0800F4FEA430318BF83F0D503DBB2D8
:10F8700013F0800F4FEA430318BF83F0D503DBB2C8
:10F8800013F0800F4FEA430318BF83F0D503DBB2B8
:10F8900013F0800F4FEA430318BF83F0D503DBB2A8
:10F8A00013F0800F4FEA430318BF83F0D503DBB298
:10F8B00013F0800F4FEA430318BF83F0D503DBB288
:10F8C00013F0800F4FEA430318BF83F0D503DBB278
:10F8D00013F0800F4FEA43034FF0000218BF83F08C
:10F8E000D5034273DBB2012282735A40DB094FEA2F
:10F8F000420318BF83F0D503DBB213F0800F4FEA49
:10F90000430318BF83F0D503DBB213F0800F4FEA37
:10F91000430318BF83F0D503DBB213F0800F4FEA27
:10F92000430318BF83F0D503DBB213F0800F4FEA17
:10F93000430318BF83F0D503DBB213F0800F4FEA07
:10F94000430318BF83F0D503DBB213F0800F4FEAF7
:10F950004303744918BF83F0D503DBB200F11005EF
:10F960006D1A13F0800F4FEA430318BF83F0D503DD
:10F97000402DDBB2A8BF40254A1C00F10F04C37321
:10F98000A41A01F144002A468BF8C0308BF881405C
:10F9900059F0E6FC00238BF80451CAF850878AF826
:10F9A000543728E40BF1C406B51800E023689B68BF
:10F9B000204698470028F9D0236816F8011B1B68D9
:10F9C00020469847AE42F1D1F6E4574B93F8911197
:10F9D00003F2844203F26C43002918BF134693EDEF
:10F9E000050A4FF499620723ABF880208BF8823028
:10F9F00056F0BCFEC0F3072282F054038BF883203C
:10FA00005B00D20918BF83F0D503DBB213F0800F7F
:10FA10004FEA430318BF83F0D503DBB213F0800F26
:10FA20004FEA430318BF83F0D503DBB213F0800F16
:10FA30004FEA430318BF83F0D503DBB213F0800F06
:10FA40004FEA430318BF83F0D503DBB213F0800FF6
:10FA50004FEA430318BF83F0D503DBB213F0800FE6
:10FA60004FEA430318BF83F0D503DBB213F0800FD6
:10FA70004FEA430318BF83F0D503C0B2DBB2434063
:10FA800013F0800F4FEA430318BF83F0D503DBB2B6
:10FA900013F0800F4FEA430318BF83F0D503DBB2A6
:10FAA00013F0800F4FEA430318BF83F0D503DBB296
:10FAB00013F0800F4FEA430318BF83F0D503DBB286
:10FAC00013F0800F4FEA430318BF83F0D503DBB276
:10FAD00013F0800F4FEA430318BF83F0D503DBB266
:10FAE00013F0800F4FEA430318BF83F0D503DBB256
:10FAF00013F0800F4FEA430318BF83F0D503DBB246
:10FB0000084A8BF885308BF8840092E803008BF864
:10FB1000C0300623CBF8C400ABF8C8108BF8043112
:10FB2000FFF7A4BB48160020C02600200AD7233CBC
:10FB300000007A44DBF8CC211FED047A5FED047AF3
:10FB4000DFF8D4E7110E81F07F038BF883105B00A0
:10FB5000C90918BF83F0D503DBB213F0800F4FEA59
:10FB6000430318BF83F0D503DBB213F0800F4FEAD5
:10FB7000430318BF83F0D503DBB213F0800F4FEAC5
:10FB8000430318BF83F0D503DBB213F0800F4FEAB5
:10FB9000430318BF83F0D503DBB213F0800F4FEAA5
:10FBA000430318BF83F0D503DBB213F0800F4FEA95
:10FBB000430318BF83F0D503DBB213F0800F4FEA85
:10FBC000430318BF83F0D503C2F30741DBB24B40B8
:10FBD00013F0800F4FEA430318BF83F0D503DBB265
:10FBE00013F0800F4FEA430318BF83F0D503DBB255
:10FBF00013F0800F4FEA430318BF83F0D503DBB245
:10FC000013F0800F4FEA430318BF83F0D503DBB234
:10FC100013F0800F4FEA430318BF83F0D503DBB224
:10FC200013F0800F4FEA430318BF83F0D503DBB214
:10FC300013F0800F4FEA430318BF83F0D503DBB204
:10FC400013F0800F4FEA430318BF83F0D5038BF8FE
:10FC50008410DBB2C2F307214B4013F0800F4FEA50
:10FC6000430318BF83F0D503DBB213F0800F4FEAD4
:10FC7000430318BF83F0D503DBB213F0800F4FEAC4
:10FC8000430318BF83F0D503DBB213F0800F4FEAB4
:10FC9000430318BF83F0D503DBB213F0800F4FEAA4
:10FCA000430318BF83F0D503DBB213F0800F4FEA94
:10FCB000430318BF83F0D503DBB213F0800F4FEA84
:10FCC000430318BF83F0D503DBB213F0800F4FEA74
:10FCD000430318BF83F0D503D2B2DBB2534013F015
:10FCE000800F4FEA430318BF83F0D503DBB213F054
:10FCF000800F4FEA430318BF83F0D503DBB213F044
:10FD0000800F4FEA430318BF83F0D503DBB213F033
:10FD1000800F4FEA430318BF83F0D503DBB213F023
:10FD2000800F4FEA430318BF83F0D503DBB213F013
:10FD3000800F4FEA430318BF83F0D503DBB213F003
:10FD4000800F4FEA430318BF83F0D503DBB28BF873
:10FD5000862013F0800FDBF8D0218BF885104FEA56
:10FD6000430318BF83F0D503110EDBB24B4013F0F1
:10FD7000800F4FEA430318BF83F0D503DBB213F0C3
:10FD8000800F4FEA430318BF83F0D503DBB213F0B3
:10FD9000800F4FEA430318BF83F0D503DBB213F0A3
:10FDA000800F4FEA430318BF83F0D503DBB213F093
:10FDB000800F4FEA430318BF83F0D503DBB213F083
:10FDC000800F4FEA430318BF83F0D503DBB213F073
:10FDD000800F4FEA430318BF83F0D503DBB213F063
:10FDE000800F4FEA430318BF83F0D5038BF88710C9
:10FDF000DBB2C2F307414B4013F0800F4FEA4303DD
:10FE000018BF83F0D503DBB213F0800F4FEA430332
:10FE100018BF83F0D503DBB213F0800F4FEA430322
:10FE200018BF83F0D503DBB213F0800F4FEA430312
:10FE300018BF83F0D503DBB213F0800F4FEA430302
:10FE400018BF83F0D503DBB213F0800F4FEA4303F2
:10FE500018BF83F0D503DBB213F0800F4FEA4303E2
:10FE600018BF83F0D503DBB213F0800F4FEA4303D2
:10FE700018BF83F0D5038BF88810DBB2C2F30721DB
:10FE80004B4013F0800F4FEA430318BF83F0D503B4
:10FE9000DBB213F0800F4FEA430318BF83F0D503A2
:10FEA000DBB213F0800F4FEA430318BF83F0D50392
:10FEB000DBB213F0800F4FEA430318BF83F0D50382
:10FEC000DBB213F0800F4FEA430318BF83F0D50372
:10FED000DBB213F0800F4FEA430318BF83F0D50362
:10FEE000DBB213F0800F4FEA430318BF83F0D50352
:10FEF000DBB213F0800F4FEA430318BF83F0D50342
:10FF0000D2B2DBB2534013F0800F4FEA430318BF65
:10FF100083F0D503DBB213F0800F4FEA430318BF21
:10FF200083F0D503DBB213F0800F4FEA430318BF11
:10FF300083F0D503DBB213F0800F4FEA430318BF01
:10FF400083F0D503DBB213F0800F4FEA430318BFF1
:10FF500083F0D503DBB213F0800F4FEA430318BFE1
:10FF600083F0D503DBB28BF8891013F0800FBBF858
:10FF7000E4118BF88A2041F2C81C4FF002004FEACE
:10FF80004303ABF880C08BF88200E14A18BF83F0CE
:10FF9000D5034FF0240C322011FB0C01DBB282FBA5
:10FFA000012013F0800F4FEAE1724FEA4303C2EBE6
:10FFB000601218BF83F0D503C2F30721DBB24B40B8
:10FFC00013F0800F4FEA430318BF83F0D503DBB271
:10FFD00013F0800F4FEA430318BF83F0D503DBB261
:10FFE00013F0800F4FEA430318BF83F0D503DBB251
:10FFF00013F0800F4FEA430318BF83F0D503DBB241
:020000040801F1
:1000000013F0800F4FEA430318BF83F0D503DBB230
:1000100013F0800F4FEA430318BF83F0D503DBB220
:1000200013F0800F4FEA430318BF83F0D503DBB210
:1000300013F0800F4FEA430318BF83F0D503D2B209
:10004000DBB2534013F0800F4FEA430318BF83F035
:10005000D503DBB213F0800F4FEA430318BF83F0E0
:10006000D503DBB213F0800F4FEA430318BF83F0D0
:10007000D503DBB213F0800F4FEA430318BF83F0C0
:10008000D503DBB213F0800F4FEA430318BF83F0B0
:10009000D503DBB213F0800F4FEA430318BF83F0A0
:1000A000D503DBB213F0800F4FEA43038BF88C20AB
:1000B00018BF83F0D503BBF8E6218BF88B10DBB2B9
:1000C00013F0800F02EB82024FEA430318BF83F064
:1000D000D5035200C2F30721DBB24B4013F0800F6F
:1000E0004FEA430318BF83F0D503DBB213F0800F50
:1000F0004FEA430318BF83F0D503DBB213F0800F40
:100100004FEA430318BF83F0D503DBB213F0800F2F
:100110004FEA430318BF83F0D503DBB213F0800F1F
:100120004FEA430318BF83F0D503DBB213F0800F0F
:100130004FEA430318BF83F0D503DBB213F0800FFF
:100140004FEA430318BF83F0D503DBB213F0800FEF
:100150004FEA430318BF83F0D50392B2D2B2DBB2A9
:10016000534013F0800F4FEA430318BF83F0D503C9
:10017000DBB213F0800F4FEA430318BF83F0D503BF
:10018000DBB213F0800F4FEA430318BF83F0D503AF
:10019000DBB213F0800F4FEA430318BF83F0D5039F
:1001A000DBB213F0800F4FEA430318BF83F0D5038F
:1001B000DBB213F0800F4FEA430318BF83F0D5037F
:1001C000DBB28BF88E2013F0800F524A8BF88D1023
:1001D0004FEA430318BF83F0D50392F89101DBB2D5
:1001E00013F0800F02F284414FEA430302F26C42A3
:1001F00018BF83F0D503002818BF0A46D2ED026A63
:10020000E6EE877ADBB2AEF14408FCEEE77A17EE51
:10021000902AC2F307214B4013F0800F4FEA4303AB
:1002200018BF83F0D503DBB213F0800F4FEA43030E
:1002300018BF83F0D503DBB213F0800F4FEA4303FE
:1002400018BF83F0D503DBB213F0800F4FEA4303EE
:1002500018BF83F0D503DBB213F0800F4FEA4303DE
:1002600018BF83F0D503DBB213F0800F4FEA4303CE
:1002700018BF83F0D503DBB213F0800F4FEA4303BE
:1002800018BF83F0D503DBB213F0800F4FEA4303AE
:1002900018BF83F0D50392B2D2B2DBB2534013F051
:1002A000800F4FEA430318BF83F0D503DBB213F08E
:1002B000800F4FEA430318BF83F0D503DBB213F07E
:1002C000800F4FEA430318BF83F0D503DBB213F06E
:1002D000800F4FEA430318BF83F0D503DBB213F05E
:1002E000800F4FEA430318BF83F0D503DBB213F04E
:1002F000800F4FEA430318BF83F0D503DBB213F03E
:10030000800F4FEA430318BF83F0D503DBB205E04B
:100310001F85EB51C02600208C16002013F0800FA3
:100320004FEA43038BF8902018BF83F0D5039BF866
:10033000C8218BF89120DBB2534013F0800F4FEAB5
:10034000430318BF83F0D503DBB24FEA430C1A0610
:1003500048BF8CF0D50C5FFA8CFC1CF0800F4FEA84
:100360004C0C18BF8CF0D50C5FFA8CFC1CF0800F85
:100370004FEA4C0C18BF8CF0D50C5FFA8CFC1CF0CB
:10038000800F4FEA4C0C18BF8CF0D50C5FFA8CFC38
:100390001CF0800F4FEA4C0C18BF8CF0D50C5FFAA4
:1003A0008CFC1CF0800F4FEA4C0C18BF8CF0D50C65
:1003B0005FFA8CFC1CF0800F4FEA4C0C18BF8CF0DD
:1003C000D50C5FFA8CFC8BF88F108BF892C0B8E8D4
:1003D0000F00AEE80F00D8F800302EF8023B1322D1
:1003E0001B0C8BF8C0C08EF800308BF80421FEF790
:1003F0003ABFAC4AC8211368ABF8801071212120A4
:100400008BF8C01059078BF8820040F1EA85D2E9D9
:100410000103A549A54A03F40043002B16BF0A4671
:1004200004210321830540F18D86A14A042113781C
:100430008BF8833083F071035B00D8B25BB2002B82
:10044000C0F2BA854000C3B240B20028C0F2AD8508
:100450005800C3B240B20028C0F2A0855800C3B211
:1004600040B20028C0F293855800C3B240B20028C1
:10047000C0F2B0855800C3B240B20028C0F2A385D4
:100480005800C3B240B200284FEA430350788BF8BB
:100490008400B8BF83F0D503DBB2434013F0800F74
:1004A0004FEA430340F0B485D8B25BB2002BC0F2F0
:1004B000A8854000C3B240B20028C0F2C4855800ED
:1004C000C3B240B20028C0F2B7855800C3B240B2F0
:1004D0000028C0F2AA855800C3B240B20028C0F27A
:1004E0009D855800C3B240B20028C0F2B3855800C1
:1004F000C3B240B25B000028B8BF83F0D503022925
:10050000DBB200F0748690788BF88500434013F0DE
:10051000800F4FEA430340F0AB85D8B25BB2002BAB
:10052000C0F29F854000C3B240B20028C0F2BB8534
:100530005800C3B240B20028C0F2AE855800C3B222
:1005400040B20028C0F2A1855800C3B240B20028D2
:10055000C0F294855800C3B240B20028C0F2AA8508
:100560005800C3B240B25B000028B8BF83F0D50387
:100570000429DBB240F04386D2788BF886205340C2
:10058000180600F1BC855A00D3B252B2002AC0F25C
:10059000AF855A00D3B252B2002AC0F2CC855A00BD
:1005A000D3B252B2002AC0F2BF855A00D3B252B2BF
:1005B000002AC0F2B2855A00D3B252B2002AC0F269
:1005C000A5855A00D3B252B2002AC0F287855A00DC
:1005D000D3B252B25B00002AB8BF83F0D503DFF874
:1005E000D8C0DBB213F0800F4FEA430318BF83F08B
:1005F000D503DBB213F0800F4FEA430318BF83F03B
:10060000D503DBB213F0800F4FEA430318BF83F02A
:10061000D503DBB213F0800F4FEA430318BF83F01A
:10062000D503DBB213F0800F4FEA430318BF83F00A
:10063000D503DBB213F0800F4FEA430318BF83F0FA
:10064000D503DBB213F0800F4FEA4303194960462C
:1006500018BF83F0D5030022DBB20CF1020800F8CA
:10066000012BA8EB010813F0800F4FEA430301F1BF
:10067000010218BF83F0D503B8F1400FDBB2A8BF69
:100680004FF04008801A8BF88100424601F1440087
:100690008CF801308BF8C03058F062FE8BF8048182
:1006A000FEF7DEBD583D0120EC2A0708F02A0708B6
:1006B000102B0708481600204F16002040F6C822CD
:1006C0009BF84630ABF8802008228BF88220002B64
:1006D00000F021849AF84422002A40F03E858BF8ED
:1006E00083209D235B0083F0D503DBB213F0800FE2
:1006F0004FEA430318BF83F0D503DBB213F0800F3A
:100700004FEA430318BF83F0D503DBB213F0800F29
:100710004FEA430318BF83F0D503DBB213F0800F19
:100720004FEA430318BF83F0D503DBB2534013F005
:10073000800F4FEA430318BF83F0D503DBB213F0F9
:10074000800F4FEA430318BF83F0D503DBB213F0E9
:10075000800F4FEA430318BF83F0D503DBB213F0D9
:10076000800F4FEA430318BF83F0D503DBB213F0C9
:10077000800F4FEA430318BF83F0D503DBB213F0B9
:10078000800F4FEA430318BF83F0D503DBB213F0A9
:10079000800F4FEA4303BBF99E13E6488BF8842091
:1007A00018BF83F0D503DBB280FB012013F0800F6C
:1007B0004FEAE1724FEA4303C2EBA00218BF83F095
:1007C000D503C2F30721DBB24B4013F0800F4FEA91
:1007D000430318BF83F0D503DBB213F0800F4FEA59
:1007E000430318BF83F0D503DBB213F0800F4FEA49
:1007F000430318BF83F0D503DBB213F0800F4FEA39
:10080000430318BF83F0D503DBB213F0800F4FEA28
:10081000430318BF83F0D503DBB213F0800F4FEA18
:10082000430318BF83F0D503DBB213F0800F4FEA08
:10083000430318BF83F0D503DBB213F0800F4FEAF8
:10084000430318BF83F0D50312B2D2B2DBB25340D8
:1008500013F0800F4FEA430318BF83F0D503DBB2D8
:100860004FEA43081B0648BF88F0D5085FFA88F8AE
:1008700018F0800F4FEA480818BF88F0D5085FFAD3
:1008800088F818F0800F4FEA480818BF88F0D5089C
:100890005FFA88F818F0800F4FEA480818BF88F010
:1008A000D5085FFA88F818F0800F4FEA480818BF9B
:1008B00088F0D5085FFA88F818F0800F4FEA4808EA
:1008C00018BF88F0D5085FFA88F818F0800F4FEA53
:1008D000480818BF88F0D5085FFA88F88BF88510AB
:1008E0008BF886208BF8C0801FF022FDDBF8A02358
:1008F000DFF844C28BF88A00C2F3074383EA080892
:1009000018F0800F4FEA480818BF88F0D5085FFA42
:1009100088F88BF8873018F0800F4FEA480318BF2B
:1009200083F0D503DBB213F0800F4FEA430318BF07
:1009300083F0D503DBB213F0800F4FEA430318BFF7
:1009400083F0D503DBB213F0800F4FEA430318BFE7
:1009500083F0D503DBB213F0800F4FEA430318BFD7
:1009600083F0D503DBB213F0800F4FEA430318BFC7
:1009700083F0D503DBB213F0800F4FEA430318BFB7
:1009800083F0D503C2F30721DBB24B4013F0800F95
:100990004FEA430318BF83F0D503DBB213F0800F97
:1009A0004FEA430318BF83F0D503DBB213F0800F87
:1009B0004FEA430318BF83F0D503DBB213F0800F77
:1009C0004FEA430318BF83F0D503DBB213F0800F67
:1009D0004FEA430318BF83F0D503DBB213F0800F57
:1009E0004FEA430318BF83F0D503DBB213F0800F47
:1009F0004FEA430318BF83F0D503DBB213F0800F37
:100A00004FEA430318BF83F0D503D2B2DBB25340A1
:100A100013F0800F4FEA430318BF83F0D503DBB216
:100A200013F0800F4FEA430318BF83F0D503DBB206
:100A300013F0800F4FEA430318BF83F0D503DBB2F6
:100A400013F0800F4FEA430318BF83F0D503DBB2E6
:100A500013F0800F4FEA430318BF83F0D503DBB2D6
:100A600013F0800F4FEA430318BF83F0D503DBB2C6
:100A700013F0800F4FEA430318BF83F0D503DBB2B6
:100A800013F0800F4FEA430318BF83F0D503DBB2A6
:100A900043408BF88920DAB213F0800F4FEA42030B
:100AA00018BF83F0D503DBB213F0800F4FEA430386
:100AB00018BF83F0D503DBB213F0800F4FEA430376
:100AC00018BF83F0D503DBB213F0800F4FEA430366
:100AD00018BF83F0D503DBB213F0800F4FEA430356
:100AE00018BF83F0D503DBB213F0800F4FEA430346
:100AF00018BF83F0D503DBB213F0800F4FEA430336
:100B000018BF83F0D503DBB213F0800F4FEA430325
:100B100018BF83F0D503DBB28BF888108BF88B30CD
:100B2000ACF1440207CA8CE807000C228BF8C030F5
:100B300004E000BF676666668C1600208BF804210F
:100B4000FEF78BBBE24A9FEDE37AB2F9323207EE51
:100B5000903AF8EEE77A40F6C80367EE877AABF88A
:100B60008030FDEEE77A9FEDDB7A17EE901AC1F345
:100B7000072080F0FA038BF883005B00C00908BFF0
:100B800083F0D503DBB213F0800F4FEA430318BFA5
:100B900083F0D503DBB213F0800F4FEA430318BF95
:100BA00083F0D503DBB213F0800F4FEA430318BF85
:100BB00083F0D503DBB213F0800F4FEA430318BF75
:100BC00083F0D503DBB213F0800F4FEA430318BF65
:100BD00083F0D503DBB213F0800F4FEA430318BF55
:100BE00083F0D503DBB213F0800F4FEA430318BF45
:100BF00083F0D50309B2C9B2DBB24B4013F0800FCA
:100C00004FEA430318BF83F0D503DBB213F0800F24
:100C10004FEA430318BF83F0D503DBB213F0800F14
:100C20004FEA430318BF83F0D503DBB213F0800F04
:100C30004FEA430318BF83F0D5038BF88410DBB26F
:100C4000B2F93012B2F9342213F0800F4FEA4303A5
:100C500007EE901A18BF83F0D503DBB213F0800FB4
:100C6000F8EEE77A4FEA430318BF83F0D50367EE47
:100C7000877ADBB213F0800F4FEA4303FDEEE77A89
:100C800018BF83F0D503DBB217EE901A13F0800F74
:100C90004FEA430318BF83F0D503C1F30720DBB24B
:100CA000434013F0800F4FEA430318BF83F0D5038E
:100CB000DBB213F0800F4FEA430318BF83F0D50374
:100CC000DBB213F0800F4FEA430318BF83F0D50364
:100CD000DBB213F0800F4FEA430318BF83F0D50354
:100CE000DBB213F0800F4FEA430318BF83F0D50344
:100CF000DBB213F0800F4FEA430318BF83F0D50334
:100D0000DBB213F0800F4FEA430318BF83F0D50323
:100D1000DBB213F0800F4FEA430318BF83F0D50313
:100D200009B2C9B2DBB24B4013F0800F4FEA430364
:100D300018BF83F0D503DBB213F0800F4FEA4303F3
:100D400018BF83F0D503DBB213F0800F4FEA4303E3
:100D500018BF83F0D503DBB213F0800F4FEA4303D3
:100D600018BF83F0D503DBB213F0800F4FEA4303C3
:100D700007EE902A18BF83F0D503DBB213F0800F83
:100D80009FED547A8BF886104FEA4303F8EEE77A2A
:100D900018BF83F0D503DBB267EE877A13F0800FBC
:100DA0004FEA430318BF83F0D503FDEEE77ADBB2C9
:100DB00013F0800F17EE902A4FEA430318BF83F019
:100DC000D503C2F30721DBB24B4013F0800F4FEA8B
:100DD000430318BF83F0D503DBB213F0800F4FEA53
:100DE000430318BF83F0D503DBB213F0800F4FEA43
:100DF000430318BF83F0D503DBB213F0800F4FEA33
:100E0000430318BF83F0D503DBB213F0800F4FEA22
:100E1000430318BF83F0D503DBB213F0800F4FEA12
:100E2000430318BF83F0D503DBB213F0800F4FEA02
:100E3000430318BF83F0D503DBB213F0800F4FEAF2
:100E4000430318BF83F0D50312B2D2B2DBB25340D2
:100E500013F0800F4FEA430318BF83F0D503DBB2D2
:100E600013F0800F4FEA430318BF83F0D503DBB2C2
:100E700013F0800F4FEA430318BF83F0D503DBB2B2
:100E800013F0800F4FEA430318BF83F0D503DBB2A2
:100E900013F0800F4FEA430318BF83F0D503DBB292
:100EA00013F0800F4FEA430318BF83F0D503DBB282
:100EB00013F0800F4FEA430318BF83F0D503DBB272
:100EC00013F0800F4FEA43034FF01E0C04E000BF05
:100ED000583D012058A08B4118BF83F0D5038BF8F3
:100EE00082C0DBB2DFF888C38BF885008BF88710EF
:100EF0008BF888208BF889309CE807000CF1440CB3
:100F0000ACE803000A218BF8C030ACF800208BF865
:100F10000411FEF79FB99AF85232012B0CBFBAF8B0
:100F20006022BAF86222C44BA3FB0232D30AD90072
:100F30008BF8833081F09D035B00C90908BF83F003
:100F4000D503DBB213F0800F4FEA430318BF83F0E1
:100F5000D503DBB213F0800F4FEA430318BF83F0D1
:100F6000D503DBB213F0800F4FEA430318BF83F0C1
:100F7000D503DBB213F0800F4FEA43034FEAD202EE
:100F800018BF83F0D503DBB2D2B2FFF7CFBB5B0053
:100F900083F0D50358B2DBB2FFF769BA5B0083F088
:100FA000D50358B2DBB2FFF75CBA5B0083F0D50320
:100FB00058B2DBB2FFF74FBA430083F0D50358B203
:100FC000DBB2FFF742BA5B0083F0D50358B2DBB265
:100FD000FFF759BA5B0083F0D50358B2DBB2FFF7D5
:100FE0004CBAD16809066CD59AF80111002968D06D
:100FF000926802F00302032A63D0904A0421FFF7AB
:1010000016BA430083F0D50358B2DBB2FFF754BAE7
:1010100083F0D50043B2C0B2FFF748BA5B0083F05B
:10102000D50358B2DBB2FFF75FBA5B0083F0D5039C
:1010300058B2DBB2FFF752BA5B0083F0D50358B267
:10104000DBB2FFF745BA5B0083F0D50358B2DBB2E1
:10105000FFF738BA5B0083F0D50358B2DBB2FFF775
:1010600049BA430083F0D50358B2DBB2FFF75DBA4B
:1010700083F0D50043B2C0B2FFF751BA5B0083F0F2
:10108000D50358B2DBB2FFF768BA5B0083F0D50333
:1010900058B2DBB2FFF75BBA5B0083F0D50358B2FE
:1010A000DBB2FFF74EBA5B0083F0D50358B2DBB278
:1010B000FFF741BA5B0083F0D50358B2DBB2FFF70C
:1010C00052BA23F060435E495E4A23F07F03002B4F
:1010D0000ABF0A4604210221FFF7A9B95B0083F089
:1010E000D5035AB2DBB2FFF775BA5748FEF708BB13
:1010F0005B0083F0D5035AB2DBB2FFF74DBA5B0059
:1011000083F0D5035AB2DBB2FFF740BA5B0083F03D
:10111000D5035AB2DBB2FFF757BA5B0083F0D503B1
:101120005AB2DBB2FFF74ABA5B0083F0D5035AB27A
:10113000DBB2FFF73DBA5B0083F0D5035AB2DBB2F6
:10114000FFF730BADAF860379B0229D510F4016F47
:1011500026D13E4A0421FFF76AB99AF8523236493D
:10116000012B0CBFBAF86032BAF86232B3FBF2F26C
:10117000A1FB0232C2F3C723990081F0A401C9B2D6
:10118000490081F0D5018BF8833001F0FD03090699
:10119000C2F3C7023FF5A6AA5B00DBB2FFF7A6BA0F
:1011A000C30528D4C3062ED4830630D441F20803E5
:1011B000834330D0C30432D4030734D403055BD453
:1011C000C30734D4800703D5214A0321FFF72FB981
:1011D00010788BF8830080F07103C0093FF42CA9CC
:1011E0005B0083F0D50043B2C0B2FFF728B9DFF847
:1011F00058C0FFF7F7B9174A0421FFF718B9DFF80D
:1012000074C0FFF7EFB9144A0321FFF710B9134A6E
:101210000421FFF70CB9124A0421FFF708B9114A5B
:101220000321FFF704B9104A0221FFF700B90F4A62
:101230000421FFF7FCB800BFCDCCCCCC002B0708B5
:10124000F82A0708342B07084D160020182B07082A
:10125000FC2A0708202B0708886407086064070831
:10126000282B0708302B070874450708082B0708A8
:10127000481600204E160020014A0221FFF7D7B879
:10128000CC64070830B41A4C1A48D4F82C2EC16824
:10129000194B003A18BF012284F87C2011F080011C
:1012A0004FF0000483F8544783F8EA461CBF082433
:1012B00083F85B47D0F82C424FF0040240F201253E
:1012C00083F85A2708BF03226407A3F8585708D4A5
:1012D0008068C00603D483F8552730BC70470029C6
:1012E000F9D09918102081F858070132F3E700BFB0
:1012F000C8150020583D0120B8370020000000002C
:10130000002070470A4B1A7A0AB10020704709483A
:10131000094AD3F84C130068D27A4FF47A73401A12
:1013200003FB02F3984294BF00200120704700BFE6
:1013300040280020A8220020B8380020404B1B681D
:10134000590714D53F49404A0B7803EB830302EB5E
:10135000C303DB899A0511D45B0510D43B4AD378CB
:10136000052B5FD8DFE803F02D345E425216354B73
:10137000D3F8F422C3F89023C3F89423704791F96B
:101380007C3903EB430301EBC30393F8C833042B0D
:10139000E4D1F3E7138CD1EDE26A91EDBD7A07EE6B
:1013A000903AF8EEE77A77EEA67AF4EE477AF1EE25
:1013B00010FAC8BFB0EE677AC1EDE57A81EDE47A44
:1013C0007047D1F8F432C1F89033C1F894337047C4
:1013D000138C91EDBD7A07EE903AF8EEE77A77EE4E
:1013E000877AC1EDE47AC1EDE57A7047D1EDE47A10
:1013F00091EDBD7AF4EEC77AF1EE10FAD8BFF0EEB7
:10140000477AC1EDE47AC1EDE57A7047138CD1EDEE
:10141000E26A91EDBD7A07EE903AF8EEE77A77EE60
:10142000A67AE7E7138C91EDE27A07EE903AF8EEB0
:10143000E77A77EE877AC1EDE47AC1EDE57A704715
:10144000583D012040280020609C0608B838002044
:10145000034B1B7A002B0CBF02200020704700BFFB
:10146000943F01200020704738B5124890F969492F
:10147000002C11DD00231A461D4602EB420200EB50
:10148000C201013391F8C823DBB2062A08BFA1F8D4
:10149000DC53A3421A46F0DB037A0BB1C37A2BB9B3
:1014A000054BDB7A13B1FFF72DFF08B9002038BDDB
:1014B0000A2038BD40280020B83800200B4A92F995
:1014C0007C3903EB430102EBC10191F8DE13A5293E
:1014D00004D092F9691901398B4201DB0D20704764
:1014E000013382F87C390220704700BF4028002079
:1014F0000E4A0F4992F97C39096803EB430302EB6A
:10150000C303B3F9D833002B0DDDD2F88C0958B1E1
:10151000C3EB4312081A03EB8203B0EBC30F34BFD3
:101520000020022070470220704700BF40280020A2
:10153000A822002010B3124B1868F8B11879E8B14E
:10154000F0B5104A1C6A5E6A0F4F1D6B0C6002EB0F
:10155000840C02EB8602DCF878E5D2F884C5E25D03
:10156000D3E90A7305F13004C1E906ECC1E902755B
:101570004E6081F820400B610A75F0BD704700BFD6
:1015800050570020609C06081C2C070860B1074BD0
:10159000186848B1187938B110B41C6B0C70DB6A4C
:1015A0005DF8044B13807047704700BF5057002010
:1015B00030B1044B186818B1187908B19B6A0B80D8
:1015C000704700BF5057002030B1044B186818B165
:1015D000187908B100230B70704700BF50570020E6
:1015E00030B1044B186818B1187908B11B6B0B7037
:1015F000704700BF5057002060B1074B186848B1D2
:10160000187938B110B41C6A0C705B6A5DF8044B31
:1016100013707047704700BF50570020704700BFDD
:101620004A1E93B2032B17D80C4B1879A0B10C4863
:1016300000EB820210B4D2F8A8259C69A24208D31C
:10164000D869824205D8D868DA6240F0020019638E
:10165000D8605DF8044B7047704700BF50570020BA
:10166000609C06084B1ED8B201281DD8501E30B40D
:10167000C4B2072C16D80D4C25799DB10C4D00EB4A
:10168000C30305EB43032069B3F8B835834209D39C
:101690006069834206D8E068A362C4E9081240F09A
:1016A0000100E06030BC7047704700BF5057002019
:1016B000609C060818B1024B186800B11879704791
:1016C000505700200520704748B1174BD3F8D4007D
:1016D00028B193F86420022A02D80020704770478E
:1016E00070B4124AD3F88850D3F88440D3F890608D
:1016F0000C6002EB850002EB8404D3F88C20D3F855
:101700009430D4F8D8454D60C1E902620B61D0F83D
:10171000F035207808753032C1E90643012070BCED
:1017200081F82020704700BF50570020609C0608B9
:1017300080B1094BD3F8D40060B193F8640002285B
:1017400001D800207047D3F88C000870D3F894308B
:1017500013800120704700BF5057002068B1074B2D
:10176000D3F8D40048B193F86420022A01D80020AD
:101770007047D3F890300B800120704750570020FD
:1017800068B1074BD3F8D40048B193F86420022A1B
:1017900001D80020704793F8A4300B7001207047E7
:1017A0005057002068B1074BD3F8D40048B193F8E4
:1017B0006420022A01D800207047D3F88C300B70C7
:1017C000012070475057002080B1094BD3F8D40056
:1017D00060B193F86400022801D800207047D3F864
:1017E00084000870D3F8883013700120704700BF60
:1017F0005057002021B9034A536F43F00403536745
:10180000704700BF5057002040B1144BD3F8D4208C
:1018100022B193F86420022A01D870477047D9B1E9
:10182000D3F8A8209142F9DC01F10042013AD3F843
:10183000AC0010B430F81200D3F880405A6FC3F8EF
:101840008C10A04228BF204642F002025DF8044BF3
:10185000C3F894005A677047704700BF5057002084
:1018600040B1184BD3F8D40020B193F8640002289B
:1018700001D870477047481E30B4C4B2042C03D856
:10188000541EE5B2072D0DD9986F48B95C6FC3F8A7
:10189000841044F00104C3F88820C3F890005C670A
:1018A00030BC7047084D04EBC00005EB40009C6F56
:1018B000B0F81406A042F3D3DC6FA042E6D930BCE6
:1018C000704700BF50570020609C060848B1054B88
:1018D000D3F8D40028B193F86400022894BF002004
:1018E0000120704750570020042070472F4B93F879
:1018F000C120722A14D0762A10D193F8C720B3F8E9
:10190000C200B3F8C410C3F89800003A18BF01220F
:1019100083F8A420C3F89C10022070470020704771
:10192000B3F8C200B3F8C420B3F8C610C3F88010EF
:10193000C3E91E020028F2D09042EFD21C4A12895D
:1019400012B1C3F880201146B1F5487F11D2B1F52C
:10195000167F1AD2B1F5C87F19D3164A1648C3F8B4
:10196000AC2004210C3202618171C3F8A81001205F
:101970007047124A1048C3F8AC2005210C320261AE
:101980008171C3F8A810012070470D4AF2E7C729FA
:10199000FBD90C4A0848C3F8AC2003210C32026181
:1019A0008171C3F8A8100120704700BF5057002074
:1019B000343800200CA30608080A0020C4A2060838
:1019C000E8A2060830A30608124A137E012B03D0B2
:1019D000937E03700120704710B492F8221092F9A0
:1019E0001A404B1E79B1243201E0013B0BD302EBCC
:1019F000C301B1F904108C42F7DBDBB203705DF870
:101A0000044B01207047002303705DF8044B012054
:101A1000704700BF080A0020154BDA7ED20703D5B5
:101A20009B8B03800120704793F91930002B1A46D5
:101A3000B8BFDA1DC2F3C702042A09D8594201F01F
:101A4000070103F0070358BF4B42DBB2072B03D952
:101A50000023038001207047013201330549D2B2CF
:101A6000DBB203EBC20301EB4303B3F80236D8E762
:101A7000080A0020609C0608D0B170B50D4E96F99A
:101A80001A3082B013B9002002B070BD0DF107000A
:101A90000C461546FFF798FF0028F4D09DF8073054
:101AA000237013B106EBC3039B8B2B8002B070BD78
:101AB00000207047080A0020002841D0294B93F9E4
:101AC0001A20002A3CD0F0B5DA7E93F91970D307BA
:101AD00083B00D46044635D501A80026FFF79CFFCC
:101AE00000283BD020460DF106020DF10301FFF75F
:101AF000C3FF002832D07B4203F007031A4ABDF827
:101B000004402E6007F0070758BF5F4201379DF879
:101B1000033002EB8606FFB2C5E902436F6002EBB9
:101B20008707D6F8D815BDF806202A61D7F8F02522
:101B30000C782C753033C5E9061285F820300EE09C
:101B400000207047002F3E46B8BFFE1DF61001363C
:101B500001A8F6B2FFF760FF0028C3D1002003B050
:101B6000F0BD00BF080A0020609C060828B1044BA5
:101B700093F91A300BB108464EE70020704700BFBA
:101B8000080A002060B1084B93F91A0048B11A7E88
:101B9000012A07D8DB7EC3F340030B700120704796
:101BA0007047704700207047080A002028B1044B96
:101BB00093F91A300BB1084606E70020704700BFC2
:101BC000080A002008B310B4104C94F91A0080B130
:101BD000E37EDB0710D500230B7094F919305942CE
:101BE00001F0070103F0070358BF4B4201331370A4
:101BF00001205DF8044B704794F91930002BB8BFF1
:101C00000733DB100133DBB2E6E77047080A002038
:101C100028B1034B93F91A00003818BF0120704710
:101C2000080A002003207047002852D070B5374CB6
:101C300094F91A3082B0002B49D00D46002951D0BA
:101C400094F82230AB4245D394F850300093304A98
:101C50002B46042109204DF07BFF237E013D022B02
:101C6000EDB241D0032B48D0012B40D0294D0022AA
:101C700028466E1D10F8013B08215A40530012F00F
:101C8000800F08BF520083F0D50314BFDAB2D2B27E
:101C90000139F3D1B042EDD11F48204B90F8D81054
:101CA00084F851204A1CA3FB02439B0890F8D940BA
:101CB00003EB4303A2EB4303A34208D000EBC101B3
:101CC0000622C1F8DC5080F8D830C1F8E02002B01C
:101CD00070BD7047124A0421092002B0BDE870406F
:101CE0004DF036BF0F4AF6E784F85050BEE704EBDC
:101CF000C5052B8D84F85030B8E704EBC50595F881
:101D0000283063F07F0384F85030AFE7080A0020E2
:101D10005C2C0708540A002050570020ABAAAAAA3E
:101D2000482C0708202C07080139CBB2042B48D8CF
:101D3000013AD1B2072945D8F0B5DFF898C001EBD8
:101D4000C3070CF15405FFB283B02E468CF85870CF
:101D50000CF1590E002016F8012B082450404200C7
:101D600010F0800F08BF400082F0D50214BFD0B23F
:101D7000C0B2013CF3D1B645EDD1CDE90017124A0E
:101D80008CF85900042109204DF0E2FE0F49104B58
:101D900091F8D82091F8D940501CA3FB00639B0810
:101DA00003EB4303A0EB4303A34208D001EBC202C1
:101DB0000620C2F8DC5081F8D830C2F8E00003B049
:101DC000F0BD7047704700BF842C070850570020B3
:101DD000ABAAAAAA080A002070B5304C237E40F0B6
:101DE0000802022B84B084F860204ED800F004066C
:101DF0002B4B2C4A2C49039110F0010F14BF1546B0
:101E00001D4610F0020F0CBF194611460095002E1A
:101E100008BF1A46254DCDE901120346244A092080
:101E200004214DF095FE6E1D0022284610F8013B5E
:101E300008215A40530012F0800F08BF520083F06F
:101E4000D50314BFDAB2D2B20139F3D18642EDD153
:101E50001848194B90F8D81084F861204A1CA3FB4D
:101E600002439B0890F8D94003EB4303A2EB4303E2
:101E7000A34208D000EBC1010622C1F8DC5080F873
:101E8000D830C1F8E02004B070BD10F00406AFD027
:101E900083071CBF012384F82030A9E7080A00202B
:101EA000D02C0708CC2C0708042D0708640A002052
:101EB000D42C070850570020ABAAAAAA00286AD041
:101EC000534890F91A30002B4AD0037E002B48D09B
:101ED00070B584B0002947D0022B43D990F8202058
:101EE000002A40F08680802300F1640580F8683085
:101EF0002C4600F1690614F8013B08215A405300B2
:101F000012F0800F08BF520083F0D50314BFDAB27D
:101F1000D2B20139F3D1B442EDD13E4C3E4B94F8EC
:101F2000D81080F869204A1CA3FB02039B0894F890
:101F3000D90003EB4303A2EB4303834208D004EB35
:101F4000C1010622C1F8DC5084F8D830C1F8E02085
:101F5000324A0421092004B0BDE870404DF0F8BDBC
:101F60007047704704B070BD022B15D8042490F957
:101F70001B2012F00800D3B218BF44F002045B0724
:101F800013D439B3002C32D1002834D02449254849
:101F90000B46012410E0704790F82030002BE5D16B
:101FA0000420FFF719FF204AD3E744F00104B1B140
:101FB00050B31B490B460846CDE90021CDE9020488
:101FC0001A4A042109204DF0C3FD204604B0BDE8A3
:101FD000704001E7134B38B111491248ECE778B96A
:101FE00010490F480B46E7E70E490846E4E70C4B5B
:101FF000F1E70024BBE70B49094B08460124DBE766
:10200000084B07490648D7E7054B0649FAE700BFE2
:10201000080A002050570020ABAAAAAA102D0708D2
:10202000DC680708D02C0708382D0708642D07083E
:1020300010B50F4A042109204DF08AFD0D490E4BC1
:1020400091F8D82091F8D940501CA3FB00C39B08FD
:1020500003EB4303A0EB4303A34207D0074881F8F7
:10206000D83001EBC2020523C2E9370310BD00BF1F
:10207000AC2D070850570020ABAAAAAA740A00206A
:102080000A4BD0B51C6814F0100403D0BDE8D04052
:1020900044F006BD44F004FD054B00260027C3E9CB
:1020A0004401C3E94667C3E94844D0BD603D01200F
:1020B0005057002008B544F0F3FC034B01221A727C
:1020C000C3E90001022008BD943F01201B4B1B689F
:1020D00010B51B4CDB06D4EDE67A08D5194BB3F8E6
:1020E000583007EE103AB8EEC77A77EEC77A9FED10
:1020F000167AF4EEC77AF1EE10FA04DAD4EDE57A46
:10210000C4EDE97A10BD94EDEA7ADFED100AB8EE7D
:10211000470AB7EE001A80EE270A4DF029FBF7EECA
:10212000007A77EEC07AD4EDE56A94EDE47A67EE52
:10213000A67AE0EE077AC4EDE97A10BD603D012091
:1021400040280020B83800200000C84200000000ED
:102150002DE9F041354D364FD5E900322DED028B9A
:10216000C01A82B061EB020151F0E0FC9FED318AB0
:10217000B7F86A6007EE900A27EE888A2EF0A0FA78
:1021800000284DD1BCEEC88A18EE103A9E4205D206
:10219000012002B0BDEC028BBDE8F081DFF89C802D
:1021A000B7F86430DFED240A01EE903AB8F9063052
:1021B00007EE906A02EE103AB8EEC88AB8EE671AD7
:1021C000B8EEC22AF8EE611AB0EE480A04468DED68
:1021D000011A4DF0ADFA97F87230DFED170A9DED58
:1021E000011A01EE903AB8F90230FDEEC07A02EE23
:1021F000103A17EE903AB8EEC22AF8EE611AB0EE35
:10220000480AA8F806304DF093FAFCEEC07A204652
:1022100017EE903A6B7202B0BDEC028BBDE8F08114
:10222000032002B0BDEC028BBDE8F081943F012099
:10223000B83800206F12833A000000007C3F012074
:10224000274AF8B5D2E90032C01A61EB020151F019
:102250006DFCDFED247A244D07EE100A67EE277A35
:10226000B5F86630B5F86C20FCEEE77A17EE904AC8
:10227000234493422DD8B5F86860B5F86470A6423F
:1022800003D21A4B0120DF80F8BD2CF0A3F8B5F87B
:102290006230DFED170A07EE907A9842B8BF184611
:1022A000B8EE672A07EE906A83B201EE903AB8EE74
:1022B000671A07EE904AF8EE611AB8EEE70A4DF099
:1022C00037FABDEEC00A094B10EE102A0020DA8062
:1022D000F8BD2EF0F5F90028CDD00320F8BD00BFE1
:1022E000943F01206F12833AB83800207C3F0120D0
:1022F00000000000F8B5204D204BB5F87070B5F81F
:102300006420DA8004460E4617BB1D4BD3E900015A
:10231000201A66EB010151F009FCDFED1A7AB5F8DD
:102320006630B5F86810B5F86C2007EE100A67EE55
:10233000277A0B44FCEEE77A17EE904A2344934247
:1023400013D8B5F86E00844294BF00200120F8BD78
:10235000F9F748FC07EE907AF8EEE77AB4EEE70A70
:10236000F1EE10FAD1DB0120F8BD2EF0A9F900281A
:10237000E7D00320F8BD00BFB83800207C3F012023
:10238000943F01206F12833A70B504460D46FAF768
:102390009FF8124B124ED3E90001201A65EB0101A0
:1023A00051F0C4FBDFED0F7AB6F86C3007EE100A7F
:1023B00067EE277AFCEEE77A17EE904A9C4206D841
:1023C000B6F86600A0422CBF0020012070BD2EF0A0
:1023D00077F90028F4D0032070BD00BF943F01209E
:1023E000B83800206F12833A08B5FAF771F8002068
:1023F00008BD00BF2DE9F84305462DED048B0020F4
:102400000F462EF031F9002800F097806B4C9FEDBD
:102410006C7AD4ED067AF0EEE76AF4EEC76AF1EE74
:1024200010FA5FDD94ED087A664E94ED078A87EE28
:10243000279A2BF0F3FF96F8733007EE903A9FED52
:10244000627AF8EEE77AF0EE408A27EE870A4DF0DE
:102450008FFAB6F85E3007EE903AF8EEE77AB4EE0F
:10246000E78AF1EE10FA6DDC4FF00009B6F85C80F7
:1024700007EE908AF8EEE77AF4EEC97AF1EE10FAF8
:1024800040F18480B5EEC08AF1EE10FA7EDD13F0E3
:10249000F5FF002873D04D4BB3F9243098456EDB1F
:1024A0004FF00109FAF714F8B9F1000F60D0D4E940
:1024B0000001281A67EB010151F038FBDFED447A87
:1024C000B6F8604007EE100A67EE277ABDEC048B81
:1024D000FCEEE77A17EE903A9C422CBF00200120D8
:1024E000BDE8F883374E94ED078A2BF097FF96F8F6
:1024F00073309FED357A07EE903AF8EEE77AF0EE1A
:10250000408A27EE870A4DF033FAB6F85E3007EEC0
:10251000903AF8EEE77AB4EEE78AF1EE10FA1BDDB6
:10252000F4EEC08AF1EE10FA2CDB13F0A7FFB6F838
:102530005C8020B34FF001092CE0BDEC048B04203B
:10254000BDE8F883F4EEC08AF1EE10FAACBF4FF0AC
:1025500001094FF0000989E713F090FFB6F85C30ED
:1025600020B11A4AB2F92420934224DBF9F7B0FFD4
:10257000BDEC048B0020C4E90057BDE8F883F9F7EF
:10258000A7FF94E7B6F85C804FF0000913F076FFE0
:10259000002887D00D4BB3F92430434582DDF9F78D
:1025A00097FFB9F1000F82D1B5EEC08AF1EE10FAB3
:1025B0003FF77DAFDCE7F9F78BFFF5E7943F0120AC
:1025C000F366DF3FB838002035FA8E3C88170020CC
:1025D0006F12833A70B504462DED028B00200D4634
:1025E0002EF042F8002851D02A4ED6E90001201AD8
:1025F00065EB010151F09AFA9FED270A07EE900A68
:1026000027EE800A40F2DC53BCEEC00A10EE102A1E
:102610009A4235D8214CB8EEC08A2BF0DBFEB4F8D4
:1026200062309FED1F1ADFED1F0A07EE900A02EEDF
:10263000103AF8EEE71AB8EE422AB0EE480A4DF02A
:1026400077F894F87230DFED171A174A9FED141AD5
:10265000FDEEC07A02EE103A17EE903AB0EE480A5C
:10266000B8EE422AF0EE610AD3804DF061F8BDEC7D
:10267000028BFCEEC07A002017EE903A737270BDA8
:10268000F9F726FFBDEC028B012070BDBDEC028B7B
:10269000042070BD943F01206F12833AB8380020A7
:1026A0000080BB44000000007C3F012038B5134D82
:1026B00044F0F6F92B7A032B0ED8114B1C6814F05A
:1026C000804401D1204638BD00202DF0CDFF0446C6
:1026D00048B10024204638BD05230224C5E9000185
:1026E0002B72204638BD2DF0EBFF0028EAD00022E7
:1026F00000232C72C5E900230424E3E7943F012062
:10270000643D012008B50E202DF064FE00B108BD27
:10271000024B1868C0F3807008BD00BF643D012003
:10272000914B1B6813F004032DE9F04700F09380F0
:102730008E4B1A79002A5ED18D4A8E4C237AE77926
:102740001BB1637A022B00F0A280218940F20223A0
:10275000994200F0AA8000264FF00008237894F8F0
:10276000681903EB830302EBC303B3F80E9009F47B
:10277000007900294DD094F96939002B49DDB9F170
:10278000000F46D17C4BD3F800A01AF0100F4AD1AD
:10279000A37C002B5CD108202DF01CFE002864D007
:1027A000B9F1000F54D116B1B8F1000F4BD10A2086
:1027B0002DF010FE002840F08F8013202DF00AFE2F
:1027C000002800F08F806D4B1B681C0511D46C4BEA
:1027D00093F82831002B00F08980002E00F08680CD
:1027E000B8F1000F00F08280002F7FD01AF0010FA7
:1027F0007CD009202DE05A79002A9DD093F828300A
:102800005B4A03EB430302EB430393F8F4364BBB01
:1028100093E75B4D002385F82831574BD3F800A090
:102820001AF0100FB4D0FFF76DFF0546002844D012
:10283000534D95F82901002840F08B804F4B1B68C1
:102840001A06A5D505E0002FB1D01AF0010FAED0C1
:102850000720BDE8F0874A4C84F82831FFF752FF83
:1028600084F829010420BDE8F08713202DF0B2FD83
:1028700070B3434D95F82831002B91D00A202DF0EC
:10288000A9FD50BB3D4B1B681B05A6D5B1E7E67AF9
:10289000002E3FF461AF218940F2022399424FF0AC
:1028A00001067FF459AFB04658E7E67A002E3FF4B0
:1028B00053AF00264FF0010850E7304B1B681B0652
:1028C0007FF566AF2DF0D0FE0028CBD02846C0E7BC
:1028D0000A202DF07FFD28B1294D002385F82831ED
:1028E0000420B6E7264B012283F8282109202DF089
:1028F00071FD38B1214B1B68980601D416B10FB198
:102900000620A6E723202DF065FD78B103202DF0E9
:1029100061FD1A4B1B68B0B141F208029A4320D006
:10292000E6B1002F0CBF1020112092E703202DF0FC
:1029300051FD002896D0114B1B68190701D4002FB8
:1029400090D0052085E703F4805333438AD01020CC
:102950007FE7002385F829310B207AE7DA04ECD5EC
:10296000F5E7112075E700BF583D0120983D002094
:10297000609C060840280020603D01205C3D01204D
:102980005057002070B5204B5C7AACB11F4EB47C20
:10299000A4B9054618B91E4B1B685B030CD4284626
:1029A00020F0A0F91B4B1B8A98420ADC1A4800EB66
:1029B00085050023C5F82C31204670BD0024204633
:1029C00070BD154A154802EB85020368D2F82C1138
:1029D00069B15B1AC3F5BB630433002BB8BF5B421C
:1029E000B3F5FA7FE8DA012D05D00124E4E70368A6
:1029F000C2F82C31E0E7D6F8F432C6F890332C4612
:102A0000C6F89433D8E700BFB8380020402800202B
:102A1000603D0120D423002050570020A822002030
:102A200010B50A4C0A482146F8F768FFD4E90A2392
:102A30000849094C0948A1FB02C281FB03C1DB170D
:102A40005209C3EB61132260038010BDC02B00202C
:102A50008C3D00201F85EB51903A0020FC3D00206A
:102A600070B5D40722D41C4C94F87C53960708D533
:102A70008268C4F888239A074CBF45F0020505F028
:102A8000FD055B07C4F88C1322D405F0FB05002379
:102A9000C4E9EA3384F87C53FEF750FCFFF7C0FF2B
:102AA0000E4A136843F00103136070BD0A4C456879
:102AB0000668C4F8845394F87C53C4F88063DE0736
:102AC0004CBF45F0010505F0FE0584F87C53CDE7C9
:102AD00045F00405DBE700BF40280020603D0120F1
:102AE00038B507EE901ADFED196A9FED197A194B88
:102AF000F8EEE77A2DED028BC7EEA68A597C03F536
:102B0000417503F53B73002908BF1D46044607EED7
:102B1000902A68EE878AB8EEE78AB0EE680A4CF031
:102B200027FFD5ED007AE8EE007AB0EE680AC4ED32
:102B3000007A4CF097FFD5ED017AAB68A360E8EE20
:102B4000007ABDEC028BC4ED017A38BD0000C842AA
:102B500035FA8E3C4028002008B527F04BF80220BB
:102B600008BD00BF08B5064B1B689B0202D5054B8C
:102B70009B7913B107203BF093FC022008BD00BFF6
:102B8000603D0120B8380020134991F97C2902EBFF
:102B9000420301EBC303500093F8C833013B072BFA
:102BA00017D8DFE803F014160E04161616160244A2
:102BB00001EBC201B1F9D833002B14BF0C200F2058
:102BC0007047064B1B68C1F88C390E2070470220F5
:102BD00070470C20704700BF40280020A82200202A
:102BE000F8B5294C002504F14E06206844F02EF873
:102BF00098B194F86030002B44D1206844F01EF85E
:102C0000E36D5BB90F28F0D1012384F84C002068F4
:102C1000E36544F01BF80028EBD1F8BD0F2B05D875
:102C2000E2180133E36582F84C00E36D102BDCD130
:102C300094F84C300F2B03D084F86050E565D4E74E
:102C400094F84D3094F83D209A42F5D194F85B20E9
:102C5000002AF1D10D4A94F85A7002F10C0012F8D2
:102C6000011F0B448242DBB2F9D19F42E4D10849F3
:102C70000C22304656F07FFD0028DDD0012084F87C
:102C80006000F8BD0020F8BD505700209D5700207F
:102C90008E570020F8B5334C002602270125D4F8C2
:102CA000D40043F0D3FF90B1D4F8D40043F0C6FF72
:102CB000D4F8D03063B90F28F1D184F8C000D4F82B
:102CC000D400C4F8D05043F0C1FF0028ECD1F8BDC7
:102CD000012B1CD00F2B07D8E2180133C4F8D030D9
:102CE00082F8C000D4F8D030102BD8D11E4A94F806
:102CF000CEC002F10D00002312F8011B0B448242EA
:102D0000DBB2F9D19C450ED0C4F8D060C7E7A0F182
:102D10007203DBB2012B01D97628F5D1C4F8D0704B
:102D200084F8C100BBE794F8CF30002BECD1D4F885
:102D3000C020D4F8B0309A4201D00120F8BDD4F8B8
:102D4000C420D4F8B4309A42F7D1D4F8C820D4F8CB
:102D5000B8309A42F1D1D4F8CC20D4F8BC309A42A1
:102D6000EBD1D1E7505700201158002038B51A4D4B
:102D70000F22034685F83D0085F83C2011B30C4630
:102D800007CCC5F83E0095F83E00C5F84620C5F8CA
:102D9000421005F13E0202F10B0101E012F8010FB1
:102DA00003448A42DBB2F9D100240C49286885F833
:102DB0004A30102285F84B4043F04CFF85F86040C4
:102DC000EC6538BDC5F83E10C5F84210C5F8461090
:102DD000084605F13E02DEE7505700208C570020E0
:102DE00030B5894CD4F8383140F20712934285B09F
:102DF00000F0C080B3F5847F21DB40F20D129342D6
:102E000000F09B8040F21B12934216D194F8603080
:102E1000002B51D1FFF7E4FE002800F0AD8094F8BC
:102E20006030002B48D1A3680133A360022B59DD29
:102E3000002323710023C4E94E3305B030BD002BBD
:102E400000F08780F52B33D1704D94F8603053B982
:102E5000FFF7C6FE002800F09A8094F8603013B99E
:102E600023796BB977E0B4F85000B4F84E30B4F879
:102E7000522023610021C4E905010123E26123718D
:102E800028680023C4E950034FF47A7140F2071216
:102E9000A360E360C4F84811C4F838212B68D4F863
:102EA0004011D4F848215B1A934236DCD4F838310B
:102EB000002BBFDB05B030BDB4F84E20A16AB4F8DA
:102EC0005030626300208A42A363A06003D0E268AE
:102ED00042F00102E260E26A934203D0E36843F009
:102EE0000203E3602379002BA4D0484DE3682A68ED
:102EF000C4F8402100204FF47A71C4E9510140F236
:102F00000712C4F83821002B7CD013F0010248D1FD
:102F100013F0020366D1E36019E000217620FFF789
:102F200025FF2B68C4F840310021FA2240F21B1320
:102F3000C4E95112C4F8383168E7344BD4F8401171
:102F40001B68D4F848215B1A93427FF776AFA368D9
:102F50006CE72E4D237100217220FFF707FF2B68CD
:102F6000C4F840310021FA22F523C4E95112C4F813
:102F700038316AE7E368C6E7244BD4F840111B6890
:102F8000D4F848215B1A93423FF749AF8EE72B688C
:102F9000D4F84011D4F848215B1A93423FF75DAF53
:102FA00084E70025238D019501A94620CDE902552E
:102FB000ADF80430FFF7DAFE144BE26819681B68BD
:102FC000C4F844515B1AFA2522F0010240F20D10B8
:102FD000AB42C4F84011E260C4F84851C4F838016B
:102FE000B5DC2AE7A38D019201A95020CDE9022288
:102FF000ADF80430FFF7BAFED4E9023222F0020243
:10300000E26013E7014D49E750570020A822002055
:1030100038B5124C00230F25A4F8B210C4E92E33A2
:1030200084F8B10084F8B050C4F8B43004F1B102AF
:1030300004F1BD0101E012F8010F03448A42DBB242
:10304000F9D10749D4F8D40084F8BE30102243F0F7
:1030500001FE0023C4F8D03038BD00BF5057002017
:103060000058002010B5694CD4F8D430002B31D072
:1030700094F86430062B2DD8DFE803F02D37425149
:1030800069760400FFF706FE00287AD00023236744
:10309000FEF72CFC022840F09480636FD90708D417
:1030A000D4F89810D4F8902091421CBF43F001034B
:1030B00063679A0708D4D4F89C10D4F894209142FE
:1030C0001CBF43F002036367514A03231268A266E0
:1030D00084F8643010BD4E4A1268A26600230122B3
:1030E000C4E91C3384F8642010BD00217220FFF76E
:1030F0008FFF474A02231268A26684F8643010BD2D
:10310000FFF7C8FD002850D0FEF7F0FB012865D07E
:103110003F4A00231268A26684F8643010BD636FD2
:10312000002B64D0590753D4DA0768D49807D1D557
:1031300023F00203B4F8941063675020FFF768FF90
:10314000334A04231268A26684F8643010BD304A02
:10315000A16E13685B1AB3F57A7FBBD91368A366B7
:10316000052384F8643010BD00217620FFF750FF5E
:10317000274B19681B680622C4E91A3184F86420B9
:1031800010BD234AA16E13685B1AB3F57A7FA1D9EB
:10319000236F0133032B23671368A366D6BF052370
:1031A00084F8640084F8643010BD194AA16E136875
:1031B0005B1AB3F57A7F8DD91368A36684F864002F
:1031C00010BD134A05231268A26684F8643010BD4E
:1031D00023F00403002173206367AFE70C4B1B68E7
:1031E000A36600220523226784F8643010BD084AD4
:1031F000E16E13685B1AB3F5FA6FAFD810BD23F018
:103200000103B4F890106367462097E750570020F9
:10321000A822002070B5164C94F8D93094F8D82024
:103220009A4224D004EBC303D3E93750002809DDC8
:103230002B181049013B6A1E12F8016F01F8016B4F
:103240009A42F9D1AB78C4F850015B0884F8543144
:10325000F9F7F0F894F8D920074B0132A3FB0213D9
:103260009B0803EB4303A2EB430384F8D93070BD02
:10327000505700204C380020ABAAAAAA2DE9F04FE5
:10328000B54D2DED028B28688BB0002800F09F8093
:103290009FEDAF8BCDE904ABB04CB14EDFF8E892B7
:1032A00043F0D4FC002845D0286843F0C7FC94F8CC
:1032B0005531052B39D8DFE803F08F9B95A42E03F9
:1032C000D4F8747102374FFA87FEBEF1000F40F355
:1032D0007C82DFF8B8C20023E6441CF8012B0821E9
:1032E00053405A0013F0800F08BF5B0082F0D502F4
:1032F00014BFD3B2DBB20139F3D1E645EDD1984228
:1033000000F0468194F85831D90740F193800023AA
:1033100084F8553109E0D4E95D23E1180133934283
:1033200081F85A01C4F8783179D0286843F08EFCCE
:103330000028B9D13288092A09D97188642303FB8E
:1033400001F3B3FBF2F3452B40F38480306094F833
:10335000C231012B00F0AB80022B00F0D080002B9B
:1033600000F0C7807F4B94F854211D687AB17E4AE3
:10337000D2E90031B5EB030A4FF0000363EB010B18
:10338000BBF1000F08BFBAF1790F80F0C18094F84B
:10339000D82094F8D9309A4253D1D4F8CC31EB1AD2
:1033A000B3F57A7F13D2704BD3E90021AB1A0693A1
:1033B0004FF0000363EB01030793DDE90634002CB3
:1033C00008BF962B03D3FEF733FEFFF723FF0BB0A6
:1033D000BDEC028BBDE8F08FAA28A6D1012384F8AA
:1033E0005531A2E7032384F8580184F855319CE74E
:1033F00055287AD0B38800220133B38084F8552150
:1034000093E7132884F85901C4F874010BDC30B138
:1034100000220423C4F8782184F8553185E7052378
:1034200084F8553181E7F38800220133F38084F872
:1034300055217AE7338901333381002384F85531EC
:1034400073E7FFF7E7FEC4F8CC510BB0BDEC028B7D
:10345000BDE8F08F454F464A042109204CF078FB27
:10346000D7F8A430B7F8A810012B5CD05A1C03D1B0
:10347000B1F5965F00F0858203EB830303EB8303D2
:1034800001EB43039BB23B4AA7F8A8300421092073
:103490004CF05EFB2868B7F8A81003681B699847D2
:1034A0000023336094F8C231012B7FF455AF2F4FC6
:1034B0003B7E002B3FF456AF022B00F01B82032211
:1034C00084F8C221012B7FF64DAFF87E2A492B4BA1
:1034D0002B4AC0F34000002818BF0B4687F8200095
:1034E000042109204CF034FB3CE7022384F85531D9
:1034F0001BE7FEF79DFD012384F8C23132E71B4B29
:10350000DB8B002B3FF42EAF032384F8C23129E775
:10351000D4F85001F8F78EFFC4F8CC510BB0BDECD5
:10352000028BBDE8F08F41F256329142A4D1154A88
:103530004FF0FF3304210920C7F8A4304CF008FBFA
:10354000D7F8A430B7F8A81096E700BFAFF3008013
:1035500000000000000024404838002050570020A0
:10356000A8380020A8220020A0380020080A002047
:103570006C300708B4300708CC2D0708C42D0708A5
:10358000E030070880300708200A0020A8580020F3
:1035900094F8588194F85431984500F01B81B8F1A3
:1035A000090F00F01481B8F1110F00F0108171893A
:1035B000B24ACDF8008001317181092004214CF01C
:1035C000C7FA08F1FF38B8F1100F00F21381DFE8F5
:1035D00018F011006A006A003B0115011101110188
:1035E000110111001101110111011101110111014C
:1035F00011011100062F56DD94F85821012A03D03D
:10360000092A0CBF0222032294F85D0194F85E118E
:10361000DFF8D48294F85C3194F85BB188F8182014
:1036200041EA0021A8F81C1094F85A0188F8190002
:10363000990788F81B3018D513F00C0398F8201060
:1036400014BF01200020814282460CD08C488D4955
:103650008D4A002B0CBF03460B46042109204CF079
:1036600077FA98F8182088F820A0032A00F08C81B7
:103670000BF1010388F81A3094F895310C2B12D114
:1036800098F91B2098F9191098F81830C4F89C1173
:10369000642101FB0323B8F81C1098F91A20C4F820
:1036A0009831C4E96812794BD9F800101A68914230
:1036B00000F09480DFF83082754A98F81830754F22
:1036C000DFF82CB2042109204CF042FA98F91B30A3
:1036D00071487249724A13F0010F08BF0146009108
:1036E000092004214CF034FA98F81B306D4A13F08D
:1036F000020F14BF5B463B46042109204CF028FA18
:1037000098F81B30684A13F0040F14BF5B463B4621
:10371000042109204CF01CFA98F81B30634A13F07E
:10372000080F14BF5B463B46042109204CF010FAF9
:1037300098F81B005E495F4B5F4A10F0100F18BFEE
:103740000B46092004214CF003FA98F81B105B4B40
:103750005B4A11F0200F08BF3B46042109204CF0C2
:10376000F7F998F91930574A042109204CF0F0F97B
:10377000B8F81C30544A042109204CF0E9F998F9B2
:103780001A30524A042109204CF0E2F9B8F81E30F0
:103790004F4A042109204CF0DBF998F820004D49EC
:1037A0004D4B4E4A002808BF0B46042109204CF01F
:1037B000CFF999E80700354B03C31A8073880133AA
:1037C0007380002384F85531AFE5002397E5012B82
:1037D0007FF4EDAE002384F85431F2E6404A596894
:1037E000106888427FF466AF92881B899A427FF402
:1037F00061AFDEE7B3890133B381DFE794F85A3173
:103800002E4A244994F85BC194F85C7113F0010FBF
:1038100014BF1046084613F0020F009014BF104664
:10382000084601901CF0040F224808BF0A4617F012
:10383000080F1F49029208BF01460391294A04213B
:1038400009204CF085F92EE7042F7FF72CAF94F870
:103850005A3194F85B2142EA03221346580412B20B
:1038600000F19A80002AC0F2A1801F491F4A8B8371
:10387000092004214CF06CF915E700BFF42D07086E
:10388000C42D0708CC2D07081C2E07080859002056
:10389000B02F0708D02C0708E42D0708DC2D0708F7
:1038A000CC2F0708E42F0708F02F0708F82F070888
:1038B000042D0708D42D070804300708DC68070822
:1038C0001030070820300708303007083C30070860
:1038D00048300708F02D0708EC2D07085830070876
:1038E000240A0020682F0708080A0020442F070830
:1038F000CC2C07089F4A092004214CF029F907F134
:10390000AC054023A7F8B030284607F1B2060022E4
:1039100010F8013B08215A40530012F0800F08BFF5
:10392000520083F0D50314BFDAB2D2B20139F3D119
:103930008642EDD1FB7E87F8B22013F0010203D15D
:10394000BB8BB3F5804F3BD094F8D91094F8D820B6
:10395000894B501CA3FB00639B0803EB4303A0EBC4
:1039600043038B4208D004EBC2020721C2F8DC50AB
:1039700084F8D830C2F8E010022384F8C2313B7ECC
:10398000A0E57E4A0123D5E5092F56DC7C4A0421B7
:1039900009204CF0DDF886E67A497B4AC3F30D0333
:1039A000CB83092004214CF0D3F87CE67549774A93
:1039B000C3F30D03CB83092004214CF0C9F872E650
:1039C00095E80300724EC4F8C401090C4FF4A073CB
:1039D00084F8CA11304606F1060CA4F8C83110F874
:1039E000013B08215A40530012F0800F08BF5200DB
:1039F00083F0D50314BFDAB2D2B20139F3D18445D2
:103A0000EDD194F8D8305C4884F8CA2103F1010C58
:103A1000A0FB0C02920894F8D91002EB4202ACEB26
:103A200042028A42A8D004EBC3030720C3F8DC603B
:103A300084F8D820C3F8E0008AE794F960010522F1
:103A400000214BF0A5FEC3B288F8223088F87A3006
:103A5000002B4FD04FF0000B5F4606E098F8223065
:103A600001377FB29F42BB4644DAE21908EBCB0331
:103A700092F862A1A3F828A007EE90AAB8EEE77A20
:103A8000F2EE047AC7EE277A17EE900A4FF00EFC9A
:103A9000B0EE480AF0EE680A41EC110B52F024FF38
:103AA00051EC100B4FF00AFF3A4A80B200F11903B3
:103AB000A2FB03231B094FEACB02BAF10E0F4244CB
:103AC00003EB830303D903EB83035B0098B2052F59
:103AD0005062C3DC08A9F5F7BDFA2F4A0BEB8B0344
:103AE000134408A9184655F092FE08EB8B0BCBF84F
:103AF0009000B3E7B8F94070B8F93800B8F9301061
:103B0000B8F92820CDE90207CDE900210920234A90
:103B100004214CF01DF894F85F7194F85B31009328
:103B20004FF0000B3B461E4A88F81AB004210920CA
:103B30004CF00EF898F82230002B3FF49DAD98F928
:103B40001A00DC465946012208EBC10E51B2BEF9FB
:103B500028E0774504BF08464FF0010C0132994236
:103B6000D2B2F1DBBCF1000F3FF486AD88F81A0049
:103B700082E500BFC4300708ABAAAAAA9C30070898
:103B8000502E0708080A0020FC2E0708202F0708DF
:103B9000145900201F85EB51CC5800208C2E0708AB
:103BA000C02E07082DE9F0414C4C94F8D05182B05A
:103BB00015B102B0BDE8F081494B1D68002DF8D069
:103BC000484B494A07460E469878116884F8D60152
:103BD0001A889888A4F8D421A4F8D8019A7918787A
:103BE00084F8DA214B0734D594F8DE31012B3ED02E
:103BF000022B18D0002B5BD02B68196819B13A46FC
:103C000033462846884794F8DE31384A0133A2FB10
:103C1000031202F4FF7101EB52029B1A84F8DE31A9
:103C200002B0BDE8F0810DF10701284642F0CCFE5C
:103C30000028E1D094F8DF31002BDDD09DF807306B
:103C4000002184F8DF11002BD6D0284642F0C4FEB4
:103C5000D2E7274B1B79002BC6D1012A03D0022AB9
:103C6000C2D10B07C0D4012384F8D631BCE72B683E
:103C70000028C2D0D3F81880B8F1000FBDD00DF1E4
:103C800007020DF106012846C0470028B4D094F879
:103C9000D4119DF8063094F8D5218B4203D19DF8BC
:103CA00007309342A8D0284642F0ACFE2B68A4E728
:103CB0002B68DA69002AA0D00DF107012846904749
:103CC000002899D094F8D6119DF807308B4293D0F4
:103CD000284642F087FE2B688FE700BF5057002030
:103CE0003038002034380020583D0120ABAAAAAA61
:103CF000983D002038B52D4C94F8E031022B26D0A9
:103D00002B4DD5ED097A012BB8EEE70A3DD09FED9A
:103D1000290AF0EE407A284BDFED280AC3ED2D7A10
:103D200052F020FFF7EE007A37EEC00ADFED247A7A
:103D300020EE270A84ED840A52F018FD214A03463A
:103D4000042102204BF004FF0020E86138BD184D2B
:103D50009FED1D0AD5ED097ADFED180AF8EEE77A36
:103D600087EE800A52F0FEFEF7EE007A37EEC00AC8
:103D70009FED137AD4ED847AD0EE077AFDEEE77AE0
:103D800017EE900AC5ED077A38BD04F5F0704CF0D7
:103D900071FA94F8E031012BD6D0022BB7D1D4EDD3
:103DA0007E7A9FED097A87EE870AB4E750570020A4
:103DB000D43D002000000000080A0020B1DC423E93
:103DC000D048874A0431070880E6C54708B5094B43
:103DD0001B681B0603D5BDE808402AF031BB2AF05A
:103DE0002FFB00B108BD044B93F81902003818BF2F
:103DF000012008BD843F0120505700202DE9F04DDF
:103E0000D94CD4E9D8232DED068B0646801A96B0FE
:103E10000F4661EB03014FF089FEDFEDD47AC4F861
:103E2000606307EE100A67EE278AC4F86473CDED6D
:103E3000098A2AF01DFB8046002800F02882D4ED74
:103E4000E07A94ED949AD4EDE19AC94BF4EEC97AF4
:103E5000F1EE10FA9CBFB7EE007A38EE877AB4EE36
:103E6000E99A94BF27EE277AB0EE677AF1EE10FA5E
:103E70008DED0C7AA4BFB7EE007A38EE877A196818
:103E8000ACBF27EE297AB0EE697A11F080058DED8E
:103E90000B7A22D0B74B93F85453F5B1D4E99A3248
:103EA000F31A9A4667EB02039B46B34A00235B452D
:103EB00008BF5245C0F00D8494EDA37AB4EEC79AC2
:103EC000F1EE10FA40F3058494EDA47AB4EEC79AAB
:103ED000F1EE10FACCBF032501254B0710D5D4E92C
:103EE000A632F31A009367EB02030193DDE900ABFE
:103EF000A24A00235B4508BF524528BF45F0040590
:103F0000C80610D5D4E9AE32F31A029367EB020368
:103F10000393DDE902AB9A4A00235B4508BF524593
:103F200028BF45F00805490613D594F8F03283B14F
:103F3000D4E9BA32F31A049367EB02030593DDE97F
:103F400004018E4A00238B4208BF824228BF45F0FD
:103F50001005F4EEC97AF1EE10FAB4EEE99A48BF12
:103F600045F02005F1EE10FAC8BF45F040059FED81
:103F7000858A0A9505F00C030C2B8DED0D8A8DEDCD
:103F80000E8A8DED0F8A8DED108A8DED118A8DEDE3
:103F9000128A8DED138A8DED148A8DED158A00F04D
:103FA0000B81D4EDDC7AD4EDE36A94EDCB8A94ED09
:103FB000937AD4F87C33C4F8943377EEE67A00230E
:103FC00094F89561C4EDE47A28EE078A84F8883382
:103FD000022E00F04181092E07D1DFED6E7A68EEE6
:103FE000277AFDEEE77AC4ED6B7A15F040071DD015
:103FF000DDED097AD4EDC65A94EDDF6A94EDDC7AF2
:1040000067EEA76AA6EE277A66EEA56AB6EE005AB4
:1040100067EEA57A66EE856A68EE085AA6EE887A9B
:10402000A7EEA56A84EDDC7A84EDDF6AAA0600F1CA
:1040300083816B0700F1C081534B1B68DA0602D401
:1040400094F8583213B1AB0700F14A831F2E00F0E9
:1040500071834FF00008E80700F12A8105F0580548
:10406000582D09D1DFED497A94EDB57AB4EEE77AAF
:10407000F1EE10FA80F2BE8294EDDD3AD4EDDE3A34
:104080009DED0D4AD4EDDA2A94EDDB2A9DED0E5A12
:104090009FED3C7AD4ED917A9DED096A77EE436A03
:1040A00037EE637A66EEA76A27EE277A66EE866AAF
:1040B00067EE067ACDED106ACDED117AB8F1000FFA
:1040C00009D09DED0B6A94ED947AB4EEC76AF1EED7
:1040D00010FA40F3BE8194EDDF6A9FED2A7AD4EDA9
:1040E000904ADDED095A37EE467A27EE247A27EE1C
:1040F000257A8DED127AD4EDDC5ADDED0F1AD4ED70
:10410000924A36EE077A34EE224A32EE055A76EEBD
:10411000836A77EEA37A35EEA16AF5EEC04AF1EE36
:1041200010FA84EDDA4A84EDDB5AC4EDDD6AC4EDA1
:10413000DE7A84EDDF7A84EDDC6A2FDDDDED147A42
:10414000DDED136A9DED157A9FED116A67EEA77A92
:10415000E6EEA67AE7EE077AF4EEC67AF1EE10FA0A
:1041600000F11E831AE000BF50570020BD3786358E
:10417000843F01204028002060E31600400D03002A
:10418000801A060000000000603D0120C3F5A83E33
:104190007DCA6A4700007A446F12833A0C990B9AE1
:1041A0000A9BC4F88013C4F88423C4F8603216B0A4
:1041B000BDEC068BBDE8F08D94F88833012B00F040
:1041C000FF81022B00F06C81002B00F0478194ED01
:1041D000E40A94EDE57A94F8956194EDCB8AD4EDF8
:1041E000937A092E28EE278A07D15FED167A68EEBA
:1041F000277AFDEEE77AC4ED6B7AD4EDC66A68EEF5
:10420000A87AA8EE870A022B67EEA67AB6EE006AB5
:1042100068EEA68A67EE867A68EE086AA7EE880AD4
:10422000A8EEA67AF0EE407A84EDE40A84EDE57A11
:1042300000F07B83012B00F0E283D4EDDC7A94ED77
:10424000E37AD4F87C33C4F8943377EEC77A022E3D
:10425000C4EDE47A7FF4BFAED4EDB57A1FED336AD6
:10426000D4EDE46A94EDE57A94F88833C4F89C318F
:1042700067EE867AFDEEE66AFDEEE77ABDEEC77A76
:10428000C4ED686AC4ED667A84ED697AADE6D4ED72
:10429000947A1FED3F7AC4F8600277EE877AC4ED16
:1042A000E07AC4EDE17A16B0BDEC068BBDE8F08D86
:1042B000A90600F10F81D4EDDA2A94ED9D4A94ED20
:1042C000DB2A94ED9E5A94EDDD3AD4EDA05AD4ED5C
:1042D000DE3A94EDA16ADDED0D1ADDED0E4ADDED5D
:1042E000106A9DED117AD4EDA37A34EE624A35EE70
:1042F000425A75EEC35A36EE636A34EE214A35EE01
:10430000245A76EEA56A37EE067A8DED0D4A8DEDCC
:104310000E5ACDED106A8DED117ACDED0C7A94ED3B
:10432000947AB4EEE77AF1EE10FA3FF5B1AEDDED36
:10433000117ADDED106AC1E6DDED098AD4EDDA9A75
:1043400094EDDB9AD4EDDDAA94EDDEAAEAEEA89A0C
:10435000A8EE8A9AC4EDDA9A84EDDB9AFFF736FD6F
:1043600000283FF466AE68EEA87A94EDC47A94ED26
:10437000C55A67EE276A67EE857AF6EE005A28EE90
:10438000877A28EE086A68EE858A66EEA56A67EE87
:10439000A57AE7EE06AA6B07A6EE28AAE6EE889AAB
:1043A000A7EE889AC4EDDDAA84EDDEAAC4EDDA9A00
:1043B00084EDDB9A7FF540AE42F072FBD84B1B6870
:1043C0005D0700F15A82D74BD4EDDC5A94EDAC8AEC
:1043D0000A9DC4EDEA5AC3184FF0000241EB0202F5
:1043E000C4E9E832012184F8AC130026D4ED877AC1
:1043F0009DED096A9DED127ADDED0F6A38EE658A52
:1044000067EEA75A28EE275A65EE885AE5EE066A47
:10441000A907A6EE257ACDED0F6A8DED127A00F18F
:10442000CB82D4EDE16A94EDAD7A37EE667A27EE71
:10443000277AE7EE066ACDED0B6A002E7FF40BAE0D
:104440009DED157A67EEA77AA8EE677A8DED157A5D
:1044500001E694EDDF6A9DED127A4CE694EDB57AB3
:10446000F6EE087AB4EEE77AF1EE10FAFFF6AFAEA8
:10447000AD48022684F888634BF086FEB4EEE99AD4
:10448000F1EE10FA40F32082D4EDDC7AD4EDB46A78
:1044900094EDDF7A77EEE67A3346C4EDE37A9AE676
:1044A000D4EDB57AB6EE087AF4EEC77AF1EE10FAEA
:1044B000BFF68DAE9FED9D7AF4EEC77AF1EE10FA5D
:1044C000C0F29080012394EDE40A94EDE57A84F83B
:1044D000883380E694EDDB2A94ED9E8AD4EDDA2AC7
:1044E000D4ED9D8A94EDDD3AD4EDA09AD4EDDE3A78
:1044F00094EDA19A38EE428A78EEE28A28EE080A14
:1045000079EEC39AA8EEA80A39EE639AB5EE400A8E
:10451000F1EE10FAB1EEC0AA00F1148394ED8C5ABA
:1045200094EDA37ADDED096AD4EDE07A9DED116A90
:10453000DDED104AD4ED8D1A9DED0D4A9DED131A57
:1045400065EE055AB4EEC7AA68EEA50AF1EE10FAB8
:1045500068EE255A58BFB0EE4A7AA6EEA56A37EE45
:10456000677AE6EEA04A27EE057A68EE858A28EE9D
:10457000058A69EEA19A29EE219A9DED0E5ADDED8C
:10458000141AE6EE877AB0EE467AA8EEA64AA6EEB0
:10459000885AE6EEA94AA6EE897A71EEE55A71EEDE
:1045A000606ACDED0C7A8DED0D4A8DED0E5ACDED94
:1045B000104ACDED136A8DED117ACDED145AAEE6A9
:1045C000D4EDB57AB6EE087AF4EEC77AF1EE10FAC9
:1045D00080F28A819FED557AF4EEC77AF1EE10FAF7
:1045E000BFF6F5AD002394EDE40A94EDE57A84F886
:1045F0008833F0E5D4EDC15A94EDC06A94EDBF7AEA
:10460000D4EDBE7AD4EDB46AD4F87C33089337EE97
:10461000657A77EEC67A27EE667A67EEA67A06A8FE
:104620008DED067ACDED077A2BF0F2F99DED066A55
:1046300094EDDD3ADDED075AD4EDDE3AD4ED8F6A24
:104640009DED098A0A9B36EE437A75EEE37A27EEF2
:10465000267A67EEA67A27EE087A67EE887ADA0776
:104660008DED107ACDED117A00F1428194F8193276
:10467000002B40F02B82DDED0C7A9DED0D4AD4ED40
:10468000DA2A94EDDB2A9DED0E5A94F89531042B2D
:104690007FF445AE94EDBE6ADFED254AD4EDBF1A36
:1046A000D4EDE66A94EDE77AC6EE245A81EEA46A68
:1046B000FDEEE55ABDEEC66AFDEEE66ABDEEC77ACE
:1046C000C4ED665A84ED676AC4ED686A84ED697A60
:1046D00025E64B074FF000057FF512ACFFF7FFBB57
:1046E000002F40F0838094ED9F6A94EDDC5AD4ED66
:1046F000A26AD4EDDF5A9DED0F7ADDED127AD4F87F
:1047000090320B9336EE456A76EEE56A37EE067A1E
:1047100077EEA67A8DED0F7ACDED127A9BE400BF8D
:10472000583D012090D00300105A0020C3F5A83E48
:1047300035FA8E3CD4EDDC6A94EDAC7AD4ED9F7AF8
:10474000FDEEE66ABDEEC77AFDEEE77AC4ED666A75
:1047500084ED687AC4ED6A7A1CF096FA94F8953183
:10476000BDEEC00A1F2B84ED6C0A15D1D4EDDF6AB3
:1047700094EDC67AD4EDA27AFDEEE66ABDEEC77A74
:10478000FDEEE77AC4ED676A84ED697AC4ED6B7A71
:104790001CF074FAC4F8B4010A9D4FF000085AE402
:1047A00013A82BF0EDF8D4ED927ADDED134A9DEDD0
:1047B000145A9DED154ADDED095A94EDC76AD4ED02
:1047C000C86A94EDC97A67EEA44A27EE855A67EE67
:1047D000847AA4EEA56AE5EE856AA5EEA77A84ED53
:1047E000C76AC4EDC86A84EDC97AD7E4D4EDDC5A4F
:1047F000D4ED9F7A94ED8A4A94EDA47AD4EDE14AFF
:104800009DED095ADDED126A94EDA26A94EDDF2A5E
:104810009DED0F3AD4ED8B2ADDED153A77EEE57A72
:1048200064EE045AF4EEC77AF1EE10FA65EEA75A78
:1048300058BFB0EE677A37EE647AE5EE256A27EE68
:10484000047A36EE426A67EE847AE5EE074A26EE8F
:10485000226AB0EE437AA7EE857AF0EE667AE5EE4C
:10486000067A73EEE55ACDED0B4A8DED0F7ACDED5C
:10487000127ACDED155AFFF7EEBB94EDDF7AF2EE2A
:104880000E7AB4EEE77AF1EE10FA23DCBB4B00228D
:10489000C31841EB0202C4E9E8320A9D2B0730D568
:1048A00094EDB47AF3EE047AB4EEE77AF1EE10FA0E
:1048B00027D594F8AC33002B00F09C8094EDEA8A65
:1048C000D4EDDC5A012691E5B0EE487A84EDE38A16
:1048D000334680E4D4E9E8238B4208BF8242DCD22D
:1048E000002384F8AC33D8E7022384F888336EE4DD
:1048F000D4F87422D4F87832C4F89823C4F89C33DE
:10490000B9E6680776D594F8AC33002B72D0D4EDB5
:10491000AC7A94EDEA8AF4EEC87AF1EE10FACFD4CC
:10492000D4EDDC5AB0EE678A5FE594EDB48ADFED32
:10493000940A38EE408AB0EE480A4AF0DDF9B7EE44
:10494000002ADFED901ADFED900AB0EE421A4AF02D
:10495000EFFE94ED887AD4ED897A94EDB55ADDEDC9
:10496000094AD4EDE45A94EDE56A94F8883368EE88
:10497000076A68EE277A20EE008A26EE807A67EED4
:10498000887A65EE056A27EE057A67EEA67AE7EE85
:10499000245A022BA4EEA76AC4EDE45A84EDE56A1A
:1049A00076D094EDCB8AD4ED937A0A9D94F89561F4
:1049B00028EE278AFFF70CBBD4EDDF7AD4EDA28A6C
:1049C000DFED720A78EEE78AB0EE680A4AF094F9F1
:1049D000D4ED8B6A9DED127A9DED096AD4ED877A4C
:1049E0000A9D68EEA68A68EE808AA8EE867A8DED2A
:1049F000127A16E5D4EDDC5A94EDAC8AF5E494ED28
:104A0000B49A94EDE37AD4EDDC8ADFED610A39EEF5
:104A1000409A78EEC78AB0EE490A78EEE78A4AF003
:104A20006BF9B7EE002ADFED571ADFED570AB0EE4B
:104A3000421A4AF07DFED4EDB57A94ED886A94ED81
:104A4000895ADDED095AD4EDE46A94EDE57A94EDE6
:104A5000CB8AD4ED934A0A9D94F8956120EE270AFB
:104A6000F7EE007A77EEC07A28EE248A67EEA87A0D
:104A7000E9EE007A27EE866A67EE857AE6EE256A29
:104A8000A5EEA77AC4EDE46A84EDE57AFFF7A0BA53
:104A900094EDE17AD4ED947AB4EEE77AF1EE10FA7F
:104AA0007FF57FAF3B48D4EDDC8A4BF06DFB94ED96
:104AB000CB8AD4ED937A0A9D94F8956138EEC00ABA
:104AC00028EE278A84EDE30AFFF782BA94EDE77AAD
:104AD000D4EDE66A94EDDB2AD4EDDA2AD4ED8E4AE1
:104AE00094EDE09AA5EE887AE6EE086AF0EE475A71
:104AF00037EE427A36EEE26A27EE070A26EE244ABD
:104B0000A6EE060A27EE247A24EE084A27EE085A73
:104B1000B5EE400AF1EE10FAF1EEC08AC4EDE75AA4
:104B2000C4EDE66A8DED0D4A8DED0E5A15D438EEC2
:104B3000C97AF0EE497A27EE247AE8EE077ACDEDCD
:104B40000C7AA2E552F0AEF8D4EDDA2AD4EDDE3AD2
:104B500094EDDD3A94EDDB2AE0E452F0A3F8D4EDD5
:104B60008E4A9DED0D4AD4EDDA2AD4EDDE3A94ED6D
:104B7000DD3A94EDDB2A9DED0E5AD8E790D0030084
:104B800000009642CDCCCC3D0000000000007A43EE
:104B900000004842105A00200B4B93F81532012BAD
:104BA0000AD0022B06D1094B186880F00400C0F32C
:104BB0008000704700207047044B1B6813F00C0FF7
:104BC0000CBF01200020704750570020583D0120A5
:104BD0002DE9F04F2DED028B91B041F061FFAE4C0D
:104BE000AE4B67691A680F97D4E9033C1206CDE90A
:104BF0000D3C49D5AA4AD2F800E01EF0020F4DD074
:104C0000A84F0E46D7E9EC210546B5EB020866EB46
:104C10000109A5480021494508BF4045DFF89082B9
:104C20003CBF012288F8B8201EF0010F06D097F88B
:104C300014221AB197F8B823002A60D0DFF8A092A6
:104C400099F85433002B36D0FFF7A6FF78BB97486E
:104C500000220DA9F6F796FE98F8B830002B00F068
:104C60004181D4E90412E068C7F8B0530023C7E9D2
:104C7000EF01C7F8B463C7F8C42388F8B83011B09F
:104C8000BDEC028BBDE8F08F864B00200021C3E90C
:104C90009A0111B0BDEC028BBDE8F08F844B01226C
:104CA00083F8B82011B0BDEC028BBDE8F08F0F9BEC
:104CB000C9F86433CBE70D9BC9F85C33002BB8BF50
:104CC0005B4207EE903ADFED7B6A9FED7B7A0E9AAE
:104CD000F8EEE77A012387EEA60A89F854330F9B92
:104CE000C9E9D82320EE070A4AF042FEDFED730A35
:104CF000B7EE001A4AF03CFD89EDD60AA7E707EEA9
:104D0000903ADFED6C6ADFED6E5AF8EEE77A87EEE7
:104D1000A67AB4EEE57AF1EE10FA00F11C82DFED2E
:104D2000697AB4EEE77AF1EE10FA00F3148207EE36
:104D300090CAF8EEE77A9FED645A87EEA66AB4EE61
:104D4000C56AF1EE10FA00F10682DFED607AB4EE8A
:104D5000E76AF1EE10FA00F3FE81B2EE045AC7EEF4
:104D6000056AC6EE057AFDEEE66AFDEEE77AF8EE34
:104D7000E66AF8EEE77A66EE856A67EE857A9FED79
:104D8000515AB4EEE57AF1EE10FAB4EEC57A8CBF62
:104D9000FDEEE65ADFED4E5AF1EE10FA05DBF2EECB
:104DA000045A76EEE56AFDEEE65ADFED476AB4EEA8
:104DB000E66ADFED466AF1EE10FAB4EEE66A8CBF01
:104DC000BDEEE75A9FED435AF1EE10FA05DBF2EE25
:104DD000046A77EEE67ABDEEE75AF8EEE56A9FEDF3
:104DE000394ADFED3A4A3C4936EE844AF8EEC55A74
:104DF000B2EE045AC4EE057A75EEA44A36EE656A40
:104E000084EE854AC6EE055AFCEEE77A37EE667AFE
:104E100017EE903AFCEEC47A03F1010C03EBC302E7
:104E200003EB82030CEBCC020CEB820C87EE056AE1
:104E300017EE902A501C03EB020E034462446044B8
:104E400001EB8E0E01EB830301EB800001EB82028C
:104E50009EED008AD2ED007AD3ED006A90ED007AE3
:104E600076EEC86A37EE677AA5EEA68AE5EE877A0F
:104E700077EEC87AA6EE278AB0EE480A2AF020FE1E
:104E8000B2EE040A28EE008A144A012382ED0D8A4C
:104E900087F8B833D2E600BF88170020843F01208E
:104EA000603D01205057002060E31600C4590020E7
:104EB000080A00208096184B35FA8E3C0AD7233C0E
:104EC0000000B4C20000B442000034C30000344308
:104ED000A6FFFFFF4CFFFFFF6CA30608943F0120D5
:104EE00040280020D7E9EC01CA4B281A66EB0101E3
:104EF0004FF0FF3210EB030A41EB020B00234CF2A0
:104F000050325B4508BF524580F06B81C24B4FF079
:104F1000FF32C318009341EB02030193DDE9009ACD
:104F2000002349F64042534508BF4A4580F05C8162
:104F3000BA4B4FF0FF32C318029341EB02030393C5
:104F4000DDE9029A002344F62062534508BF4A4532
:104F500080F04D81B24B4FF0FF32C318049341EB08
:104F600002030593DDE9049A002342F210725345CF
:104F700008BF4A4580F03E81AA4B4FF0FF32C3186C
:104F8000069341EB02030793DDE9069A002341F201
:104F90007072534508BF4A4580F02F81A24B4FF0F5
:104FA000FF32C318089341EB02030993DDE908239C
:104FB0004FF0000A4FF47A699A4508BF914580F096
:104FC0001F81DFF8ACC24FF0FF3E10EB0C030A93D9
:104FD00041EB0E030B93DDE90A239A4508BF914587
:104FE00080F011814EF0A2FDDFED907A07EE100AFD
:104FF00027EE278AD4F80C90DFED8D6A9FED8D7A2D
:1050000089EAE973A3EBE97307EE903AF8EEE77AE1
:1050100087EEA60A20EE070A4AF0AAFCDFED860A10
:10502000B7EE001A4AF0A4FB97F8180200284FD0F8
:10503000A378002B4CD0B4F91E3007EE103AB4F927
:10504000203007EE903AB8EEC77AF8EEE77A87EDAF
:10505000A07AC7EDA17AE378002B69D0B4F92230A9
:105060005B4207EE903AF8EEE77AD7E9F22352EA8C
:105070000301C7EDA27A78D1704BC7F8C853A3F5E6
:10508000AE7207CAA3F5A87C83E807009CE8070076
:105090000C3383E8070097F87022C7F8CC6300232D
:1050A00087F8712287F870326379002B56D0238DF0
:1050B00007EE103A638D07EE903AB8EE477AF8EEB5
:1050C000677A87EDA37AC7EDA47AC7E99A56C8E54F
:1050D000D7F8BC132369D7F8C023DFED596AD7EDA1
:1050E000A05A97EDA16AA9EB01019B1A07EE901A4D
:1050F00007EE103A20EE260AF8EEE77AB8EEC77A05
:1051000067EEA67A27EE007AC7EE886AC7EE087ABD
:1051100036EEA57A77EE867AF6EE006A27EE267AE4
:1051200067EEA67A87EDA07AC7EDA17A002892D122
:105130006369D7F8C42397EDA26A9B1A07EE903AE9
:10514000B8EEE77AF6EE006AC7EE087A77EE867A6E
:1051500067EEA67A89E79FED3B8A8DE63A4A3B4B9C
:10516000C7F88C22C7F89032AFE7A81A66EB0301A4
:105170004EF0DCFC9FED2D8AD7EDF56A97EDF86ACD
:1051800097EDF47AD7EDF77A05EE900A25EE888A46
:10519000B0EE660AA8EE060AB0EE476AA8EE276AE5
:1051A00030EE660A76EE477A20EE000AA7EEA70AEE
:1051B000B5EE400AF1EE10FAF1EEC08A26D49FED6A
:1051C000247ADFED247A28EE077AE8EE077AF4EE07
:1051D000E78AF1EE10FA7FF64FAF0123A7F870329D
:1051E00062E7B5EE008A05E79FED1B8A02E79FEDB7
:1051F0001B8AFFE69FED1A8AFCE69FED1A8AF9E604
:105200009FED198AF6E69FED198AF3E651F04AFD03
:10521000D5E700BF1891FCFFE040FDFF70A0FEFF46
:105220003850FFFFD08AFFFF28A6FFFFBD37863525
:105230008096184B35FA8E3C0AD7233C205B002021
:105240002C7D8E3F00000000000048430000FA4320
:105250000000FA4300007A43CDCC4C3ECDCCCC3D8F
:10526000CDCC4C3D2F88083DCDCCCC3C0AD7A33CBF
:10527000B0B9FFFF08B52DED048B9FED178AF0EE56
:10528000418AB0EE619AF0EE429AF0EE481AB0EE22
:10529000601AB7EE002AF0EE480AB0EEC00A4AF0F3
:1052A00047FAF0EE480AB7EE001A4AF061FAB0EE9B
:1052B000691AF0EE490AB0EE682AF0EE481A4AF090
:1052C00037FAB0EE681AF0EE480ABDEC048BBDE880
:1052D00008404AF04DBA00BF00000000054A08B57A
:1052E000136843F08003136029F074F8024BD880F0
:1052F00008BD00BF603D01207C3F012038B5002083
:105300002BF0B2F948B10D4CB4F8625029F062F8B4
:1053100085420BDD0124204638BD044629F05AF8A9
:10532000FFF7DCFF064B5C72204638BD044B94F857
:1053300072205A720224204638BD00BFB8380020BF
:10534000943F012070B5334C2DED028B94EDFA8A19
:10535000B5EE408AF1EE10FA08EE900A0D460DD136
:10536000D4F8EC339FED2C2AB3F80A3108EE103A4A
:10537000B8EEC88A28EE028A84EDFA8A274B93F8A1
:10538000773003EB830303EB8303002A4FEA8301A7
:10539000284614BF042600264AF002FAF8EEE88AEE
:1053A00000EE900A9FED1E1A9FED1E0A1E4828EE81
:1053B000811AF8EEE00A3146B0EE482AF1EE481ABA
:1053C0004AF0AAFC94F895319FED137A112BC0EEA8
:1053D000077A1AD1154BC4F8A451D3EDB55A93ED01
:1053E000B46AD3EDB66A93EDB87AFDEEE55ABDEE38
:1053F000C66AFDEEE66ABDEEC77AC4ED665A84ED74
:10540000676AC4ED686A84ED6A7ABDEC028BB0EE1F
:10541000670A70BD505700200000C842B83800200D
:10542000BD37863500000000DC2A0020402800201F
:1054300010B5154BD3F8EC3393F8E630012B15D0AB
:10544000022B0AD1114BB3F9043013F1FA0F10DA21
:105450000F4B012483F8B94000E0012428202AF0F2
:10546000B9FF08B1644264B2204610BD4FF0FF346A
:10547000F4E7FA2B064BC9BFFF2293F9B94083F832
:10548000B9204FF0FF34E9E7505700207C3F01205E
:10549000080A002038B50F4D0F4C00232846C4F8E9
:1054A000F033C4F8F433C4F8F8334AF029FC05F1BA
:1054B00048004AF025FC002304F58060A5F83C373D
:1054C000A5F8403784F8FC3384F8FD33BDE8384054
:1054D000F5F714BB942A0020505700202DE9F8431B
:1054E000124D2B6813F010041CD1DFF84880104FC8
:1054F00008F1EC00B9464AF003FC002608F59A7062
:1055000049F8046F3E60A8F890494AF0F9FB2B680F
:10551000C9F8006023F46053A8F892493E602B60FC
:10552000BDE8F883BDE8F843B4E700BF603D012063
:10553000605B00204028002008B50C4B93F89521B3
:105540000A2A04BF0322C3F89821094B1A7B1AB90F
:10555000FFF7C4FF022008BD0649D3F81C230968E1
:10556000C3F8C413C3F8BC23002008BD5057002063
:1055700040280020A8220020154B1B68DA0620D501
:1055800010B5144B144A00EB800003EBC00092F8F6
:105590009531C4890A2B04BF0123C2F898310F4BFF
:1055A000DB7A13B1FBF7AEFE80B9A3070BD50C4B2A
:1055B000D3F81C230021C3E9EF22C3F8C41302204F
:1055C00010BD03207047FFF789FFF0E7042010BDEE
:1055D000603D0120609C060850570020B83800202C
:1055E0004028002008B52DED028B35F0A1FCB5EE6A
:1055F000400AF1EE10FA04D1BDEC028B9FED0B0ACC
:1056000008BD0B4BB0EE408A93ED000A51F0AEF8A6
:105610009FED080A07EE900A28EE008AF8EE677AF6
:1056200087EE880ABDEC028B08BD00BF00000000B9
:10563000D83100200000C84208B5094B094A1B7840
:1056400003EB830302EBC30344F21900DB89184028
:1056500000D108BD25F06EF8003818BF012008BD44
:1056600040280020609C06080A4B987C88B11B7873
:10567000094A03EB830102EBC102D08910F40270E6
:1056800007D00D2B04D0192B0CBF0220012070472E
:105690000220704740280020609C0608064A517C82
:1056A00002F5417302F53B72002908BF134603EB74
:1056B000800393ED030A70474028002070B5AC4E7C
:1056C000AC4C96F84130AC4D07EE903A2DED048B82
:1056D000F8EE677A9FEDA98A96F842309FEDA89A76
:1056E00087EE887A00EE103AB8EE400AF0EE490AEA
:1056F000B7EE001A80EE080A84EDB97A4AF038F85D
:10570000D5F8EC3384EDBA0AB3F87A3000EE103AEB
:10571000B8EE400A04F1140080EE080AF5F7F2F939
:10572000D5F8EC33B3F8882004F1EC0001EE902AB0
:10573000B3F8862093ED3A2A01EE102AB3F88420BC
:1057400000EE902AB3F8822000EE102AF8EE611ADB
:10575000B8EE411AF8EE600AB8EE400AF3EE048A99
:10576000C1EE881A81EE081AC0EE880A80EE280A77
:105770004AF08EFAD5F8EC33B3F87A3004F15C00D5
:1057800000EE103AB8EE400A80EE080AF5F7BAF9D2
:10579000D5F8EC33B3F8882004F59A7001EE902A1E
:1057A000B3F8862093ED3A2A01EE102AB3F884204C
:1057B00000EE902AB3F8822000EE102AF8EE611A6B
:1057C000B8EE411AF8EE600AB8EE400AC1EE881A47
:1057D00081EE081AC0EE880A80EE280A4AF058FACC
:1057E000D5F8EC3396F8382004F1A40007EE902A9F
:1057F00093F8EC2006EE102A93F8ED2006EE902A9E
:1058000093F8EE20B3F8723007EE102AF8EE677ABC
:10581000B8EEC66AF8EEE66AB8EEC77AC6EE085A7F
:1058200086EE886AC7EE086A87EE887A00EE103A3C
:10583000B8EE400A534B80EE080AC3ED0E5A83EDD2
:105840000F6AC3ED106A83ED117AF5F75BF9D5F8AD
:10585000EC339FED4D0AB3F8A42000EE902AB3F884
:10586000A620B3F8A23001EE102A07EE903AF8EE27
:10587000600AF8EE677AB8EE411A87EE800A04F5FE
:10588000BE70C0EEA80A81EE081AF0EE491AB2EE18
:10589000042A4AF0FDF904F5E270B0EE000AF5F7CB
:1058A00031F9D5F8EC33DA8C01EE102A9A8C5B8C46
:1058B00000EE902A00EE103AB8EE411AF8EE600AB7
:1058C000B8EE400A81EE081A04F51570C0EE880A99
:1058D00080EE080AF0EE491AB2EE042A4AF0D8F92E
:1058E000D5F8EC33DA8B01EE102A9A8B5B8B00EE45
:1058F000902A00EE103AB8EE411AF8EE600AB8EEBF
:10590000400AF2EE048A81EE281A04F50370C0EE14
:10591000A80A80EE280AB0EE682AF0EE491A4AF08A
:10592000B7F9D5F8EC33B3F8562001EE102AB3F8E6
:105930005420B3F8523000EE902A00EE103AB8EE40
:10594000411AF8EE600AB8EE400A81EE081A04F532
:105950002770C0EEA80A80EE280AF0EE491ABDECC6
:10596000048BB0EE002ABDE870404AF091B900BF48
:10597000B838002040280020505700200000C842BE
:1059800000000000943F012066668542094B0A4AE8
:105990001B7803EB830302EBC303D889830607D488
:1059A00010F0400005D0054B1868C0F30010704798
:1059B0000120704740280020609C0608603D0120BF
:1059C0001149124A0B7803EB830302EBC303D88916
:1059D000430513D591F969399BB191F97C29013BB4
:1059E0009A420ED002EB420201EBC20191F8DE03B3
:1059F000A0F1A500B0FA80F040097047C0F3400064
:105A000070470120704700BF40280020609C0608B6
:105A1000044B1B6813F0040304BF034AA2F868395F
:105A2000704700BF583D01204028002070B50C464B
:105A300000230421A522C4E90133C4E9033384B05F
:105A40002170A275A38260B92A4B1B68DB0706D5BB
:105A5000294BD3E900129B68E360C4E9011204B04A
:105A600070BDFF281ED0FE2831D0431EDAB23B2A7B
:105A7000F5D8224D95F969299042F0DC03EB4303F8
:105A800005EBC30505F572750FCD26460FC695E8E3
:105A9000030086E803002378062BE0D1238A013334
:105AA0002382DCE7154B597C03F5417203F53B7308
:105AB000002914BF1146194601A8F5F71FFFDDE9BB
:105AC0000112039BE360C4E9011204B070BD0B49ED
:105AD00091F85433002BC2D00B78094A03EB8303AF
:105AE00002EBC303DB8903F00303032BB7D101F5FA
:105AF0004C71E1E7603D01208C3D002040280020F2
:105B0000609C06080D4B1B685B0770B512D40C4BEC
:105B100093F8686966B10B4D01242946E0B201345F
:105B2000FFF784FF3D2C05F11805F6D139F076F822
:105B3000304670BD0026304670BD00BF583D012084
:105B400040280020685B0020F8B5294C2DED028B21
:105B50000746B0EE408A40F0A3FF657C04F5417330
:105B600004F53B72002D08BF1346D3ED028A0546AB
:105B70000E463FB9C4EDCE8ABDEC028B1D4BC3E986
:105B80000001F8BD1C4B1B68DB060DD4D4ED2A7A4E
:105B9000184FC8EE270A70EEA80AC4EDCE0ABDEC75
:105BA000028BC7E90056F8BD124FD7E90001281A49
:105BB00066EB01014DF0BAFFDFED107A9FED107A30
:105BC00006EE900A66EEA77AF4EEC77AF1EE10FAC6
:105BD000E5D894EDCE0ADFED0B0AA8EE270A38EEE1
:105BE000A01A78EEE00A49F0C3FD84EDCE0AD6E7AC
:105BF0004028002008610020603D0120BD37863527
:105C0000CDCC4C3E0000FA4308B50C4B1B689B0200
:105C100003D423F0EFFF002008BD094B9FED090AD4
:105C20001B8B07EE903AF8EEE77A012027EE800A08
:105C3000FFF78AFF23F0DEFF002008BD603D012052
:105C4000B83800209A9999BE024B93ED000A50F0A3
:105C50008DBD00BFD831002008B5134BD0ED000A30
:105C6000597C90ED010A03F5417203F53B7300295D
:105C700018BF134693ED007AD3ED017A70EEC70A90
:105C800030EE670A49F006FEDFED087A9FED087AEC
:105C900020EE270ABDE80840C0EE077AFDEEE77A5D
:105CA00017EE900A49F08CBD402800200000C84241
:105CB00035FA8E3C01072DE9F84F08D54D4B0022EF
:105CC0001A609A804C4AB2F8C029DA808FE010F04E
:105CD000020F804600F08B80474C1F46D4F8D8391D
:105CE000C4F8D829D31A1546444AC4F8DC7993423B
:105CF00006DDC4F8E059C4F8E479FFF7CBFB54E0C3
:105D00003F4E337A002B4ED0B378002B47D0D4F8D7
:105D1000E039C4F8E479A5EB03093A4BC4F8E0593B
:105D2000994538DC06F54C70FFF796FFD6F81C3322
:105D3000C01A49F051FDD4F8E839D4F8EC29B5EB94
:105D4000030A67EB020B00232F4A5B4508BF52454D
:105D500014D2D4F8F439C4F8E859002B80EAE07280
:105D6000B8BF5B42A2EBE0729342D4BF0023012391
:105D700084F8F039C4F8F409C4F8EC79014694F8D1
:105D8000F0294846FFF7DEFABDEEC00A10EE103AE1
:105D9000A6F8943901E0FFF77DFB0123737101231D
:105DA00084F8F83901E084F8F839124D002318F42A
:105DB000004F2B600AD0AB80144B1B68DB044CBF38
:105DC000B4F9003AB4F9063AEB8010E094F8F839E7
:105DD0001BB10B4BB3F89439AB800D4BB4F8042ACC
:105DE000B4F8061AB3F8480049F0D2FCE880BDE8E0
:105DF000F88F00BF7C3F012050570020400D03006A
:105E0000402800203F0D03001FA10700643D012032
:105E1000B838002070B51446D20705460E4603D5A3
:105E20001A4B1B681B0517D5A0071ED4610703D5A5
:105E3000174BC3F8486370BD220720D4E306FAD598
:105E40002846FFF709FFA0F58C40503849F0B8FC10
:105E50000F4BC3F8480370BD0D4B01684268C3F88F
:105E60003423A007C3F83013E0D59FED0A0A0020C1
:105E7000FFF76AFE064BAA68C3F83823D6E7284620
:105E8000FFF7EAFE024BC3F8480370BD603D0120F6
:105E9000402800200000000010B5094C607CD4F8B8
:105EA0001C1304F53B7304F54172002814BF10461F
:105EB00018460222FFF7AEFF00232374E37310BDE0
:105EC00040280020074B1B7C53B100B583B00190E4
:105ED000FFF7E2FF019803B05DF804EBFFF72CBB7E
:105EE000FFF72ABB4028002008B5034B1B7C0BB1F1
:105EF000FFF7D2FF002008BD4028002038B5034638
:105F000007C8084D05F66C1484E807001846FFF72B
:105F1000A3FE0146C5F8781920460722BDE838409F
:105F200078E700BF40280020F0B50C46D4E90223F2
:105F300089B049680393CDE90112054670B9424B17
:105F40001B68590708D5414B1A7A2AB193F8542394
:105F500012B1DB7B002B6BD109B0F0BDFF282ED135
:105F60002578012DF8D1384B1B685A07F4D5374BEB
:105F70001A7A022AF0D193F85423002AECD0DA7B63
:105F8000002AE9D01B78052BE6D12A4601A904A8EE
:105F9000F5F7F8FCB4F91010E2684B1E002A9BB22A
:105FA00018BF0325B3F5B37F98BF45F004056423FC
:105FB0002A4604A801FB03F1FFF72CFFCCE7461E9D
:105FC000F3B23B2BC8D8204B1B685B07C4D42378A3
:105FD000012B02D0033B052BBED8DFF870E09EF901
:105FE000693901339D4201D0012DB5D1A446BCE8E9
:105FF0000F0006EB46060EEBC60606F572770FC7D6
:106000009CE8030087E803002378062B04D1B6F848
:10601000D833013BA6F8D8338EF86959A37DA3F194
:10602000A503B3FA83F35B098EF8683909B0F0BDB4
:1060300001A904A80122F5F7A5FC072304A8294615
:106040001A46FCF70DFD87E7583D01204028002047
:10605000F8B5114E336813F004031BD10F4F104CE9
:10606000A7F86839012501E03D2D0AD02146E8B2A4
:10607000FFF75AFFA37DA52B05F1010504F11804D4
:10608000F2D197F8680920B933685B0701D4A7F803
:106090006809F8BD0020F8BD583D012040280020C7
:1060A000685B002008B5164B90ED010A597CD0EDD5
:1060B000007A03F5417203F53B73002918BF1346BC
:1060C000D3ED016A93ED007A30EE660A77EEC77A77
:1060D00020EE000A2DED028BA7EEA70AB5EE400ACE
:1060E000F1EE10FAB1EEC08A06D4FCEEC87ABDEC2F
:1060F000028B17EE900A08BD50F0D4FDF5E700BF03
:1061000040280020F0B5044687B008202AF062F944
:1061100000284DD0FCF7F6FA01260CB100232370BD
:106120005C4D6B7813B9002007B0F0BD5A4A92F865
:10613000201A002957D0594A127A3AB3584A12689D
:10614000D10723D5574B1B6803F00403034301D148
:10615000002E6CD1514C94F969190029E3DDEB89CB
:10616000002B4DD0D4E9F321D4F8D4330392049119
:10617000012203A968460593F5F704FC6846FFF77A
:1061800091FFEB89984237D90320CDE7022B27D125
:10619000434A1268520406D418461CF0A3FD40F28C
:1061A000D66398421CDD002CBDD001232370BAE7D2
:1061B00013202AF00FF90028ACD109202AF00AF99F
:1061C00098BB374B1E6816F0100632D1FCF79AFACE
:1061D0000028A2D003202AF0FDF8C0B301209CE7DC
:1061E000012007B0F0BD92F8C7190229A3D092F898
:1061F000D229022AA6D19EE794F96919002992DDD5
:106200000023184618260FB200EB400204EBC2022E
:106210005D1C92F8C823062A04D0EBB28B421846C4
:10622000F2DB80E7BBB904207EE70126CEE702203F
:106230007AE703202AF0CEF80028F6D123202AF0AE
:10624000C9F80646FCF75EFA00283FF466AF232043
:106250002AF0C0F861E706FB0043421EB3F9D833C9
:106260009A4202DC421C9342DDDDBB42DBDA06FBD4
:106270000040B0F9DA230132D5DB9BB206FB0343C1
:1062800093F8C83303F0FD02012AC6D0082BC4D00E
:10629000C9E700BFB8380020505700204028002030
:1062A000603D0120583D012070B5184C184AE38C20
:1062B00016682BB1174DD5F86833F31A642B01D843
:1062C000012070BD05F56070FFF7ECFE07EE900A47
:1062D00095EDDE7AF8EE677AB4EEE77AF1EE10FA31
:1062E00010DCE38C77EEC77A07EE103AB8EEC77A87
:1062F000F4EEC77AF1EE10FAD4BF01200020C5F801
:10630000686370BDC5EDDE7A0120F8E7B83800207B
:10631000A82200204028002070B5FFF7C5FF2C4DB3
:1063200048B92B7A3BB92B4EF37A2BB1FAF7EAFF37
:1063300010B10A2070BD274E274B748CA3F11C02AC
:1063400007CA83E807008CB3728A687C95EDE27A0D
:1063500007EE904A00EE102AF8EEE77AA3F19802D1
:10636000A3F1B001002808BF0A46D2ED026A77EE19
:10637000877AB8EEC00A37EEE67AB7EE006AB0EE7A
:10638000C77AC7EE005AC5EDE97AF4EEC65AF1EEC7
:1063900010FA16D4F4EEE76AF1EE10FA58BFB1EE37
:1063A000400A0120FFF7D0FB002070BDD5F89463B0
:1063B000C5F8A463184602222146FFF72BFD2046AC
:1063C00070BD184602220021FFF724FD002070BD99
:1063D00040280020B8380020DC2B00209CE700BFBC
:1063E00070B52D4DEB7A03B32C4C2068820222D578
:1063F0002B7A33B92A4BDB7A1BB1FAF783FFA0B9AA
:10640000206810F0100418D1D5F81C33D5F88C038F
:10641000C01A49F0E1F90028B8BF404240F2DB530E
:10642000984235DDFFF740FF00BB0A2070BD1D4BD1
:106430001B689B0518D5022070BDFBF721FE0020CC
:106440009FED190AFFF780FB95F97C3903EB4303B5
:1064500005EBC30595F8C833082BECD0104BDB795E
:10646000012BE8D0022BE2D0082070BD0F4BD5F8ED
:106470009463A3F11C0207CA83E807001846D5F805
:106480008C13C5F8A4630722FFF7C4FC204670BD37
:10649000FBF7F6FD2046D3E740280020603D0120B1
:1064A000B83800205C3D012000000000DC2B0020FB
:1064B00007C838B5094C0A4D04F55B7383E807003B
:1064C0002B68C4F8683304F56070FFF7EBFD07EE46
:1064D000900AF8EE677AC4EDDE7A38BD40280020D5
:1064E000A82200202DE9F041734C0120FCF74AFA64
:1064F000E37A002B00F09D80704E3368990240F1E2
:10650000C680237A6E4F33B9FB7A23B1FAF7FAFECD
:10651000002840F08A80D4EDE46AD4EDE27A9FED61
:10652000696A9FED697A76EEE77AF0EEE77A67EED0
:10653000867AF4EEC77AF1EE10FA51D4F1EE677A6A
:10654000624D627CA5F11803002A18BF2B4693ED1B
:10655000027A37EE667AB4EEE77AF1EE10FA42DCB0
:106560003B79002B3FD00020FCF70CFA00283AD1F1
:1065700005F17C0393E807003368D4EDE47A98359D
:10658000DB0685E80700C4EDE97A61D53B799FED2C
:106590004E7A022B40F084807A8A4C4B617C77EEF5
:1065A000877A00EE102AA3F11802C4EDE97A0029D7
:1065B00008BF134693ED027AF4EEC77AF1EE10FAB3
:1065C000BFEE007AB8EEC00AF7EE007AD8BFF0EE60
:1065D000477A20EE270A0120FFF7B6FA002621E0CD
:1065E000DFED3B7AACE73368DA0626D4394BD4EDDD
:1065F000EA7A7D79D4F89073A3F11C0207CAF8EE09
:10660000677A83E80700C4EDE67AC4F8A4731DB185
:10661000316811F0100134D02E480B220021FFF711
:10662000F9FB02263046BDE8F0813B7A002B7FF46F
:1066300072AF0A263046BDE8F081244B607CA3F19E
:106640001802002814BF18461046FFF731FFCDE7A7
:10665000FFF72AFE0028ECD03168D4EDE97A11F07A
:10666000100893D19FED187A7E7977EE877A2846C5
:10667000C4EDE97A7EB112224146FFF7CBFB4646D4
:10668000D0E718461322FFF7C5FB0226CAE7022609
:106690003046BDE8F0810A223146FFF7BBFBC1E777
:1066A00077EE877A00210B48C4EDE97A02220E4684
:1066B000FFF7B0FBB6E700BF40280020603D012097
:1066C000B83800209A99193E0000C842442B002097
:1066D0000000C8C2DC2B002010B50C46FFF7E2FC1E
:1066E0001C4B1D4A1B6807EE900AF8EE677A13F000
:1066F000100FC2ED007A194B0CD05CB19A8907EEED
:10670000102AB8EEC77AF4EEC77AF1EE10FA0ED876
:10671000204610BD9B8907EE103AB8EEC77AF4EE1A
:10672000C77AF1EE10FA94BF0120002010BDB3F833
:106730005830DFED0B6A07EE103AB8EEC77A27EE55
:10674000267AF4EEC77AF1EE10FA94BF0120002009
:1067500010BD00BF603D0120C8310020B8380020C6
:10676000CDCC8C3F30B52DED028B4F4B1A7A85B0D6
:1067700092B1DA7A82B193F97C2902EB420203EBFF
:10678000C20393F8C833013B072B10D8DFE803F0AE
:106790000F0F0F230F0F0F0F444BDB7A13B1FAF7D4
:1067A000B1FD98B9002005B0BDEC028B30BD404C66
:1067B00000212046FFF790FF18B9F5F771FE054656
:1067C00080B3022005B0BDEC028B30BD0A2005B0BD
:1067D000BDEC028B30BD36480121FFF77DFF00285C
:1067E000EFD1F5F75DFE0028EBD1304B5B7923B19B
:1067F000304B196811F0100149D02D4809220021B1
:10680000FFF708FB2C4CA4F11C0393E8070084E875
:106810000700FBF75BFC204602220021FFF7FAFA93
:106820000020C0E794ED068A236894ED070A0193DF
:10683000F2EE047AC8EE278A63680293B0EE481A33
:10684000F0EE680A48F094FF94ED022AD4ED051AA0
:10685000B0EE681AF0EE480A48F06AFF0B222946AB
:1068600001A88DED030AFFF7D5FA124B1B685B03F5
:1068700098D5124890F8243A012B0DD0022B91D1D3
:10688000D0F8281A04222846FFF7C4FA8AE70848F5
:106890001122FFF7BFFAB5E7294600F62C2008229F
:1068A000FFF7B8FA7EE700BF40280020B838002084
:1068B000AC310020603D0120DC2B0020505700202F
:1068C00070B51A4D0120FCF75DF8EB7AE3B12C7A34
:1068D0003CB9174BDB7A13B1FAF714FDA0B9204687
:1068E00070BD05F5607393E8070005F5677686E8E7
:1068F0000700FBF7EBFB30460121FFF7EDFE0446F6
:1069000058B9FFF7D1FC10B90A24204670BD3046B3
:1069100003222146FFF77EFAE1E7D5F88C133046D3
:106920000722FFF777FA0224D9E700BF40280020AA
:10693000B838002030B56C4C94F97C3903EB430136
:1069400004EBC10187B091F8C81301395A00072937
:1069500005D8DFE801F004040427485E74041344FA
:1069600004EBC303D3E9F3216846D3F8D43303928D
:106970000491012203A90593F5F704F86846FFF78F
:10698000BDFA5A48FFF78EFB07EE900A584BD4F831
:10699000F42243F8042CF8EE677A0220C3ED007A63
:1069A00007B030BD534DD4EDEA7A607CF8EE677ADB
:1069B000A5F11803002814BF28461846C4EDE67A4E
:1069C000FFF776FD05F17C0393E80700983585E82D
:1069D0000700D4F89033C4F8A4332846FFF78EFAA2
:1069E000022007B030BD44490968480347D41A441F
:1069F00004EBC20292F8DE23A52A3DD094F969295E
:106A0000013A9A4238DD0133002084F87C3907B01E
:106A100030BDD11804EBC101B1F9DC03451C04D031
:106A200000284FD00138A1F8DC03134404EBC30362
:106A30000020B3F8D83384F87C3907B030BD2E4934
:106A4000096849030CD5D11804EBC101B1F9D81379
:106A500088B2B0F5B47F29D32849002081F8240AF0
:106A60001A4404EBC20292F8DE23A52A04D094F95A
:106A70006929013A9342C6DB0D2007B030BD1344AB
:106A800004EBC303D3E9F3211C4DD3F8D4330392B1
:106A9000CDE90413012205F62C2003A985F8242A48
:106AA000F4F770FF94F97C395A00A0E701EB8101FB
:106AB000124801EB810189000225C0F8281A80F8EC
:106AC000245ACDE791F8DE23B1F8DA53A1F8DC536C
:106AD000A52AD1D094F96929013A9342CCDA01333D
:106AE00084F87C395CE700BF40280020AC310020EE
:106AF000C4310020442B0020603D0120505700206D
:106B00002DE9F047854F864AFB7AD2F800A02DED9B
:106B1000048B814682B023B1FAF7F4FB002840F0E1
:106B2000F780804E96F895510A2D05D10222002358
:106B3000C6F89821C6F8A0317B4C237B002B40F08F
:106B4000E18094F80E80D4F8C433B8F1000F31D14D
:106B5000AAEB030ABAF57A6F03D9D4F8BC33C4F8A8
:106B6000C033724BA9F11D00B3F92420C0B2C2EBAF
:106B7000021205284FEA82027DD82D2323FA00F065
:106B8000C30775D5D4F8BC136948FBF7A9FF0A2DD4
:106B900009BF0123D4F8BC13D4F8BC13C6F8A03144
:106BA00063480122FFF736F9002002B0BDEC048BE8
:106BB000BDE8F087AAEB0303642B98BF07EE903A79
:106BC0005C4B97F87410B3F904309FED5B1ADFED5E
:106BD0005B0A88BF9FED5A8A00EE103A01EB8103F1
:106BE00003EB83036FF063024FEA830302EE103A74
:106BF00002FB01F301EE903AB8EEC22AF8EEE11A78
:106C0000B8EEC00A98BFB8EEE78A48F091FDDFED14
:106C10004D6AD4EDEF7A20EE080AF8EEE77A80EEBE
:106C2000267A77EEC77AFDEEE77A17EE900A48F0FB
:106C3000C7FD0A2DC4F8BC0307D1434B83FB0023D7
:106C4000C017C0EB6310C6F89C01384BC4F8C4A34E
:106C5000B3F92420A9F11D00C0B2C2EB021205282D
:106C60004FEA82028ED82D2323FA00F0C30789D47D
:106C7000B8F1000F86D12E480192FFF713FAB7F84A
:106C80005830DFED326A019AD4F8BC1307EE903A1F
:106C900007EE100AF8EEE77AB8EE477A67EEA67AC2
:106CA000B4EEE77AF1EE10FA3FF67AAF06EE901AFC
:106CB0009FED277ADFED277A0191F8EEE66A06EE7E
:106CC000102AC6EE878AB8EEC68A68EEA78A94EDC7
:106CD000EC9AB0EE680A48F04BFEA8EE009AB0EECF
:106CE000680A84EDEC9A48F0BDFED4EDED8A019976
:106CF000E8EE008A0A2D04BF0223C6F8A031C4EDD5
:106D0000ED8A4DE7122002B0BDEC048BBDE8F087A0
:106D1000042002B0BDEC048BBDE8F087B838002039
:106D2000A82200205057002040280020881700206B
:106D3000F02B00207C3F01200000FA430000FAC342
:106D40000000000000007A441F85EB51CDCC8C3F41
:106D50000000C84235FA8E3C064B1B7C4BB100B597
:106D600083B00190FFF798F8019803B05DF804EB49
:106D7000C6E6C5E640280020054B587C03F5417265
:106D800003F53B73002814BF10461846704700BF38
:106D90004028002008B50146FFF7EEFF0A4B90EDB2
:106DA000036A93EDB97AD0ED007AD0ED046AE6EE8D
:106DB000077AC1ED007AFFF7DFFFD0ED017AE7EE49
:106DC000267AC1ED017A08BD4028002038B5FFF7CA
:106DD000D3FF0A4C0546204648F092FF04F14800D4
:106DE00048F08EFF6A69C4F8C8210023A4F81A3855
:106DF0000348BDE83840F3F781BE00BFBC2900203E
:106E0000886100200C4B1B6810B50C4CDB066074CD
:106E10000ED504F5037048F073FF094A02F64C21C1
:106E200000230020086082F8483AA4F8923910BD87
:106E3000BDE81040CAE700BF603D012040280020A7
:106E40005057002008B50020FFF7DCFF022008BDE6
:106E500008B50020FFF7D6FF074B0848D3F81C33CE
:106E600080FB0320DB17C3EB601000B222F0A2F816
:106E7000FEF734FB002008BD402800201F85EB51A1
:106E8000F0B52DED028B83B008EE100A27F0A2FAC0
:106E9000234B244FDB8D244EB7F8045A96EDD10ACC
:106EA000C01AED1A04B2FFF767FFB8EEC81ADFED9B
:106EB0001F7AD0ED050A2DB221EE271A07EE905A5F
:106EC000B8EEE72A07EE904A06F5BE70F8EEE71A2C
:106ED00000218DED011A48F01FFFBDEEC00A9DEDA7
:106EE000011A10EE103A1BB207EE903A07F638205E
:106EF000B8EEE70AF1EE000AA6F8963944F0ECFF86
:106F0000BDEEC00A2A4610EE103A214618B248F0EB
:106F10003FFCA6F8960903B0BDEC028BF0BD00BFA4
:106F2000B83800205057002040280020BD37863553
:106F300010B52DED028B08EE100AFFF71DFF2C4C4B
:106F400090ED027A94EDCE0AD4ED2A7A637B30EE8E
:106F5000470A20EE270A002B44D0264BDB8A5A42F0
:106F600007EE903A00EE902AB8EE671AF8EEE00AC3
:106F700048F0FEFBDFED206A9FED207AD4EDD10AC8
:106F800084ED3A0AF8EEC87A67EEA67A70EE606A87
:106F900027EE877AB1EE476AB4EEE66AF1EE10FAB0
:106FA00023DAB4EEE67AF1EE10FA0ED984EDD10AC6
:106FB0004FF0DCFB124947F6FF7248F0E9FBBDECED
:106FC000028B104BA3F8540A10BD9FED0F7AB0EE60
:106FD000601AA7EE871AE7EEC70A48F0C9FB84EDEE
:106FE000D10AE5E7034B5B8AB9E79FED087AEEE744
:106FF00040280020B8380020BD3786350C22C44216
:107000005A80FFFF505700208F2AF5430C2244443A
:107010002DE9F04FB84EB94C96F8FC13B4F84E80F9
:10702000B4F848A0B4F8509085B0054617460093D0
:10703000B9B1A80723D496F8483A0BB1EA0742D46D
:1070400005F4804ABAF1000F08D0AD4BDA79002A76
:1070500040F0E2809A7A022A00F00E8105B0BDE885
:10706000F08F96F8FD33002BE5D08107E3D5A44BD4
:10707000DFF8A8B2B3F89439ABF80430DBE794F842
:1070800044109F4B019301EB81026FF0090000FB5C
:1070900001F15200B3F99009DFF880B248F078FBB3
:1070A00003B2D6F8EC2300EE103AB2F9C800B8EEFD
:1070B000C00A22F06DFD96F8FD23019BABF800009D
:1070C000002AB8D0D6E794F845208D4B94F84610A6
:1070D000B3F9920903936FF0090C02EB82020CFBE7
:1070E00001F1520048F054FB01B207EE901AD6F8B5
:1070F000EC230291B8EEE70AB2F9CA008DED010A5D
:1071000022F046FDB4F85420D6F858CADFED7D6A67
:10711000DFED7D0A9FED7D1ADFF800B29DED010ADB
:10712000C6F8587AC2F10A0292B2A7EB0C0302FB2E
:1071300002FC02FB0CF207EE103A07EE902ADFF891
:10714000E4C1009BCCF80430B8EEC77AF8EEE77AD9
:107150004242E7EEA60A0CF10800ABF8022027EE47
:10716000011A44F0B9FEBDEEC00A029994F8560027
:1071700010EE103A0FFA83FCA1EB0C02002AB8BF04
:1071800052428242039B624A94F8520040F390803C
:1071900082FB01C2C917C1EBA20110FB01F108B2C9
:1071A000A9EB0A09A8EB0A010FFA89F915F4804A3C
:1071B00009B214BF00224A460293019148F0E8FA4E
:1071C00044F202021540022DDDE9011300B279D02C
:1071D000B4F84870B4F85020B4F84E10384448F071
:1071E000D7FA94F8752085B2002A53D0494B1B6812
:1071F0009B054FD4BBF9063040F29D72934274DC7C
:10720000DA1B002AA8BFAD18ADB29F42ACBF002365
:10721000012386F8783A40E00093FFF7ADFD638BD9
:1072200090ED027A07EE903AF8EEE77A009BB4EE22
:10723000E77AF1EE10FA3FF60DAF27F0CBF894F9AC
:107240005A30354A354C116803EB83035B0000EE7E
:10725000103A0546D6F8EC03E58041F08001B0F91C
:10726000CA001160B8EEC00A0025258022F090FC0B
:10727000608005B0BDE8F08F628B93EDC37A07EEB6
:10728000902AF8EEE77AB4EEE77AF1EE10FA3FF6DC
:10729000E5AED2E7002386F8783A27F09BF8B6F8F7
:1072A000042A0146284648F073FAABF80600C9E6FE
:1072B00082FB0C124FEAEC71C1EBA20110FB01F052
:1072C00000B26DE71A7A9AB19A786ABB144BD3ED83
:1072D000007AFDEEE77A17EE903A9AB2104400B2C7
:1072E0004A4648F055FA00B272E7B6F8045A8CE7FD
:1072F0000B4B00251D60F1E750570020B8380020E7
:10730000402800206F12033B0AD7233CBD37863547
:10731000676666665C3D0120603D01207C3F012080
:107320009C610020A8610020D6F870CADFF8B0E0A8
:10733000254AC6F8707AA7EB0C07009D5560774583
:1073400028DCD3EDCB6ADFED217A9FED216A36EEA2
:10735000E77AB0EEC77AB4EEC67AF1EE10FA1EDC28
:1073600012ED090AA2F124059FED1A1ADFED1A0A9F
:107370000090CDE9011348F0FBF9FDEEC07ADDE99C
:10738000000117EE903A9AB2029B85ED000A0125A2
:107390005D71A3E7002542F8245C0022F7E737EE91
:1073A000E67A07EE907ADFED0D6A12ED090AF8EE43
:1073B000E77AB7EE086A27EE067A67EEA67AA2F1B8
:1073C0002405A7EE270ACFE7C061002000002F4464
:1073D000000048420000FA4300000000BD37863537
:1073E0003F0D0300F8B5314B186810F010001DD1A7
:1073F00029F03AF92E4B1B780446C3B900283ED039
:107400002C4B2D4CB3F90650A4F8BA5026F0E2FFED
:107410002A4A92F87F3AB2F8042AC118D21A2846AA
:107420000A310A3A48F0B4F9A4F8BA00F8BD234D7D
:10743000214EB5F97A7AA6F8BA7026F0CBFF95F806
:107440007F3AB5F8042AC118D21A38460A310A3AE6
:1074500048F09EF9A6F8BA00002CE7D1FFF78CFCA3
:10746000D0ED027A9FED167AF0EEE77AF4EEC77A65
:10747000F1EE10FA9CBF012385F8863AF8BD0F4D56
:107480000D4CB5F97A6AA4F8BA6026F0A3FF95F816
:107490007F3AB5F8042AC118D21A30460A310A3A9E
:1074A00048F076F9A4F8BA00D8E700BF603D0120A3
:1074B000B83800207C3F0120080A002050570020E7
:1074C0000000484238B5164C94F9693913B194F864
:1074D00068390BB9032038BDFEF700F80020FFF72C
:1074E00091FCFFF77FFF94F96909002812DD002362
:1074F0001A4602EB420204EBC201013391F8C823A1
:10750000062A04BFB1F8DA53A1F8DC53DBB2834298
:107510001A46EEDB002384F87C39022038BD00BF18
:1075200040280020254B264A2DE9F04100EB800041
:107530001D68244C02EBC00015F01005677CC6895D
:1075400027D0002316F001002374E3731BD180467B
:10755000FFF758FC40F201233340012B01D17305A2
:1075600014D5FFF73FFF184B607CD4F81C13A3F130
:107570001802002814BF184610460222FEF74AFCE3
:107580000220BDE8F081B7B11846E0E74745E8D1F1
:10759000F6E7182028F01EFFF20780462574E573F1
:1075A00003D4182028F016FFD2E78742D2D0182043
:1075B00028F010FFCCE7B846CCE700BF603D0120C3
:1075C000609C060840280020442B0020074B1B68C5
:1075D000DB0608D510B50446FFF7A4FF2046BDE83A
:1075E0001040FDF7C9BF0320704700BF603D012078
:1075F000064B1B68DB0607D510B50446FFF7BCFB3E
:1076000007C884E8070010BDFFF7C4BB603D012038
:107610002DE9F0413F4CE37A86B0002B3BD0E37973
:10762000002B38D0257A022D35D13B4E3368DA074E
:1076300031D5DF06DFF8F48005D5D4F8A823B8F8F3
:1076400024309A4251D3354B00EB800003EBC0004D
:10765000C789B90757D5FA0722D5637C03BBB8F8A9
:107660002420D4F8A8339A422AD92D48D4F81C13E0
:1076700007230522FBF7F4F92A4B607CD4F81C138E
:10768000A3F11802002814BF184610460722FEF77F
:10769000C1FB0C2500E00A25284606B0BDE8F081B4
:1076A0000020FFF7AFFBFFF79DFEB8F82430D4F8B9
:1076B000A8239A4204D2637C002BD6D01948D5E780
:1076C0003368DB0616D598F8043003A8022B019026
:1076D0001CD0154AD4F81C13FBF702FA0198D4F811
:1076E0001C130522FEF796FBD6E7A37C002BAAD13C
:1076F0000425D1E703A80190FFF77AFF0198FEF770
:10770000D7FE0198EBE7FDF7E9FEA4E7FFF770FF6E
:107710000198E4E740280020603D0120609C0608B5
:107720002C2B0020442B0020A0860100B83800201C
:1077300010B5124C237C84B013B9002004B010BDE6
:1077400001A8FFF755FF607CD4F81C1304F53B73C8
:1077500004F54172002814BF104618460222FEF7B5
:1077600059FB01A8D4F81C130522FEF753FB002394
:1077700000202374E37304B010BD00BF4028002034
:107780002DE9F0432D4BDFF8C0902D4DD9F80020A6
:107790006F7C00EB800103EBC10385B0DE89D3066B
:1077A000044634D54FF000080023B0072B74EB7368
:1077B0002AD5F10701D5474508D0D9F80030DA06B7
:1077C00037D50020FFF71EFBFFF70CFE40F2012328
:1077D0003340012B13D01B4B687CD5F81C13A3F14D
:1077E0001802002814BF184610460222FEF712FBAA
:1077F000093C022C10D8022005B0BDE8F0837305C7
:10780000E9D44745E7D1F3E7FDF768FED1E7182053
:1078100028F0E0FD8046C7E701A8FFF7E9FE01A8D0
:10782000D5F81C130522FEF7F5FA022005B0BDE8D5
:10783000F083182028F0CEFDC4E700BF609C060846
:1078400040280020442B0020603D01202DE9F84F06
:10785000794B1B68990240F1AF80784A1268520751
:1078600040F1AA80DB0653D53FF01AF9FEF71CFD64
:10787000002800F0AD80DFF8E4C19CF80A30022B4C
:1078800000F0A9806E4B6F4C9CF81150A3F11C02C4
:1078900007CA83E80700608BDCEDE96AA28BA3F1DD
:1078A0009801B03B002D18BF0B4693ED027A07EE0E
:1078B000900A37EE667AF8EEE77A121A37EE677AB0
:1078C00007EE902AF8EEE77AF5EE000A87EE276ACF
:1078D000F6EE086AB0EE600AA6EE260AB7EE001AC7
:1078E00047F046FF238B9FED587A07EE903AF8EE6B
:1078F000E77A20EE670AB4EEC70AF1EE10FA58BF35
:10790000B0EE470A0120FEF71FF90020BDE8F88F0E
:10791000DFF84C813FF0C4F8D8E946AB5AEA0B03D4
:1079200081464CD0FFF728FAB9EB0A06474ADFF840
:107930002CC1D0ED057A9CEDCB7A61EB0B070023CF
:10794000BB4208BFB2423CD2D8F82421B8F9886AB9
:10795000D8F820310132334493FBF2F028388642C4
:10796000C8E948322DDAF0EEE77AF3EE096AF4EE70
:10797000E67AF1EE10FA24DCDFED357AB4EEE77A40
:10798000F1EE10FA1DDC9CF80A30022B41D02D4A92
:10799000D8F81031168ED8F814014FF47A72B9EB7A
:1079A000030402FB06F24FEAE27361EB0005AB420F
:1079B00008BFA242BFF45AAF0220BDE8F88FC8E961
:1079C0004601C8E94491FEF76FFC00287FF453AFED
:1079D0000A20BDE8F88FDFED1F7A9CEDC37AB4EE84
:1079E000E77AF1EE10FA7FF54DAF164B9FED1A7A5C
:1079F0001B8B00EE103AB8EEC00AFBEE0E7A20EEBA
:107A0000070AB4EEE70AF1EE10FA58BFB0EE670AC3
:107A100078E7DCEDC36AF5EEC06AF1EE10FAB6DB8A
:107A2000DCEDCA7AB1EE047A77EE877AF4EEE76A93
:107A3000F1EE10FAABD9C4E7603D0120583D0120BA
:107A4000DC2B0020B8380020000048C240420F0064
:107A50000000C842000048429A9919BE4028002000
:107A60005057002010B5FFF7F1FE022802D0002485
:107A7000204610BD064B1B689B02044603D5054BF0
:107A80009B79002BF4D0072036F00AFD204610BD6C
:107A9000603D0120B838002038B52E4C84EDC31A63
:107AA00084EDBD0AC4EDC00AC4EDC61A38BB2A4B2A
:107AB000E0711B68A0725B07E07002D4274BC4F82A
:107AC0002833274B607C274C2749A3F11802002854
:107AD00008BF1346D3ED027A93ED057AFDEEE77AFF
:107AE000BDEEC77A17EE903A17EE100A47F6FF720E
:107AF000C4F8943A47F04CFEA4F89C0A38BD0D46F1
:107B0000F9F71CFC144B194A1B681068A572012276
:107B10000221E2705A07C4F85003E171CED5022D5C
:107B2000CFD1B5EEC01AF1EE10FACADDD4EDCA7AA3
:107B3000F5EEC07AF1EE10FA09DDF4EEC17AF1EE5D
:107B400010FA58BFF0EE417AC4EDCA7AB9E784ED75
:107B5000CA1AB6E740280020583D0120000080BF27
:107B6000442B0020505700205A80FFFFA8220020FD
:107B70002DE9F047674D684C2B78684A03EB830783
:107B800004EBC7071668B96881461A464FEA830CAA
:107B9000B9B3FF7CAFB3DFF88881D8F8A00A301AF8
:107BA00081422ED8BB4206D007EB87022F7014F813
:107BB00032206A703A4602EB820004EBC00091006A
:107BC000D0F804A0BAF1000F00F0A1801846D04709
:107BD0002B78002800F0918003EB830204EBC202B3
:107BE00011181A468F7C990007EB8700002F00F0D0
:107BF0008680BB42DFD014F830206A702F703A467E
:107C0000D9E76146B9F1000F39D0881804EBC000FC
:107C1000814499F8120090B3984207D000EB80019C
:107C2000024614F83110697028708100881804EB3E
:107C3000C0004768D7B91FE02B7803EB830204EB41
:107C4000C20210449900807C1A46A8B1834206D033
:107C500000EB8001024614F831102870697002EBC5
:107C6000820004EBC000910047682FB11846B84766
:107C70000028E1D12A789100294BC3F8A06A29484D
:107C8000294B0068002647071E7007D5881804EBAB
:107C9000C000C089860526D5022018700A4404EB6E
:107CA000C2042A7B217B607B597000219870D970B7
:107CB0000AB10122DA706A7B1AB1DA7842F0020264
:107CC000DA7095F97C29D1B24C1C00203B291C713B
:107CD000587106D802EB420205EBC20595F8C8239D
:107CE0005A71BDE8F087470504D406070AD50F206E
:107CF0001870D3E703201870D0E71A469900C8F827
:107D0000A06A7FE7800744BF01201870C6E73B46A2
:107D1000F5E700BF40280020609C0608A82200204C
:107D200050570020583D0120CC3D002038B5074A6F
:107D3000074B0020002400250121C3E900451872EB
:107D40009174FAF7EDFCBDE8384011E740280020B7
:107D5000943F01202DE9F04FBA4F2DED028B3B6887
:107D600013F004088FB040F0DB80B74C227A002A71
:107D700049D1DFF80083B54DD8F80030C5F8103B85
:107D8000E37B1620002B40F0C28028F023FBE07339
:107D9000FAF7C6FCFFF7ECFE2378AD4F03EB830345
:107DA00007EBC303DE89300504D5AA4B1B68990590
:107DB00040F129810023637316F4805300F08A8018
:107DC000A44B1B689A0540F10A81A34A1368D9069F
:107DD00040F133810023A373237803EB830307EB84
:107DE000C30741F6B8003E8A20EA060028F070FA80
:107DF000304628F07DFA6378A5F8203B0FB0BDEC43
:107E0000028BBDE8F08F914D94F87C2395F8161203
:107E100002F00302033A18BF012201294CD00229C3
:107E20004FD18E4B8E4EB3F82A90FF22002309F1DA
:107E3000010985F8A42A0D93A246337801220BA9E3
:107E400005A89BB1D6E90143CDE90B43F3F79AFDB1
:107E500005A8FEF727F9484508D2059B069A08931E
:107E6000079B85F8A48A814609920A9308F10108C4
:107E7000B8F1080F06F10C06DFD195F9A43A9AF88B
:107E80000B20002B54469AF8083080F29680002B85
:107E90004FF00000DAF81C13C5F8080B18BF0323D5
:107EA0000AB143F0040307226E48FAF7D9FD3A6895
:107EB000217A02F0040248E083F00803C3F3C00310
:107EC0001A43002AADD1DFF8AC81D8F80030C5F8EC
:107ED000103B58E02373B2047FF57CAF5D4B1B6809
:107EE0009B053FF577AF5C4B5F4A1B6813F01003AF
:107EF00000F0AB81B2F9042095F87E3A002AB8BFB1
:107F0000524292B293422CBF0023012363E728F030
:107F100061FA00287FF43BAF01231620237434E775
:107F2000152028F057FA494D00283DD10123464C31
:107F3000DFF8249185F80C3BD9F80030DB0700F11D
:107F40009B803A68217A02F00402DFF82881D5F894
:107F5000100BD8F80030C5F8103B8AB11B1A07EE99
:107F6000903A9FED426A424BD4EDCB6A93ED007A92
:107F7000F8EEE77A67EE867AA6EEA77A83ED007AC6
:107F800000293FF4FDAE344B1B68DE077FF5F8AEE9
:107F900095F8143B002B7FF4F3AE0E201FF058FF32
:107FA000012385F8143BEBE695F80C3B002B40F0E1
:107FB000A980254CDFF8A090BEE7002BC5F8089BF0
:107FC00018BF03230AB143F004030722002108A8C5
:107FD000FAF746FD3A68217A02F00402B5E7DFF8C5
:107FE0007890D9F80020D30640F1AE801E4B95F86A
:107FF0007E1AB3F9000047F0D3FB00B2011E18BF90
:108000000121217367E7144B1B6813F0100A48D055
:10801000154B95F87F9AB3F90200494647F0C0FB2B
:1080200000B2002840F06F8194F80D90B9F1000F74
:1080300040F0618184F80D90BEE623F46053136034
:10804000C8E600BF583D01204028002050570020BE
:10805000609C06085C3D0120603D0120B83800208E
:10806000F86100202C2B00207C3F01206F12833A06
:10807000D8310020A8220020D04EA6F11C0393E89E
:10808000070086E807003046FEF70CF80346304646
:10809000C4F8A833FDF7E0FDC4F8AC03FAF7C0FC60
:1080A0004FE794F81190B9F1000F40F0F380C44A03
:1080B000C44BB2F9BA90B3F9060095F87FAAA0EBC9
:1080C0000900514647F06CFB00B20028ACD040F3E9
:1080D0009381BD4AB5F8043AD28AA3EB090900FBA3
:1080E00002F0A9EB0A0907EE900A07EE109AF8EEE3
:1080F000E77AB8EEC77A87EE870A01208146FDF756
:1081000023FD97E7B14BB24C1E6816F4216640F090
:10811000AD80237ADFF8CC92002B3FF40DAFD9F875
:108120000020E37AD4F81C1312F0010F14BF0522CB
:108130000722002B0CBF0323072304F53B70FAF73B
:108140008FFC85F80C6BF7E6DFF878A295F87E1ABD
:10815000BAF902000292019147F022FB019983468D
:10816000BAF9000047F01CFB9A4B029A59780FFAB3
:108170008BFB03B203934BEA030AB9B1032915D071
:1081800022F46052C9F80020BAF1000F7BD1217BA4
:1081900000293FF436AF0BA8FEF7FCFD00210BA829
:1081A0000122FDF737FE0021217394E6242001927D
:1081B00028F010F9019A00285BD090045BD4824B20
:1081C00094EDCB7A588E07EE900AF8EEE77AB4EE8B
:1081D000E77AF1EE10FA06DDBAF1000F03D19978D3
:1081E000012900F03081D30411D5774994EDCB7A81
:1081F000CB8F07EE903AF8EEE77AB4EEE77AF1EE3D
:1082000010FA00F2F18022F48052C9F80020100523
:10821000BAD56D4994EDCB7A8B8E07EE903AF8EE95
:10822000E77AB4EEE77AF1EE10FA03D9BAF1000F6B
:1082300000F0F98022F4C052C9F80020FEF79CFD3E
:1082400001220021FDF7E6FD9EE7B2F9042095F832
:108250007E1A002AB8BF524292B29142BFF4BBAD1F
:10826000D4F81C33C4F848330123B4E5DFF8749123
:1082700062E69104B7D5BAF1000FB4D022F40052EF
:10828000C9F80020AFE7504B9978012954D001215B
:10829000217320E64B4BB3F906B026F09BF8A37A86
:1082A0000190022B21D1484BB5F8042A1B8DDFED3C
:1082B0004A1A07EE900A01EE102A02EE103AF8EE82
:1082C000E70A07EE90BAB8EE422AB8EEE70AB8EE2F
:1082D000411A47F02DFAF2EE047AB4EEE70AF1EE15
:1082E00010FAB0EE408A00F3A6809FED3C0A012010
:1082F000FDF72AFC9EE69FED380A0020FDF724FCDE
:108300004FF0000996E6304B9FED350ADB8A07EE09
:10831000909A404203FB00F0F8EEE77A07EE100A6D
:1083200030EE670AB8EEC77A012087EE000AFDF743
:108330000BFC4FF001097DE69A8A039895F87E3A86
:10834000D4EDC85AD4EDC94A02FB00FA07EE90AA50
:10835000C3F5FA73F8EEE76A07EE903AB8EEE77AFB
:1083600002FB0BF2C6EE877A06EE902AF8EEE66A7A
:1083700025EEE76A86EE875A67EEA47AF0EE466A43
:10838000E5EE246AE5EE257AFEF7F6FCD4ED065A12
:1083900090ED006A86EEA57A37EE067A84EDCC7A07
:1083A000FEF7EAFC94ED186AD0ED016A217387EEBE
:1083B000867A77EE267AC4EDCD7A8CE5DC2B002028
:1083C000080A00207C3F0120B83800205C3D0120D5
:1083D00040280020CC3D002000000000000048C2E2
:1083E0000000FA43603D0120D8F80010D5F8180BC2
:1083F0008842BFF40CAF06E72A4BDB8A00FB03F090
:1084000007EE900AB8EEE78A25F0E4FF95F87F3A88
:10841000A9EB0000A0EB030907EE909AF8EEE77ACB
:1084200088EE270A69E6D8F80010D5F81C0B8842B8
:10843000BFF4ADAEFEE69FED1C0A5046FDF784FB8F
:1084400084EDCE8AF6E500283FF4CDAEFEF794FC2D
:108450000A465146FDF7DEFC124B94EDCB7A9A8F1B
:10846000D9F80000D8F800C0D98E07EE902AF8EEAF
:10847000E77A40F42052B4EEE77A6144F1EE10FA64
:10848000C9F80020C5F81C1B7FF7ADAE598FD8F88E
:10849000003040F460521944C9F80020C5F8181B98
:1084A000A1E600BFB838002000000000C0F343037D
:1084B000C0F382025A4000F01F0353405B0130B406
:1084C00003F0200300F01F0444EA0301CA0882EA13
:1084D000910282EA1112920102F0400211430D0949
:1084E00085EA91050B46694043EAC113DBB2984225
:1084F0000CBF20464FF0FF3030BC7047054A0123C7
:10850000D2F8242B03FA00F0104214BF18460020C2
:10851000704700BF505700202DE9F84FCB4DD5F8DC
:10852000282B002A63D005F5336806460F46D8E9A4
:10853000000150EA01035CD195F8393B95F8384BBE
:10854000DFF80CC39C4288BF0A331B1BDBB2002B35
:1085500000F08A809CF9BC104B1C00F023819CF930
:10856000BD00431C0BD0D5F8243BC0B2012404FA53
:1085700000F023EA0003C5F8243B481C7CD0C1F37B
:108580004604C1F385036340CCB25C40640104F04F
:1085900020040C43C4F3C400C4F385034340C4F374
:1085A000031043409B0103F040031C43C4F38503C5
:1085B000C4F303105840E3B2434044EAC314FF231A
:1085C000E4B28CF8BC3013688CF8BD1010461B6800
:1085D0007E219847D5F8280B036821461B689847E9
:1085E000002385F8953BC5F8306BC8F80470BDE8EA
:1085F000F88F301A42F6E06398429DDC95F8953B7F
:108600000BB985F8963B924CDFF84C8213E080F072
:1086100020000023C0B285F8963B95F8951B4B1CB3
:10862000DBB229440A2B85F8953B81F8980B00F0C2
:108630008F80D5F8282B136810465B689847002870
:10864000D5D0D5F8280B0368DB68984794F9BD208E
:10865000511CEED095F8963B002BD8D17D28DCD16B
:10866000012385F8963BE4E79CF9BD009CF9BC101A
:10867000441C7FF478AF80E7D5F8240B00284DD058
:10868000D5F890EBBEF1000F0BD173464FF0010906
:1086900009FA03F401331C2B4EEA040EF8D1C5F895
:1086A00090EB3EEA000300EA0E0B00F0F3809CF82A
:1086B000BE30002B00F0F180012B94D195F88C3B5B
:1086C000DFF890919C08A9FB04E4C4EBC404A3EB7D
:1086D0008404E4B24FF0010E0EFA04FB1BEA000F13
:1086E00003F11C0A04D127E01BEA000B00F01D81F6
:1086F0000133DBB29C08A9FB04B4C4EBC404A3EBB4
:108700008404E4B253450EFA04FBEDDBFF240020A1
:1087100085F88C0B00238CF8BE3054E795F88C4B11
:108720004C49A308A1FB0313C3EBC303A4EB8303CE
:108730000121DCB28CF8BE101B2C40F0CC8021460D
:108740004FF0000E85F88CEB00283FF43CAFE1E7DA
:1087500095F89A0B95F89BCB95F89C1B95F89D3B4B
:108760008444614495F89ECB0B4495F89F1B9C4430
:1087700095F8A03B61440B44FF2B04D9190A51FA28
:1087800083F3FF2BFAD895F8A11BC3F1FF03DBB2EB
:10879000994200F0F980FF22002384F8BD2085F87B
:1087A000953B46E7DFF8B49019F83430990881EA30
:1087B00053015940490101F020011943CB0883EAD4
:1087C000910383EA11139B0149B203F040030B4369
:1087D000C3F38501C3F303104840D9B20FFA84FAFA
:1087E000414043EAC11309F83A30136810461B6848
:1087F0007E219847D5F8280B19F83A10036809EB41
:10880000C4041B6804F1010A984708344FF0000BB8
:1088100007E0494698470BEB0901A2451FFA81FB87
:108820001ED01AF8019BD5F8280BA9F17D03012B66
:1088300003684FF07D011B68EBD89847D5F8280BEB
:10884000036889F020011B689847E4E7505700202F
:10885000080A002025499224086400208C62002028
:10886000D5F8280B5FFA8BF1036801EB1B21C1F1EE
:10887000FF011B68C9B2984795F8382BB84B0132F5
:10888000A3FB0213DB0803EB8303A2EB430385F88E
:10889000383BA8E600238CF8BE3095F8944B1B2C8F
:1088A00012D84FF0010A0AFA04F3034243D101340B
:1088B000E3B202E019EA000F3DD1DCB21B2C0AFA48
:1088C00003F903F10103F5D90024012385F8944B42
:1088D0008CF8BE30F2E6A30883EA540363405B01E0
:1088E00003F0200361B241EA030ECEF3C409CEF3D4
:1088F000850383EA0903CEF3031983EA09039B0185
:1089000003F040034EEA0303C3F3850EC3F30319D8
:108910008EEA09095FFA83FE8EEA090E013443EA02
:10892000CE135FFA84FEDCB20CE71B2C71D185F804
:108930008CBB2146EEE61B2C61D0630883EA9403CE
:1089400063405B0161B203F020030B43C3F3C40E29
:10895000C3F3031080EA0E00C3F3850E80EA0E0015
:10896000800100F040000343C3F30310C3F3850EFE
:1089700080EA0E0ED8B280EA0E00013443EAC0133A
:1089800085F8944BDCB21EE6D5F8241B5FFA82FC16
:10899000012303FA0CF30B43C5F8243B00283FF4F2
:1089A000FAAE10287AD1B5F89B3BB3F5407F00F0C2
:1089B0008E8055D8B3F5807F00F0C280B3F5887FF4
:1089C0000ED1D5F89D3B95F895115B001BB21A2985
:1089D000A5F8E03B08BFC5F89C31624BC3E91067BE
:1089E0006149C2EBC202AB18D1F800C088888A790D
:1089F000C3F8F0CBA3F8F40B83F8F62BCBE60023F7
:108A0000F34585F8943B60D001238CF8BE302146B5
:108A1000D9E5A30883EA540363405B0161B203F024
:108A200020030B43C3F3C40EC3F3850080EA0E009A
:108A3000C3F3031E80EA0E00800100F040000343F0
:108A4000C3F3031EC3F3850080EA0E005FFA83FEC2
:108A50008EEA000E43EACE13601CC0B2DCB257E6C9
:108A6000B3F5616FBCD1D5F89D3B95F895E1190A36
:108A7000180C4FEA136CBEF1190F85F8C21B85F86C
:108A8000C00B85F8C1CB05D1C0B2C9B2C5E9680138
:108A9000C5E9663C334BC3E90867A1E795F8B43CE8
:108AA000092B3FF678AE304908F833C008EBC30213
:108AB000D1F800C088888979C2F801C0013385F8EF
:108AC000B43CA2F80500D17165E621467BE5D5F8F6
:108AD0009D3B03F00F0104292ED8C3F30310062891
:108AE0002AD895F8959185F8A80BC3F30B2C05EBC4
:108AF000410E1B0D4FEA4C0C5B00B9F1180FAEF89C
:108B0000AACBAEF8AC3B17D1B5F9AA1BB5F9AC3B73
:108B1000C5F89C11C5F8A031B5F9AE1BB5F9B03B4D
:108B2000C5F8A411C5F8A831B5F9B21BB5F9B43B25
:108B3000C5F89801C5E96B130A4BC3E904674FE711
:108B4000D5F89D3B95F8951103EB83031A29C5F8D9
:108B5000D03B08BFC5F89831024BC3E90C673FE72B
:108B6000CDCCCCCCF8620020EA62002030B4164DA7
:108B700095F8383B95F8394BA34286BF04F10A02B9
:108B8000D31AE31ADBB20A2B1AD0104A104B02F8A0
:108B90003400601C02EBC402A3FB0043DB080C683A
:108BA000C2F8014003EB83038C888979D171A0EB73
:108BB0004303A2F8054085F8393B012030BC7047DB
:108BC000002030BC704700BF505700208C6200204E
:108BD000CDCCCCCCF8B5164E96F8B45C2DB306F6D9
:108BE000B8473B46002205E00132D4B2A54203F16A
:108BF000080318D917F832408442F5D11C46013DCC
:108C000054F8010F0860EDB2A088A4798C71AA1AFB
:108C10008880D20003F10801184686F8B45C50F051
:108C2000B8FD0120F8BD0020F8BD2846F8BD00BF02
:108C3000505700201B281BD830B40F4C0122D4F809
:108C4000245B02FA00F32B400ED0C0EBC003234498
:108C5000D3F8F00BB3F8F44B93F8F63B08608C8034
:108C6000104630BC8B7170471A46104630BC7047B6
:108C700000221046704700BF5057002030B54FF417
:108C8000000085B01EF0FCF818B3134C90F90400F6
:108C900094F8082D94F8093D002A14BF08220022F8
:108CA00083F001031A434FF4614100230325CDE90A
:108CB000015200911A464FF400011DF017FF48229F
:108CC0000346002104F6A830C4F8283B50F07BFD91
:108CD000012005B030BD00BF50570020F0B46D4EEC
:108CE00006604FF4C0766C4CA0F8C2604FF04C1692
:108CF0006A496B4AC0F866604FF02C16694D6A4BA2
:108D0000C0F86A60C0F86E404FF4C176C0F87A10BF
:108D1000A4F5DE046549A0F89A600E3C40F2731693
:108D2000C0F8AA50C0F8AE30614D624BC0F8B22016
:108D3000C0F8BA10A2F127125F49C0F8B640A0F8F7
:108D4000BE60A4F127145D4EC56503665C4D5D4BA6
:108D5000C0F8C82002F1D612C0F8CC40C0F8D2103A
:108D6000C0F8D6608239C0F8DA50C0F87230C0F866
:108D70007630C0F88230C0F88630C0F88A30C0F84B
:108D80008E30C0F89230C0F89630C0F89E30C0F8EF
:108D9000A230C0F8A630C0F87E20C0F822204A4A8F
:108DA000C0F8E21004F16D14A6F14A1601F1046155
:108DB000464D474BC0F8DE40A6F57F46454CC0F80F
:108DC0001A2001F6410102F5B8126C32C0F80A60AF
:108DD000C0F80E50404E414DC0F81240C0F8161079
:108DE0003F4C4049C0F81E303F4BDFF818C13F4FA1
:108DF000C0F82660C0F82A503D4E3E4DC0F82E40C7
:108E0000C0F832104FF0A1143B49C0F83620C0F82A
:108E10003A303A4A3A4BC0F8E6C0C0F80670C0F89B
:108E20003E60C0F84250C0F84A10C0F84640C0F852
:108E30004E20C0F8523000F1F20100F5727700F1D7
:108E4000F005C0F1040600F1040C7318002B01DDDD
:108E50008C4514D80C46024652F8043B23F00823F4
:108E6000954244F8043BF7D1B0F8F03023F40063A6
:108E7000A1F8F030F2318F42E7D1F0BC7047821E8A
:108E80008C1E32F8023F23F40063954224F8023F1F
:108E9000F7D1EFE717080C080101820182014201B6
:108EA000B300D30037005300730093003301530124
:108EB000C300E300F700D700A30041006100820176
:108EC0009801780182018201370060098D09540000
:108ED000010842014108C8002F00920180016E0183
:108EE00021004C00B700F8009701A109C808C80884
:108EF00040012C0046005200C100E100A1004100E9
:108F00000101E100610081002DE9F0412DED048BAC
:108F1000027B0589478902EB4203A5EB830584B0F8
:108F200005EBD575044602EB82029B006D10884666
:108F300003935600B0EE408AB0EE609A3EF026FEF3
:108F4000039B00972946204600223EF049FE039BE2
:108F500000972946204600223EF05EFAB8F1000F45
:108F600054D0012120463EF059FE012120463EF01A
:108F700043FEDFED2B7A238962899FED2A0AC8EE32
:108F8000270A5B0852082046F7EE087A60EEE70AE7
:108F900007EE903AB8EEE78A07EE902AF8EEE78AF5
:108FA0003EF000FEB0EE490A20463EF0F5FDF0EE40
:108FB000680AB0EE480A20463EF0F4FD2368DB69FB
:108FC00013B1022120469847204604213EF01AFEA4
:108FD00071082046494200223EF0F0FD2046002262
:108FE0006FF005013EF0E4FD7108204600223EF0DE
:108FF000E5FD2046002206213EF0DAFD204604B0C1
:10900000BDEC048BBDE8F0413EF0BABD2046022124
:109010003EF004FE414620463EF0EEFDA9E700BFCB
:1090200035FA8E3C000000002DE9F04FAC4EAD4DFE
:10903000AD4FD5F800800FCE91B008AC0FC496E8C4
:109040000F00D8F8006084E80F00336C01223A70FA
:1090500033B1404602219847D5F80080D8F8006027
:10906000B368404698472868FF2388F80E300268A6
:109070009E4B4FF0010940F21711002688F80D9021
:1090800041810096546949464A46A047984B1B685F
:10909000180600F1498106220523CDE902234FF08D
:1090A00004084FF003094FF0020A05AC2868914B01
:1090B000026880F80BA01326002186720091566981
:1090C00001215246B04797F85C307869002B00F0D8
:1090D000F480013B012B0AD8874A884982FB003281
:1090E000C017C0EB6212B923204645F029F920468B
:1090F00049F070FFD5F800B00026DBF800308BF89F
:109100000BA014308BF80A00009652465846D3F84C
:1091100014A014212346D0472868794B026880F8B0
:109120000B904FF0130A80F80AA00096D2F814B002
:1091300001214A46D8472146B7F90E00EFF78AFFCA
:10914000204649F047FF6F4A2B681188215200F1F1
:10915000150219689A7283F80B9000964A461846D1
:10916000D1F8149023461421C8472868664B02683A
:1091700080F80B8080F80AA00096D2F814900121A4
:109180004246C8472146B7F91000EFF763FF224671
:109190005E49EC23204645F0D3F8204649F01AFFFB
:1091A000D5F800901430D9F8003089F80A0089F811
:1091B0000B80009642464846D3F81480142123467B
:1091C000C047286803990268C17280F80AA0009617
:1091D000D2F814804E4B89460A460121C0474FF40D
:1091E0007A720023D7E91C014AF036FD4AF09EFC52
:1091F000DFED487A484A494907EE100A67EE277AB8
:109200002046FCEEE77A17EE903A1FFA83FCA2FBA9
:109210000C3E4FEA5E13A2FB03825209C3EB031E0E
:10922000ACEB8E0EC2EB021C1FFA8EFEA3EB8C037E
:10923000CDF800E09BB245F083F8204649F0CAFE25
:10924000D5F800801430D8F8001088F80A0088F8A3
:109250000B90009623464A464C6940461421A0478D
:10926000286802990268C17280F80AA000965469C1
:109270002B4B88460A460121A04797F878302C6886
:1092800010AA02EB830353F8203C0293184649F0DE
:10929000A1FE216884F80B801430A0720096029B16
:1092A0004E69424620461421B047286803685B6C2B
:1092B00003B1984711B0BDE8F08F07EE900A9FED1B
:1092C000197A0E49F8EEE77A0F2367EE877A20467F
:1092D000FDEEE77A17EE902A45F032F807E700BF77
:1092E000CCAE06080832002098710020A031070893
:1092F000643D0120F43107081F85EB51083207084F
:109300001032070834740708243207083832070877
:10931000403207086F12833A8988888854320708D8
:10932000643207084B59063D2868644B026840F2D6
:10933000132141810096D2F814804946022205ACDF
:10934000C047B9884A46204605F08AF9204649F0C8
:1093500041FE9DF81430202BC1B240F08F8033467F
:109360000133DBB210AA1A4412F82C6C202EF7D06D
:10937000A0EB030CBCF1000F1E4640F39C80ACF147
:109380000900F62823447BD806A8834278D31968BD
:109390005B68CDE9051312F8243C8DF81C3020469B
:1093A00049F018FED5F800800026D8F800300222D7
:1093B000143088F80A0088F80B20009640461421E3
:1093C000D3F814802346C04728683D4B026840F21A
:1093D000133141810096D2F8148001210322C04745
:1093E000BB69642101FB03F1204605F073F92046B7
:1093F00049F0F0FDD5F800800322D8F8003088F855
:109400000B20143088F80A000096D3F814904046D8
:1094100023461421C84728682A4B026840F21341AA
:1094200041810096D2F8148001210422C047264BC6
:1094300093ED000A4DF09AF90146204605F04AF9ED
:10944000204649F0C7FDD5F800801430D8F8003028
:1094500088F80A00042288F80B2000965E694046CE
:1094600023461421B04709210823CDE902134FF008
:1094700007084FF006094FF0050A17E6844670B159
:109480000020024610AB1A44324403440130C0B2FB
:1094900012F82C2C03F82C2C60450246F2DB884293
:1094A000BFF47DAF4A1E121AD2B2013220442021ED
:1094B00050F089F973E70020F1E700BFB8310708E1
:1094C000CC310708E0310708D83100202DE9F04FF2
:1094D000A04E34682368DA6B91B09AB12046904769
:1094E000346870B9237A002B40F039822368204613
:1094F0009B6A984723682046DB68984711B0BDE80F
:10950000F08F2368DFF8849299F86420012189F8AC
:109510007910002A00F00E81002289F87A201A6C56
:1095200022B1204602219047346823689B68204678
:109530009847FF233168A3730B685B6B0127677340
:10954000002B4CD007A89847002848D0BDF81E2013
:109550009DF81C300421CDE900320A207E4B7F4A61
:1095600046F0F6FABDF81E30B3F5807F40F2D180A8
:109570003468637A063B03EBD373C3F34703059365
:1095800040F2071A4FF0000B0599AAF1060517E003
:10959000934220463A4688BF01F1010809D8D4F821
:1095A00000C084F80A80E772CDF800B0DCF81840FB
:1095B000A0470135AA455FFA88F100F0D7813468E9
:1095C000628A01F10108ABB2002AE1D12046CDE95F
:1095D00003313EF0A9FBDDE90331628AD8E7BDF82B
:1095E0001E209DF81C300421CDE900320A205C4B7E
:1095F0005A4A46F0ADFA30685A4B417A04680C3941
:10960000C1F3470101F10C05857203220025C272E6
:1096100000956469A0474FF007084FF0060A052738
:109620000425514A514908A844F08AFE08A849F087
:10963000D1FCD6F800B00024DBF800308BF80B50DA
:1096400005308BF80A00009458462A46D3F814B027
:10965000052108ABD8473068454B0168C772142212
:10966000827200943A464F690721B8473068414BEF
:10967000016880F80BA01527877200945246D1F834
:1096800014A00B21D04730683B4B0168877280F8EB
:109690000B8000944F6942460B21B84799F89830E7
:1096A000002B75D1306803685A6C12B1904730684E
:1096B00003689B6A9847314B5B68C3F30803A3BBFD
:1096C000EFF311838BBB2E4A2E4C1368A0681168F0
:1096D0008B42FAD1D9F89C108842F6D8D9F8A0105C
:1096E0004FF47A7404FB01F2101AB0FBF1F0002180
:1096F000E4FB030102460B4623490020511843EBCB
:1097000000000122C9E92A1089F8B02011B0BDE893
:10971000F08F9DF81C30002B3FF46DAF4FF0070821
:109720004FF0060A052704257BE73DF08BF902463A
:109730000B46E1E79A6C002A00F01681214609F1F8
:109740007C009047002840F022813468236889F823
:109750007A00E4E6083200201C590708783207082E
:10976000BC510708A03207083C2B0708B032070895
:10977000C4320708D4320708E032070800ED00E0E1
:10978000A822002010E000E000093D0098710020B0
:1097900030688B4B02680D2105F10508817280F855
:1097A0000B800094546904214246A04799F85C302C
:1097B000D9F89020002B00F0C680824B8249A3FB91
:1097C0000232920908A844F0BBFDBA238DF8253077
:1097D000002708A88DF8267049F0FCFB3468133088
:1097E0002368A07284F80B80009742462046D3F885
:1097F0001480132108ABC0473068744B0268AC1D5D
:109800000F218172C4720097D2F81480042122467D
:10981000C047D9F88C306E4A6E49A2FB03035B093E
:10982000A2FB03025209C2EB0210A3EB800308A8BB
:1098300044F086FD08A849F0CDFBD6F8008013302F
:10984000D8F8003088F80A0088F80B4000972246C4
:1098500040465C69132108ABA0475F4B1A6840F68D
:10986000020393437FF41EAF30685C4B0268DFF85D
:10987000808105F1070A1121817280F80BA0009701
:10988000546904215246A047D9F894300097A8FBA8
:1098900003230424D9083A460223019408A804F0BB
:1098A000ADFF08A849F096FB4D4A336811880DF1C9
:1098B000200C00F115022CF8001019689A7283F838
:1098C0000BA0009752461846D1F814A06346142105
:1098D000D0473068434B0268083513218172C57246
:1098E0000097214654692A46A047D9F89030002BAA
:1098F0005ED0344A0097A2FB03230320D9F89420BA
:1099000001909B09B2FBF3F3A8FB0331C1403A4637
:10991000022308A804F072FFAC22AD2308A88DF83A
:109920002320ADF8243049F055FB34681530216808
:10993000A0720023E57200932A4608AB20464C69CA
:109940001521A047AEE6284B1F49A3FB0232520A5D
:1099500008A844F0F5FCBB238DF8253038E7637A7E
:10996000002B7FF4C7ADC1E51046F0E60AF1060A08
:1099700040F21F1301379A45FFB201D0346803E665
:109980004FF009084FF0080A0727062549E6627AD2
